:020000040800F2
:1000000000A00020F90B0108610C01082DFC00087C
:10001000610C0108610C0108610C0108000000007E
:10002000000000000000000000000000610C01085A
:10003000610C010800000000610C010833ED0008AC
:10004000610C0108610C0108610C0108610C0108D8
:10005000610C0108610C01087966000875660008EA
:10006000610C0108610C0108610C0108610C0108B8
:1000700085570008610C01080FC40008610C0108D5
:10008000610C0108610C0108610C0108610C010898
:10009000610C0108610C0108610C0108716600081F
:1000A00019C0000855C0000809C0000879C0000840
:1000B00049C0000839C0000829C00008610C0108C7
:1000C000610C0108610C0108610C0108610C010858
:1000D000610C01089DC2000891C2000885C2000899
:1000E00041ED0008610C0108610C0108610C010878
:1000F000610C0108610C0108610C0108610C010828
:10010000000000000000000000000000610C010879
:10011000610C0108610C0108610C0108610C010807
:10012000610C0108610C0108610C0108610C0108F7
:10013000610C0108610C01080000000000000000D3
:10014000610C0108610C0108610C0108000000004D
:10015000000000000000000000000000000000009F
:100160000000000000000000610C0108610C0108A3
:10017000610C010800000000000000000000000009
:0801800000000000610C010801
:100188002DE9F04F2DED068B6B4F6C4B3B60AFB0FC
:1001980000237B600DF049F918B90DF069F909F0F1
:1001A80029FF09F0E5FF664A664C137843F001031E
:1001B8001370654B4FF47002C3F88820002309932D
:1001C8000A93236843F480332360236803F40033DD
:1001D8000A93099B013309930A9B1BB9099BB3F541
:1001E800A04FF2D1236813F4003318BF01230A93F8
:1001F8000A9B012B6AD0544E544BF360636ABB6070
:10020800636ADFF878B1DFF87881DFF878A143F026
:1002180080736362636943F4FC032EAD6361032357
:100228008DF86A3041F6FF7325F8503D4FF0904045
:10023800294605F097FB4FF6FF7358462946ADF857
:10024800683005F08FFB4248294605F08BFB414892
:10025800294605F087FB4048294605F083FB2946D7
:100268003E4805F07FFB284608F000FC3C4A1A9BF4
:10027800B3FBF2F33B4A3C4813600021102212F012
:10028800CAFE3A4B3A4A5A60F02286F823200022E6
:100298009A60384E07221A60B368CAF8003098E8A6
:1002A8000300636985E8030043F48023636108233E
:1002B800CBF818301A981BA905F054FBDAF800306F
:1002C80013F0080FA8F10C0829D163E02A4B122279
:1002D8001A606368636063686360636843F480639B
:1002E8006360636823F47C136360636843F4E81312
:1002F8006360236843F0807323602268114B900188
:10030800FBD55A6822F003025A605A6842F002028A
:100318005A60636803F00C03082BFAD16BE796F870
:100328009031012B36D8044B96F891219B6813F035
:10033800805900F0F1852DE0D8000020EB980008E6
:10034800AC2F00200010024000ED00E00005FA0587
:1003580000080048000C004800100048001400483D
:1003680040420F00082C00200C2C002010E000E078
:100378003F190100D0160020002002400004004868
:1003880064490108A82B0020BE4B002283F8912164
:100398000AF090F864200EF0BEFCBB4800214FF430
:1003A8008C7212F038FEE369B84843F00703E36142
:1003B800A36943F4E123A361636943F4C023636140
:1003C80000F58874837B416890F80FE003F007021A
:1003D800DB0801EB83039200196A4FF00F0C0EFA49
:1003E80002FE0CFA02F221EA02021A62196A1030BD
:1003F8004EEA0102A0421A62E4D10022A449002375
:1004080053540132112AF9D1A24AFF2199540133D8
:10041800072BF9D1A04BDAF80040A04A1A60A0488F
:1004280000213C2212F0F7FDC4F3801905234FF098
:10043800000E9C4A9A481EF802100C2202FB0EF28B
:100448001154B9F1000F07D11E3901299FBFFF21AF
:1004580003F1FF331154DBB20EF1010EBEF1050FAB
:10046800E7D1914A96F805B01370904B904983F8FC
:1004780000B0904B7B62C0330B608F4B8F4A03EB0D
:10048800CB03A1065B7848BF0123936200238C4A03
:1004980040F2DC5122F813100133082BF7D113A8CE
:1004A80000211C2212F0B7FD14F4007A1DBF854B01
:1004B80019950393CDF80CA0BBF10E0F03D00BF0E8
:1004C800EF03082B02D101238DF85E30022007F0DC
:1004D800FFFC18B14088003018BF0120C4F3400366
:1004E8008DF85230C4F340338DF84C30C4F3C03328
:1004F80000F001008DF84F3014F400638DF85100BE
:100508008DF8559007D096F8843103F1FF3EDEF15F
:10051800000343EB0E038DF85030C4F300438DF80D
:100528005630BB6AB6F844E1ADF862E01AF1000A49
:1005380018BF4FF0010A003318BF01238DF8583057
:10054800C4F300538DF85930B6F84631ADF85C3035
:10055800B6F85231ADF85A30C4F380438DF85330B1
:1005680096F854318DF857A0181C04F00101C4F313
:10057800C00218BF0120E40448BF424C8DF8540063
:10058800B6F8500144BFB4F84C41ADF86240B0F53C
:10059800FA7F8DF84D108DF84E20ADF8600002D925
:1005A8000BB9ADF8623096F8D431474887F82C304B
:1005B800002387F82D3043709DF85E30002B0CBF68
:1005C8000023022301B902B1013308EB83084FF07D
:1005D8000009D8F81430A3F1020A203304933AF83A
:1005E800023F4FF6FF72934200F0C5819DF851100B
:1005F800DAB21B0ADEB279B12448344C00EB02109F
:100608004168A14208D10189B1F5806F00F0AF813E
:10061800B1F5006F00F0AB819DF8551031B11101B3
:100628001A4840582A49884200F0A1819DF856107E
:1006380079B11101154C6018645826498C4200F0B4
:1006480096814168B1F1904F03D1817B082900F070
:100658008E819DF8521051B10C4800EB0210416890
:10066800B1F1904F03D10189102900F080819DF8E4
:100678004F10A9B30548154C00EB02104168A14280
:100688002ED129E0D0160020502C002090660108B9
:10069800E4000020F5000020C01E0020BE18002045
:1006A800C41E0020287501082C100020A008002076
:1006B800E42D0020E01600203C730108D80000203B
:1006C800D80F0020584901080501002000040048FF
:1006D80000040040002C01400189042900F04781F2
:1006E8009DF8501051B1B94800EB02104168B1F1C2
:1006F800904F03D10189202900F03981199C7CB1E0
:10070800B24F216807EB02177868884208D1398907
:10071800A088884200F02B81E088884200F0278179
:10072800022B02D19DF84C3003E0012B04D19DF837
:100738004D30002B00F01B819DF85810A34B17017A
:1007480059B19DF85E1041B9A2F10E01012904D8F2
:10075800D9599F48814208BF04269DF85910DC19D1
:1007680031B19DF85E1019B9043A032A40F2E780C6
:10077800012E49D1DFF864820693D919FF2291F836
:100788000DE088F8742088F875204868C8F8844017
:1007980001F108020989ADF868104FF0000B022139
:1007A8008DF86B1088F878B01AA98DF86AE0059270
:1007B80088F830B0C8F834B0C8F838B0C8F83CB0D9
:1007C800C8F870B088F876B088F877B005F0CAF83D
:1007D800069B059AD85991785A4604F079FF204625
:1007E800594632460BF09AFC7A4BC8F888307A4B57
:1007F800C8F88C30C8F890B0204608F1880108F194
:100808008C020BF0E1FCB2E0022E4BD15FFA89F3C7
:100818001C2101FB03FC714BCDF81CC003EB0C0B36
:1008280001238BF878300693684B8BF87990D919A7
:100838004FF0000891F80DE048688BF87A8001F1D4
:1008480008020989ADF868108BF882801AA9CBF8DC
:1008580084408DF86AE005928DF86B6005F082F8A7
:100868005A4B059AD8599178424604F031FF069BB5
:1008780020461A4641460BF051FC584BDDF81CC087
:10088800574ACBF8882003EB0C01564ACBF88C204A
:100898008831CBF8908020460A1D0BF095FC09F1B1
:1008A800010964E0032E48D19DF853304B4E4E4F5A
:1008B800E3B19DF85430DFF8408196F82EB053B17B
:1008C8004A4BBDF86020B3FBF2F22046082192B2F1
:1008D800BDF8623003E0204608214FF6FF7205F0AC
:1008E8006AF847F82B00C0F80C8020E0BDF86020BB
:1008F80096F82E80BDF86230B2F5FA7F0BD93B49E5
:10090800B1FBF2F22046082192B205F054F8384BB8
:1009180047F828000AE03749B1FBF2F220460121E6
:1009280092B205F048F8344B47F82800C36096F8AF
:100938002E30013386F82E3019E0042E17D1274EB9
:10094800BDF85A2096F82D702A4B93FBF2F22046F8
:10095800BDF85C30012192B205F02DF896F82D30E3
:1009680006EB87070133C7F8580186F82D30049B3A
:100978009A457FF434AE194E204B96F82D2086F810
:1009880078211F4A1778A7F117020024022A1C7041
:100998009E4639D8736A2344D3ED007AF5EE407A3F
:1009A800F1EE10FA03D1B36A002B4CD144E0154A9A
:1009B80004EB020C0FCB8CE80F009EF800301034CB
:1009C8000133C02C8EF80030E4D1ECE790660108C2
:1009D800004001406D5400084D550008D800002023
:1009E80015570008455400081C2C002000127A00F6
:1009F8006D55000840420F005D5500084C2C002042
:100A0800A0080020DC0700203A4B13F837808EF846
:100A1800008003EBC703D3F80490B9F1000FC2D0EC
:100A28004445C0DA344A230103EB020C4B440FCB94
:100A380001348CE80F00F3E7304B1A6812F4805F3A
:100A4800994626D11FE02E4B2E4A13F83700107016
:100A580003EBC7035C68002CEED000238342EBDA7B
:100A6800C3EBC3016218DFF8A880D2F8009041F800
:100A7800089001EB080C9188ACF8041092798CF876
:100A880006200133EAE707F0EF03082B1E4B20D1BD
:100A980021E09EF80020012AF5D91C4B03EB021235
:100AA800103210339342EED053ED047AB6EE007A4A
:100AB80067EE877A43ED047A53ED057A67EE877A15
:100AC80043ED057A53ED037A67EE877A43ED037AAF
:100AD800E7E70E2F08D11A7842F010021A70182F83
:100AE80018D10EF041FB15E01A7822F010021A70A6
:100AF800192FF5E73C730108DC070020A82B00201C
:100B0800E4500108702D002000280020E407002090
:100B1800712D00200EF00CFBD9F80030B24CB34810
:100B28005F0358BFB24BB34F5CBF01221A70B24A81
:100B3800137843F0040313704FF40043ADF86830A2
:100B480063694FF0020843F400234FF0010B8DF85E
:100B58006B8029468DF86AB0636104F003FFA74BE8
:100B6800A74A1A6000200EF0FDF8E36943F48043B9
:100B7800E361236943F480432361636943F4802379
:100B880063617B6A23F470037B627B6A43F4A0038E
:100B98007B627B6A23F070637B627B6A43F0A063AD
:100BA8007B627B6A23F070437B627B6A43F0A043DD
:100BB8007B627B6A23F470237B627B6A43F4A02305
:100BC8007B624FF460431A938DF86C8003234FF0D7
:100BD8000008384629464FF4805A8DF86D30049342
:100BE8008DF86E808DF86F800DF0A6FE049B8DF851
:100BF8006D3038462946CDF868A08DF86CB08DF870
:100C08006E808DF86F800DF097FE236943F4804362
:100C18002361236923F4804323617A4B9A8822F461
:100C280080521204120C9A809A8892B242EA0A02FE
:100C38009A801A8802F4415242F4457242F0030243
:100C48001A809A8822F470621204120C42F4E0624C
:100C58009A809A8B22F400621204120C9A8307225B
:100C68001A821A8892B242F040021A80C7F818A075
:100C7800D9F8003003F41073B3F5107F00F09E80AC
:100C8800614B624F1F606369DFF8689143F480230A
:100C98006361E36943F40013E361236B23F01003FA
:100CA8002363236B43F010032363D9F8203023F028
:100CB8007063C9F82030D9F8203043F08063C9F850
:100CC8002030D9F8203023F07043C9F82030D9F803
:100CD800203043F08043C9F820304FF000084FF02F
:100CE800020C4022484629464FF0030B8DF86CC091
:100CF800CDF818C01A928DF86E808DF86F808DF837
:100D08006DB00DF019FE8022484629461A920DF062
:100D180013FE3A68DFF80C9122F001023A60396854
:100D28003B4A0A403A603B4A3A613A6842F001025B
:100D38003A60C7F80880C7F80C80C7F80880BA6816
:100D480042F40042BA603A683A607A6822F078421F
:100D580022F400427A603A6842F001023A60D9F817
:100D680000502D4F05F400434FF0100A04935246EB
:100D780005F4006338464146059312F04CF94FF6E6
:100D8800FF72DDF818C00E9215F002058DF83DC00F
:100D98008DF83E808DF83F808DF83CB044D02EA968
:100DA8004FF0904041F880AD0DF0C6FD01250723B6
:100DB8003D7087F80180FB70BD7035E0174A1378E5
:100DC800174918F901001F2802BFFF2008F8010081
:100DD80003F1FF3308F10C0808BFDBB2B8F13C0F90
:100DE800EED113704CE700BF001002400008004825
:100DF800080D002000040048AC2F0020BC2F002064
:100E08003DEC0008003800409C0F002000540040D2
:100E1800FFE0CF00300E5000F82A00202C100020F0
:100E2800C41E0020A82B0020049B7BB12EA90423FC
:100E380041F8803D92480DF07FFD0C233B7107235C
:100E4800FB7101237D711D44BB71EDB2059B83B11C
:100E58002EA9202341F8803D4FF090400DF06CFD05
:100E680002233B730723FB7301237D731D44BB736C
:100E7800EDB2E36A834823F4F873E362E36A43F468
:100E8800D873E362636943F0805343F002036361FC
:100E980007F09BFC1AA807F06DFC7B4B1A937B4B61
:100EA8001B93012D4FF0000394BF1A4680221F9216
:100EB8004FF48072734C20924FF48062219220226A
:100EC800204622921AA94FF400521C931E93239293
:100ED8002493ADF8745007F05AFC236843F00103DB
:100EE80023606B4CA36823F04053A360A36843F0CE
:100EF8008053A3600A200DF00EFFA36823F08043FF
:100F0800A360A368A360A36843F00043A360A2683A
:100F18005F4B002A31DAFAE7531E092B3FF63AAA4B
:100F2800D8F8400028602946584604F01BFD4FF4C5
:100F38000063CBF818303C200DF0EDFE96F89131A7
:100F48009945BFF621AADFF838B108224FF40063AB
:100F5800CBF8182078200492ABF8283003930DF0D2
:100F6800CFFE049A039BABF828207820CBF81830E2
:100F78000DF0C6FE09F10109E0E79A68454922F03B
:100F880040529A609A6842F000529A608868424AD1
:100F9800024042F468328A60D968404A0A4042F402
:100FA8000052DA601A6B013D22F00F0215431D63EF
:100FB800002101237A189078002800F084805C1CB6
:100FC800042B17F801E0D278DFF8C4C0E4B20ED8D9
:100FD80003EB4303DCF830505B001F20984025EA00
:100FE80000000EFA03F30343CCF8303031E0092B4C
:100FF8000ED80620053B4343DCF834501F209840A8
:1010080025EA00000EFA03F30343CCF8343020E05D
:101018000E2B4FF006050ED8A3F10A006843DCF842
:1010280038801F23834028EA03050EFA00F32B4378
:10103800CCF838300DE00F3B05FB03F0DCF83C80C2
:101048001F23834028EA03050EFA00F32B43CCF84C
:101058003C30BEF1090F0E4822D983698569AEF18B
:101068000A0303EB43034FF0070E0EFA03FE25EACB
:101078000E05856185699A402A43826122E000BF96
:10108800000400480804024040010050082B0020DA
:101098000001005000030050E010FCFF07C0FFFDF6
:1010A800436945690EF1FF3303EB43034FF0380EF4
:1010B8000EFA03FE25EA0E054561456903339A4099
:1010C8002A4342612346043110297FF473AFA24BAF
:1010D8009A6842F001029A601A4611689E4BCC0742
:1010E800FBD5DA689D4C22F00202DA60DA6842F039
:1010F8000202DA60DA6842F00102DA609A6842F0C5
:1011080004029A60B4F85831002B40F00C87B4F907
:101118005A21002A40F00787B4F95C21002A40F0E0
:101128000287DFF894828E4DD8F800308D48B3F8E6
:101138006230049300210C22002794F85FB194F8E0
:101148006AA111F068FF00211422874811F063FF9B
:1011580039460C2286F8797105F5BE7085F87A71E2
:1011680011F059FF814BC6F8883123200DF0D3FDCB
:10117800752001210BAA0AF081FD002862D07C4B62
:10118800C5F880317B4BC5F88431384643230121AB
:101198000CAA85F87C310AF071FD9DF8303003F017
:1011A8007E038DF8303040B1682B06D1012385F8D5
:1011B80079311D2385F87C3144E09DF82C3003F00B
:1011C8007E03682B8DF82C3037D10223062086F851
:1011D80079310146D6F880311AAA98479DF86D10E2
:1011E80001F001029DF86B1001F001014B0043EA88
:1011F80082019DF8692002F001030B430AD05BB21B
:10120800012B01D1002302E0022B0FD1012386F824
:101218007A3117E0524B0C20D3F8803101210EAA05
:1012280098479DF8383013F00F0303D103200DF0D1
:101238009FFD07E0042BE9D1E4E7702B04BF0423EA
:1012480086F8793196F879214B4F0023022A3B70B2
:1012580013D1454D494B2B60494B6B60494B4A496B
:10126800EB604A4B2B61042308683B70484B1A70AB
:1012780040F001020A609E4603E001200DF078FD6F
:10128800FBE05A460A2A28BF00220123934040F275
:10129800B23C03EA0C0CBCF1000F17D113F04D0F50
:1012A80014D0304B3B4A1A603B4A5A6096F87A2170
:1012B800002A0CBF6F226E221A72384B04221A7051
:1012C800032318438EF80130086006E0012A4FF026
:1012D800000BD6D8314B83F800B0BAF1040F6DD8A3
:1012E800DFE80AF003770303030096F88CB1DFF810
:1012F80070A0BBF1000F40F00E8614200DF00BFD1E
:101308000AF28D137620D021012204F041FC9AF8CC
:101318008D31582B5DD10AF5C873882118227620A3
:1013280004F036FC31227620F42104F0ADFC0123D0
:101338008AF88C311A4B1B4A9A601B4A5A6045F648
:10134800D8125A80194ADA60194A1A61194AA3F858
:1013580000B05A6100F0DFBD00010050D016002037
:10136800D8000020DC280020082700207C4901083C
:1013780085BC0008A5BC00081C270020C1BD0008CA
:10138800A9BB00088DBB0008A40F002090C1793DBF
:101398006400002061BE0008F1BB0008D42F0020C3
:1013A8001406002089BB00088BBB00089BBC000802
:1013B80039BC0008C5B90008E80F0020BAF1010FD0
:1013C80007D0254B254A83F802A0136843F004038D
:1013D8001360224B1A6812F0020F9A4602D0204B73
:1013E8001B6898471F4B4FF47A724FF0000B1A6036
:1013F80086F8ACB12B68BC2098471B4B94F8552154
:1014080083F800B002B13A7094F856210AB117492E
:101418000A7094F8572102B11A70DAF800301807E8
:1014280028D5BDF91010DFED126A642291FBF2F3A2
:1014380002FB131212B207EE902AB8EEE77A07EE13
:10144800903AF8EEE77AE7EE267AB2EE047A67EE9B
:10145800877AC6ED6C7A10E064000020A40F0020A3
:10146800DC28002024100020D02F0020D42F0020BA
:101478008988883C0023C6F8B031B84A137843F00D
:1014880002031370B64B08229A610A25B44EB38A38
:101498009BB283F00803B38219200DF03CFC0120B5
:1014A8000DF060FC19200DF036FC013D00200DF018
:1014B80059FC15F0FF05E9D10823B361A94B9FED4D
:1014C800AA8A1E68DFEDA98A337B00EE103AB8EECF
:1014D800C00A20EE080A08F02BFDA54B83ED000A90
:1014E800A44B1B8807EE903AF8EEE77AB7EE007A3D
:1014F800C7EE277AA04BB0EE680AC3ED007A9F4B7F
:10150800D3ED047A9E4B67EE887AC3ED007A337880
:101518009C4E07EE903AF8EEE77A9B4BC7EE277A97
:10152800C3ED007A77EE677A984BC3ED007A984B53
:1015380083ED027AC3ED008AC3ED018A954B83EDF2
:10154800027AC3ED008AC3ED018A08F0F1FCB0EE1F
:10155800408AB0EE680A08F08BFC20EE006A68EE5C
:10156800086A66EE007A8C4BE6EE887A3046FF21F0
:1015780020EE087AC3ED007A67EE007A1B22F0EEBF
:10158800675AD7EE085AE7EE087A28EE468AC3ED7E
:10159800015AA6EE808AC3ED027A83ED038A7F4B57
:1015A8001D7011F038FD35707D4D7E4B2A68012184
:1015B80012F0020F18BF717019701FBF0321197044
:1015C8000221B170510748BF1978304641BF4E1CFF
:1015D8001E700326465412F00A0F0CD01A78042104
:1015E8008154511CC9B205264654D11C0232D2B2CC
:1015F800197006218154D9F800108A0641BF1A785B
:10160800561C1E70072648BF86546679082E01D0DE
:101618000E2E04D11A78571C1F700B2787541A787E
:1016280011F4803F4FF00C0E00F802E002F10107C0
:101638001CBFDFF870E10232FFB21F701FBF8EF8C7
:101648000020504A4FF00E0E02F807E04A0741BF4B
:101658001A78571C1F70102748BF87541A78571CD0
:10166800FFB24FF0120E11F4806F1F7000F802E005
:101678000ED094F818E2BEF1000F09D0DFF824E18B
:1016880002328EF800203F4A4FF0130E02F807E0AE
:101698008F0541BF1A78571C1F70152748BF8754FC
:1016A800182E0DD11A7816278754571CFFB24FF001
:1016B800170E00F807E0D71C0232D2B21F7086540A
:1016C8000E0341BF1A78561C1E70192648BF86544F
:1016D800CA0541BF1A78511C19701A2148BF815494
:1016E8001A78511C197014238354002198222E480B
:1016F80011F091FC06F00BFF2C4B2D492D48196079
:101708002D4BB4F84E2101602C491A8000232C4A35
:10171800D8F800800B70B4F89611138093701FFAF4
:1017280081FC08F18502274E27483768DFF89CE0DE
:1017380020F813C007F596774EF823700133122B63
:10174800F1D1D9F800E01EF4805F08BFB4F89CC15D
:10175800A0F806C008F1D5073AE000BFAC2F00207A
:10176800000400480428002035FA8E3C00000000E0
:10177800FC2700200C000020B427002008270020A8
:10178800B8270020B10F00201828002008280020C2
:101798001C2800200C280020EC270020722700209D
:1017A800A40F0020B00F002038160020080F0020DA
:1017B80058180020A42B00200C0F0020430E0020F6
:1017C800DC2B0020D82B0020AC2B00208C0E002016
:1017D8001378F3B992F802C0D3789C4519D2BCF1BA
:1017E800000F08D00CF1FF3C0CEB8C0C0CEB8C0CB4
:1017F8000CF5617306E0013303EB830303EB83030A
:1018080003F5617392F801C00CF1040C9BB220F847
:101818001C300432BA42DBD11EF0080F00F0E4801D
:1018280094F89031062B00F2D980DFE803F0040722
:101838000E35506F6F0045F2F05201E042F6F82283
:10184800434B1A8006F011FFC7E0414B42F6F822DD
:101858001A8009010A2391FBF3F10023A1F5B06175
:101868003C4A42F823100133122BF9D13A4A3B493A
:1018780011603B4A4020137006F004FC002800F079
:10188800AD8001234FF0070E90F90000354A8DE82E
:1018980008404021344B9BE02D4B42F6F8221A8039
:1018A8002D4B324A1A602E4B102240201A7006F037
:1018B800E9FB002800F092800123002790F900003E
:1018C8002B4A8DE8880040214FF4E13380E0204B1B
:1018D80042F6F8221A80204B264A1A60204B08222A
:1018E80040201A7006F0CEFB002877D00123002490
:1018F80090F90000204A8DE8180040214FF4E133A8
:1019080006F096FA1D4BC3F8B40163E0104ADFF8FD
:101918007C80DFF87CC0DFF87CE0194F194C1A484E
:1019280042F6F82111800E490C22062B0A7033D09A
:10193800002388F800308CF800308EF800301B2324
:101948003B700523227003704FF4E13430E000BF90
:101958008A070020AC2900202000002071E600083A
:10196800B81E0020F1E80008A08601005DE6000826
:1019780045E8000845E60008F9E70008D800002017
:101988003A2A0020392900203B2A00203A29002041
:10199800392A0020382A0020002188F800108CF805
:1019A80000108EF8001022702121C04C397003708D
:1019B800BF4BC04A1A60402006F064FB70B1012199
:1019C8000023BD4A90F900008DE80A004021234613
:1019D80006F02EFA003018BF012028B9082008F0B8
:1019E800CFFAB34BB54A1A60B54FB64A3B6813F401
:1019F800804F1FBF12211170AD49B34818BF08604E
:101A080042F20101194003F0010003F4005481B1CE
:101A1800AE4944F6206EA1F800E024B10821117007
:101A2800A349AB4C0C6020B10C211170A049A94806
:101A38000860117813F4007FA1F1040151700DF1D1
:101A480068085CD0DFF8D492039BC9F80030A24B39
:101A5800A2485A6942F480225A619A6942F0010206
:101A68009A61039B1B88ADF83030012402230CA92E
:101A78008DF833308DF8324003F074FFD9F8003018
:101A880096485B88ADF830304FF0000A0CA98DF805
:101A980032A003F067FFD9F800302046197A06F023
:101AA8000DFFD9F80030586806F058FED9F8003014
:101AB8005B681A93404610238DF86D308DF86CA042
:101AC8008DF86E4006F082FCD9F800305B7A8DF80C
:101AD80038300EA803238DF839308DF83AA08DF8E8
:101AE8003B4006F055FC33687D4A3C3B13602B684D
:101AF80043F010032B607B4B4FF0FF321A607A4A99
:101B08007A4B13607A4A7B4D803313603B6800241C
:101B1800DA032C7040F1AA8004F0F0FADFF800C272
:101B2800DFF8B491CDF810C040F22A3B0126604698
:101B380021465A462E7011F06EFAD9F814306E4DBF
:101B48004FF0904043F40033C9F81430436A23F04F
:101B58000F034362436A43F00603436202220323EE
:101B68004FF4807A0CA98DF8342003928DF8353023
:101B78008DF83640CDF830A08DF837600CF0DCFEDB
:101B8800D9F81830039A43F40063C9F818302B8841
:101B980023F45C731B041B0C2B801D23EB620EA922
:101BA8002A8560232C8628466E610E93ADF83E4048
:101BB8001094ADF84440ADF84640ADF84840ADF853
:101BC8004A40ADF83C6006F013FFAB6943F00803E8
:101BD800AB616B6C43F400436B64D9F81430334346
:101BE800C9F81430A9F6E479484606F0EEFD4046F7
:101BF80006F0C0FD414B1A9310231C938023DDF897
:101C080010C01F9341464FF400534846CDF86CC0AE
:101C18002393ADF874B01E94CDF880A0219422943B
:101C2800249406F0B4FDEB6843F40073EB60D9F834
:101C3800003043F00203C9F800300BA80C238DF8DC
:101C48002C308DF82D608DF82E408DF82F6006F021
:101C58009FFB21462A4B1A682A4B43F82120013161
:101C68002029F7D103F0A0FD03F09EFD3B685B053A
:101C780040F18180244C254BD4F8E4641E60042094
:101C880006F000FA0421C4F8E80406F0D7F9204B5E
:101C980084F8EC0408201E6006F0F4F91D4B1E4D74
:101CA8001860082106F0CAF92C223BE090D0030006
:101CB800200000206DE50008D9E60008D5E60008F8
:101CC800A82B0020B81E0020A5E600088A070020DF
:101CD800C5E60008B5E60008001002400004004808
:101CE8005407002014100020F4150020F8180020D4
:101CF800F0150020930D0020002C0140342C0140E9
:101D080094490108940D0020D8000020140D0020EB
:101D1800500D00206C0D0020200D002058070020D9
:101D280090020020002184F8ED04284611F073F990
:101D38007C232B708E236B70E023EB7010207D23A7
:101D480085F82B30C4F8F06406F09CF91021C4F82B
:101D5800F40406F073F984F8F8042020C4F8FC644D
:101D680006F090F92021C4F8000506F067F984F818
:101D780004050DF057FEA34A138823F040031B0403
:101D88001B0C1380138823F038031B041B0C1380CF
:101D980013889BB243F04003138000249F23322012
:101DA8008DF838308DF839408DF83A408DF83B4041
:101DB8000CF0B1FF8DF86940934C4FF48055042224
:101DC800258540460EA906F0ADFAA5619DF86A2062
:101DD8009DF86930120242EA03429DF86B301A43BB
:101DE8008A4B9A428A4B17D008D88A498A420CD023
:101DF80001F51A4102318A4209D01CE086498A421B
:101E080005D001318A4207D015E0202200E0802267
:101E18001A804FF4807202E04FF480721A805A8060
:101E28009A88198812029A604A43DA607B4A01212B
:101E380082F8051504E000221A805A809A60DA6058
:101E4800DC680CB3E40A26464FF00009A14509DA1C
:101E580009EB04056D10E802414610220AF0AAF8C1
:101E68000F2806DC04F08AFB6C4BF602C3F8086501
:101E78000AE0002358F82320013250D10133042B03
:101E8800F8D12E462C46E1E73B68654A13F4002357
:101E980018BF012313700CF017FF624B1860624BD8
:101EA8005A79052A194602BF604B4FF4C8721A8046
:101EB8005F4B4FF47A721A805E4BC8221A805E4AD2
:101EC800137843F0080313705C4A137823F0020375
:101ED80013703A6840F6020313406BB1584B594AE5
:101EE8001A60594B03221A70584B01221A70584A2B
:101EF80000231380574A13808B683B60564B01229E
:101F08001A70564A137863F07F0313702FB0BDEC34
:101F1800068BBDE8F08F4FF0040AFFF752BA05F1BF
:101F280001092546AEE71BB208EE103AB4F95A315A
:101F3800DFED4B7A4B4A09EE103AB4F95C31B8EE52
:101F4800C88A08EE903A28EE278AB8EEC99AF8EEC1
:101F5800E88A0021B0EE480A29EE279A68EEA78A97
:101F6800117007F0E5FFF0EE40AAB0EE480A07F05E
:101F78007FFFF0EE409AB0EE490A07F0D9FFB0EEC5
:101F880040AAB0EE490A07F073FFB0EE408AB0EEFF
:101F9800680A07F0CDFFB0EE409AB0EE680A07F085
:101FA80067FF60EE2A6A69EE897AF0EE665AE7EE14
:101FB800885A2D4B29EE2A6A29EE807AC3ED035AF6
:101FC800F0EE465A2AEE400AE7EE485AE6EE887ADC
:101FD800A6EE487A29EE0A9A83ED010A69EECA9AB2
:101FE8002AEE2A0A83ED009A83ED028AC3ED045A89
:101FF800C3ED059A83ED067AC3ED077A83ED080AE7
:10200800FFF78FB8003800400004004818BA2000D5
:1020180010000020152020001740EF00D8000020F5
:10202800EA2D00205C070020D0160020862700201B
:10203800CE2F0020CC2F002000280020D22F0020F7
:10204800F42A00204A180020D82800206800002020
:10205800700F0020720F0020080D0020AC2F002008
:1020680035FA8E3C5C000020D02A00202DE9F04F84
:10207800A149A24C0A6802F59C432DED028B20333E
:1020880023609F4B87B01E780091C6B19D490968AF
:102098008A4240F20381013E1E70FFE0D9F8003009
:1020A8009948072D98BF595D984B88BF29461B68EA
:1020B8009847032D0CD904EB45050136A880924BAF
:1020C800DFF86C921A78F5B2AA421946E6D820E0F1
:1020D800D9F8002005F10E0302EB83039988DA880A
:1020E8000028E8D04FF47A73401A5843531A90FBEB
:1020F800F3F040F6C90300F57A70984205DC40F227
:10210800EE239842B8BF184601E040F6CA0080B2F4
:10211800D1E77F4B1B6842F2010803EA08087D4BB0
:10212800B8FA88F84FEA58181B68B8F1000F06D1BA
:1021380094F8292084F82820774A5078107094F869
:1021480028701FB1744A177887F0010794F82BB0EC
:1021580091F800A00F220326BBFBF6F606EB460615
:1021680084F82A20C6EB0B06D9F80020DFF8C891BE
:10217800F6B20025554559DA4FEA450C1FB16749B3
:1021880031F8150000E03846918ADFF8B0E1814265
:1021980002D8D18A81421ED25EF82500574983426F
:1021A80003D25F4931F80C0019E0E8B202920193BA
:1021B80003910CF0C7FC032D019B029A0FDC0399D5
:1021C8004FF0010C91F82AE00CFA05FC2EEA0C0EEF
:1021D80081F82AE003E003F596714EF82510B8F16E
:1021E800000F1CD194F8BC1029F8160031B9BBF1C6
:1021F800020F14D94149012081F8BC00B9F8021036
:10220800B9F800000844B9F804100844454980B2F8
:1022180021F8150000B2032190FBF1F080B240498B
:1022280009F1060921F815000135A3E794F82A20D9
:1022380038493D4BA2F10F077A427A4184F8D620FB
:102248006AB13A4A1268560109D40A68D9689A608C
:10225800521AC82A1DD9012283F8212019E02E4AD2
:102268000120507010700A689968DA605B68521A29
:102278009A4282BF2C4B002283F821200025554525
:1022880007DAE8B20CF05EFC254B23F8150001359F
:10229800F5E794F82B30013384F82B301C4B1A687F
:1022A80012F4805F984605D0204B1B68DD0701D4E7
:1022B8000DF06EF9009B19681D4B1F68BB7A002B47
:1022C8003ED0013B16483A7B30F813301AB1C3F5BB
:1022D8003B6308339BB21BB2A3F57A73B3F57A7FDD
:1022E800A8BF4FF47A7323EAE37307EE903A9FEDA1
:1022F800117AF8EEE77A5CE0B82F0020180E00207B
:10230800D42B0020D02B0020B81E00202000002055
:10231800A82B0020D82B0020080000201C0E00202D
:10232800AC2B0020D60E0020DC2B0020AC0F0020A8
:10233800A42B002000007A44440E00208C0E0020BC
:10234800D8F80020100440D5D4F8D800934E081AC5
:1023580000283ADB924A01F59C402030C6F8D800A4
:102368005079904A32F81050A8B2FD7A90FBF5F5F2
:1023780096F8DC00013000F00F0286F8DC203244C9
:1023880082F8DD501A468848185C01330244102B45
:1023980092B2F8D112B292FBF3F31BB2642BA8BF2E
:1023A800642323EAE37307EE903A9FED807AF8EE10
:1023B800E77AC7EE877A7E4A9FED7E7A67EE877A5C
:1023C800FCEEE77A17EE903A1380D8F800307A4F8F
:1023D80013F4807F00F00981784BDFF8E49199428B
:1023E80005D999F8022012B9012289F8022099F832
:1023F8000220002A00F0F980714A3E7892F82150B4
:102408006A1E554255416F4A1168002DC1F3806319
:10241800C6F380060093924614BF4FF0000B4FF0AE
:10242800030B99F82020052A00F2D980DFE802F092
:10243800034D527584A1002E3AD0D4F8F000B4F8B8
:10244800F41005F0C0FE012809D15F495F4A096808
:102458001268C988642000FB0122C9F81020009B7B
:102468006BB1594A126812794AB10DF0A3FA0322E6
:1024780089F820204FF47A72C9F81C20D1E7002D82
:1024880040F0AD80514AD9F8101010684C4A884283
:102498000AD901920DF08EFA019A032182F82010D0
:1024A80040F6B831D161BCE7012182F82010B8E7C5
:1024B800009B4FF4806013B107F052FD01E007F074
:1024C8003FFD0022C9F8102089E0002D46D10DF00B
:1024D80071FAA6E725B1052289F82020012000E03D
:1024E800284666B1D4F8F020D189394A1180518044
:1024F8009180354909684988D1804FF0020B334AE9
:102508001168D9F81420914201D8002E64D147F2FD
:102518003052C9F81C20032221E03A7842F0020226
:102528003A700DF035F8294AD9F81C1012680A4497
:10253800C9F81820042212E0244A9DB11168D9F87C
:10254800182091424BD9234A92781AB9DAF8002018
:10255800D30744D43A7822F002023A70052289F867
:1025680020205EE71268D9F81C100A44C9F8182020
:1025780035E01549154A09681268C988642000FBC6
:102588000122C9F810204FF48060002289F8202029
:1025980089F8032007F0D4FC43E700BF180E002099
:1025A800F82A0020082B0020F50E00200000C84261
:1025B8001C10002000C07F44D22F0020404B4C004C
:1025C800DC2B0020AC0F0020A82F0020D82B0020E7
:1025D800AC2B00200800002000287FF422AFBBF1BC
:1025E800000F02D058460CF039FB8F4D05F5C4702A
:1025F800B5F84E1105F0E7FD834668B90DF0CCF942
:102608008A4BC3F800B0C3F804B0C3F808B0884BCD
:1026180000221A605A609A603B785E0736D5D8F86F
:102628000030D80632D5834B1B78D9062ED4824B7E
:102638009B7893B195F8E031BBF1000F15D17BB1D0
:102648007E4B1A68D4F8F8309B1A002B08DA0CF085
:102658009FFF7B4B83F8FCB018E0BBF1000F0DD156
:1026680010200CF0FBFA01230EE03BB1734A12680C
:102678004FF47A7101FB0323C4F8F83094F8FC3066
:1026880023B105F0FFFD002384F8FC30002295F803
:10269800DEA195F8DF11B5F898E1B5F89AC11346AF
:1026A8006848009030F912609B087645C4BF63F013
:1026B8007F03DBB201326645B8BF43F04003042A0A
:1026C800EED194F8FD205E489A4205D190F8FE209C
:1026D800F92A04D8013200E0002280F8FE2084F8AC
:1026E800FD30554B584E9A789946E2B93368DA0767
:1026F80008D5BBF1000F16D13B78DB0713D50CF0DA
:10270800C1FD10E03B7858070DD54D4B93F82830A4
:102718004BB14E4BDB7833B911B10CF039FF02E005
:10272800BBF1000FF9D094F8FE30454ADFF838B114
:10273800142B40F0AB8099F802301AF1000A18BF48
:102748004FF0010A6BB392F8FD305F2B11D13B7843
:1027580003F0040303F0FF0113B10CF019FF08E0C4
:102768000B20029101920CF079FA019A029982F8F1
:10277800FE10BAF1000F14D094F8FD307D2B10D163
:102788003B7803F0040303F0FF0213B10CF000FFE1
:1027980007E00B2001920CF061FA294B019A83F8AB
:1027A800FE203B7803F0040303F0FF01002B6DD1FA
:1027B80094F8FD30224A572B10D1254B4FF47A72EA
:1027C8001A80244B1B685A0742BF234A0A211180EA
:1027D80013F008035AD1214A138057E0D8F80000B3
:1027E800400716D55A2B14D11D4B187820B11970F3
:1027F8001C4B01221A7049E092F8FF3083F0010364
:1028080082F8FF300BB10C2000E00D200CF026FA06
:102818003CE05D2B00F034845B2B00F033845E2BAE
:1028280024D1032000F02FBCD0160020AC260020B5
:10283800481F00200028002008000020D82B002076
:10284800180E0020AC2B0020AC0F0020DC2B002041
:10285800CE2F0020A40F0020CC2F0020081000202D
:10286800B1270020B2270020E80F0020562B01D105
:1028780007F020FE99F80230002B00F0198494F834
:10288800FD306F2B40F00E840CF0FCFCD8F80030C3
:102898005A0732D594F8FF30A3B13B785B0711D5BE
:1028A800009BB3F90620B5F898319A420ADD3368DF
:1028B80013F0010301BFAC4A32211180AB4A08BFB3
:1028C80082F8FF303368D8030AD5A94B1A782AB999
:1028D800A84A127812B9A44A3221118001220BE0C9
:1028E800A44A13784BB13B7803F0040303F0FF01CB
:1028F8001BB9A14B117001221A70DBF800A000234C
:1029080033600AF187090AF1D70B99F8002099F882
:10291800013019F8010C9A420BD2494605F01CFC0B
:1029280038B119F8022C012303FA02F23368134371
:10293800336009F10409D945E7D1904B1B782BB1D5
:102948008F4E3368990700F13D8334E30AF1D606C8
:102958000AF58F793278737816F8010C9A4225D2E5
:10296800314605F0F9FB08B3B37896F804C0854AF8
:1029780096F803A07D480C21013B01FB0C4103EBB9
:1029880043031344D1F804219A420FD0C1F804310B
:10299800002390F83021C1F80831012303FA0CF321
:1029A80022EA030381F800A180F8303106364E454B
:1029B800D0D1754B1E68754B1B68029394F828306C
:1029C8000393734B019300230093019B1A68002A19
:1029D80000F0E68292F800A0BAF1000F00F0E08261
:1029E8005B680299CB1A002B0CDB01F5FA7301998D
:1029F8004B60009901238B4094F8301121EA0303BE
:102A080084F83031039B002B00F0CA82019B517877
:102A180013F8043C0433DBB2002940F080825D499E
:102A280031F91310B5F8963103F1C800814202DD7F
:102A380092F802B015E0C83B994203DA9178C1F1E7
:102A4800000B0EE0009A0123934094F8302122EA0B
:102A5800030384F83031029B019A03F5FA7353603B
:102A68009EE2009A94F830311341DA0700F1988217
:102A7800BBF1000FCCBF0220012005F0E9FB0AF1F1
:102A8800FF33DFF8E890132B00F28282DFE813F0BF
:102A98001400250037004B0064008A00ED00500147
:102AA800B701E501150280024B005A008A00ED00CB
:102AB8005001BF002201870196F80090D944B9F16E
:102AC800FA0FA8BF4FF0FA0929EAE979304686F8E3
:102AD800009005F027FB01200FE096F80190D944FB
:102AE800B9F1640FA8BF4FF0640929EAE9793046C3
:102AF80086F8019005F016FB02204946DAE196F8BF
:102B080003A0DA44BAF1640FA8BF4FF0640A2AEAB6
:102B1800EA7A86F803A03046D9F8341105F0B8FAF5
:102B280003205146C6E1717959446429A8BF64213C
:102B380021EAE17171710D2005F076FBBAF10D0FF4
:102B480000F02682317959446429A8BF642121EA1A
:102B5800E17131710E20ADE1B179594481F3080179
:102B6800B1710520A6E100BF98270020180E0020AB
:102B7800B0270020B1270020B2270020D32F002043
:102B8800AC0F0020684C010828100020D82B00202A
:102B98001C0F0020AC2B002000007A440000C84223
:102BA80000000000D9F838311A78022A20D107EE3F
:102BB80090BAB8EEE70A5FED077A93ED097A80EEEE
:102BC800270A30EE070AB5EEC00AF1EE10FA07D46C
:102BD800B4EE670AF1EE10FAC8BFB0EE670A01E07A
:102BE8001FED110A83ED090A0F2005F007FB0AE023
:102BF80099785944C829A8BFC82121EAE171997078
:102C08000F2005F011FBBAF10F0F00F0C181D9F8C0
:102C180038311A78022A1ED107EE90BAB8EEE78A40
:102C28005FED227A93ED080A88EE278A38EE000ACB
:102C3800B5EEC00AF1EE10FA07D4B4EE670AF1EE69
:102C480010FAC8BFB0EE670A01E01FED2B0A83ED4A
:102C5800080A122056E159785944C829A8BFC82142
:102C680021EAE1715970122024E1D9F838311A7833
:102C7800022A20D107EE90BAB8EEE70A5FED397A5A
:102C880093ED0C7A80EE270A30EE070AB5EEC00AFB
:102C9800F1EE10FA07D4B4EE670AF1EE10FAC8BFE5
:102CA800B0EE670A01E01FED420A83ED0C0A10201E
:102CB80005F0A4FA0AE0197B5944C829A8BFC8211D
:102CC80021EAE1711973102005F0AEFABAF1100F7C
:102CD80000F05E81D9F838311A78022A1ED107EE41
:102CE80090BAB8EEE78A5FED537A93ED0B0A88EE57
:102CF800278A38EE000AB5EEC00AF1EE10FA07D4BA
:102D0800B4EE670AF1EE10FAC8BFB0EE670A01E048
:102D18001FED5D0A83ED0B0A1320F3E0D97A5944BD
:102D2800C829A8BFC82121EAE171D9721320C1E0DE
:102D3800D9F838311A78022A22D107EE90BA1FED55
:102D48006A0AF8EEE77A87EE800AD3ED0F7A30EE5A
:102D5800270AB5EEC00AF1EE10FA09D45FED717AD0
:102D6800B4EE670AF1EE10FAC8BFB0EE670A01E0E8
:102D78001FED750A83ED0F0A112005F03FFA0AE0EE
:102D8800997D5944C829A8BFC82121EAE1719975DC
:102D9800112005F049FABAF1110F00F0F980D9F8BD
:102DA80038311A78022A20D107EE90BA1FED860A28
:102DB800B8EEE78A88EE008A93ED0E0A38EE000A2C
:102DC800B5EEC00AF1EE10FA09D45FED8C7AB4EED4
:102DD800670AF1EE10FAC8BFB0EE670A01E01FED0E
:102DE800900A83ED0E0A14208CE0597D5944C829B5
:102DF800A8BFC82121EAE171597514205AE0D9F811
:102E080038311A78022A1ED107EE90BAB8EEE78A4E
:102E18005FED9E7A93ED0A0A88EE278A38EE000A5B
:102E2800B5EEC00AF1EE10FA07D4B4EE670AF1EE77
:102E380010FAC8BFB0EE670A01E01FEDA70A83EDDC
:102E48000A0A09205EE0D9785944C829A8BFC821D0
:102E580021EAE171D97009202CE0D9F838311A78C3
:102E6800022A1ED107EE90BAB8EEE78A5FEDB57A6E
:102E780093ED0D0A88EE278A38EE000AB5EEC00AEF
:102E8800F1EE10FA07D4B4EE670AF1EE10FAC8BFF3
:102E9800B0EE670A01E01FEDBE0A83ED0D0A0A20B5
:102EA80030E0597B5944C829A8BFC82121EAE171FB
:102EB80059730A2005F0B8F96AE0D9F838311A7858
:102EC800022A22D107EE90BA1FEDCD0AB8EEE78AA2
:102ED80088EE008A93ED100A38EE000AB5EEC00AB3
:102EE800F1EE10FA09D45FEDD37AB4EE670AF1EE89
:102EF80010FAC8BFB0EE670A01E01FEDD70A83EDEC
:102F0800100A0B2005F07AF942E0D97D5944C82906
:102F1800A8BFC82121EAE171D9750B20CAE70129A8
:102F280036D19078864A32F91390B9F5617F05DB7E
:102F380040F633039945A8BF994601E04FF46179FB
:102F4800BAF10C0F24D17F4A4FF4966393FBF0F04B
:102F58001378A9F5617999FBF0F95FFA89F94B457E
:102F680016D0B9F1040F34BF4B4602231370764ACA
:102F78000AFB035303F2B273136007F0D5F8504607
:102F8800494605F051F909F10100C0B205F060F9B0
:102F9800009A0123934094F83021134384F8303188
:102FA800009B01330093019B0C330193009B042B7E
:102FB8007FF40BADC4E4D8F80030DB0511D5634BC2
:102FC800DB7873B1624B1B689C070AD5614B1B8881
:102FD80013F001040AD10CF0DFFC012006F0C0FF59
:102FE80004E0012006F0ACFF012300E00023326872
:102FF80050070DD563B1012006F0A2FF554B1B8881
:10300800990708D40CF0C8FC022006F0A9FF02E0DA
:10301800022006F095FF33681A054FF4807002D538
:1030280006F09EFF01E006F08BFF6B79082B01D0BC
:103038000E2B02D1402006F083FFD8F800305B0544
:1030480078D595F818321BB93B7813F0040F02E0D5
:10305800336813F4002F0AD03F4B00221A703C202B
:1030680005F048FB002865D00AF09AFFF7E70CF056
:10307800D9FC07B0BDEC028BBDE8F04F05F047BAAC
:10308800012000E002205FFA80F909F1FF3385F89A
:10309800B03706F0AFFF07F06BF8484605F0D8F8F0
:1030A800FFF7F4BBBAF1000F02D07E2B3FF4ECAB74
:1030B80094F8FD30972B05D1284B4FF4C8721A802D
:1030C800FFF7E4BBA72B06D1254A137843F0040386
:1030D8001370FFF7DBBB0022BB2B059201D1022343
:1030E80003E0B72B04D14FF6FE73ADF816300AE0B3
:1030F800BE2B01D1022304E0BD2B7FF4C7AB4FF6F2
:10310800FE73ADF81430DBF80030BDF81410B3F8D6
:1031180064200A44A3F86420BDF81610B3F86620AA
:103128000A44A3F8662007F0C5F9002384F8FE30A6
:10313800FFF7ACBB07B0BDEC028BBDE8F08F00BF5A
:10314800AC2B0020B028002028100020DC2B002009
:10315800A40F0020A80F0020BD1E002086270020F5
:10316800002800202DE9F04FBB4BB3F90610BB4BEC
:103178002DED028B1F687A8991B0914201930EDB85
:10318800B1F5FA6FFC79BDBF8B1A6343A2F5FA64F7
:10319800C4F16404BCBF93FBF4F4643400E0642419
:1031A800AF4AB04BB2F896A192F95E211868049024
:1031B80092B20592054600220293A74B33F91230CA
:1031C8000393CAEB030303F2F31640F2E630864298
:1031D8004FEA420B03D8002BB8BF5B4201E04FF423
:1031E800FA73022A00934FF06400049B9E4E31D07C
:1031F80093F81DE1BEF1000F06D0009B7345CCBFCC
:10320800CEEB030300230093009BDFF8A0E293FBBF
:10321800F0FC6FF063093EF81C8009FB0C390CF1D7
:10322800010C3EF91CE00FFA88FCCCEB0E0E0EFBED
:1032380009FE9EFBF0FEC64426F80BE0BE18367960
:1032480073438A4E93FBF6F364339BB2634393FB59
:10325800F0F031E093F81EE1BEF1000F06D0009BBC
:103268007345CCBFCEEB030300230093009BDFF82C
:10327800288293FBF0F06FF0630C38F910E00CFB38
:1032880000390130BDF8143038F91000CEEB0000D9
:1032980000FB09F999FBFCF9CEEB090919FB03F9C5
:1032A800009BA6F80490B879002BB8BF5B42434353
:1032B8006E4893FBF0F064306B786D4E4FF0640EFF
:1032C800434393FBFEF3B3546A4EEB7A434393FBB9
:1032D800FEF3B3546B7D644E5843674B90FBFEF08E
:1032E800022A9854654B0FD183F802E0039B53459B
:1032F8000EDB5B4CB4F89821914215DBB1F5FA6FFF
:10330800A8BF4FF4FA6110E09C54039B534504DABC
:1033180036F80B305B4226F80B300132032A05F1F0
:1033280001057FF44AAFE4E71146891A4FF47A732E
:10333800DFF87CE14C4D59436FF06303C2F5FA6244
:103348006427B1FBF2F191FBF7F23EF8120003FBA0
:103358000211013203B23EF91220D21A514391FBF5
:10336800F7F30344F380464B1B885B0635D5454B82
:10337800454A1B881288DFED457A9B1A1BB208EE76
:10338800103AB8EEC88A28EE278AB0EE480A06F046
:10339800CFFDF0EE408AB0EE480A06F069FDB5F9B7
:1033A800023006EE903AB5F90030F8EEE66A07EE1C
:1033B800903A20EE667AF8EEE77AA7EEA87A67EEFA
:1033C800807ABDEEC77AE6EEA87A17EE103AFDEEDF
:1033D800E77A2B8017EE903A6B802D4D2B689F076C
:1033E80040F1A1802B4B2C4F1A687B6945F20721CD
:1033F800D31A8B4240F397807A610BF08BFB274BF3
:10340800DFF8B0901A78032A9846B9F8003053D1FB
:103418000A2B5BD90023282088F800300BF07BFCAE
:103428000BF078FB1E4B18880BF05EFB1D4B1A68DF
:10343800D37890FBF3F0013008281B4BA8BF082075
:103448001870537980B213FB00F33B83137913FB95
:1034580000F078833AE000BFAC2B00202810002051
:10346800D0160020E80F0020942600200CFEFFFF55
:103478005C1F0020660F0020701F00209C26002083
:10348800A80F002008100020E82D002035FA8E3CF7
:10349800A82B0020B82F0020580F0020D828002083
:1034A800102B0020F42A00206800002016160020A7
:1034B800FE150020A02B00200A2B07D80323A54ABD
:1034C80088F80030002313703B837B8398F8003022
:1034D800A14A012B0CD002D3022B1BD023E03A8B3C
:1034E800B9F800309A421EDD012388F800300FE059
:1034F800B9F800107B8B8B4202DD022313700FE0BA
:10350800964B1B8B0133994202DD002313700AE0AE
:10351800082006E07B8BB9F8002001339A42E3DCEF
:1035280007200BF09BFBD5F800B08D4D1BF4006F06
:1035380078D08C4B894F1B68FA69C2EB030845F2B7
:10354800072290456EDDFB61874BB6F906C0D3F8BC
:103558000090B4F84E1199F80A30844E012BACF55E
:103568007A7C03D045D3022B20D044E0804B396AC3
:103578005A7B804B33F81220082092B291FBF0F36B
:10358800C91A8B18BA843B6240F6E44293FBF0F305
:103598009BB25343B9F80820C2EB13334FF47A7245
:1035A8005343B9F9062093FBF2F323E02B78B9F8DB
:1035B80008A0C6F800A058071DD56F48CDF800C070
:1035C80004F001FEDDF800C020B91BF0100F18BF91
:1035D8004FF0000C32220CFB0CF393FBF2F3B9F919
:1035E800062063445A434FF47A7392FBF3F353442F
:1035F80000E000233360D7E90A01336803FB08F8C9
:103608004FF47A7398FBF3F810EB080241EBE87378
:10361800C7E90A2310461946584A00230CF024FD2E
:10362800574B1860574F00973B6813F4805F02D0E0
:103638000A200BF013FB544E3268002A57D0534926
:10364800534B08681F688742894698464FD8514BA4
:10365800DFF84CA11878516808BB01201870BAF837
:103668000030CB5C5BB31378013B00FA03F2D4F86B
:10367800DC371A4201D10BF075FB474B01221A7057
:103688000BF0B2FABAF80030CBB933681B78053BB7
:10369800012B14D80BF018FB404B18600FE04FF0CB
:1036A800000B83F800B0BAF80030CB5C3BB1584649
:1036B8000BF058FB384B83F800B00BF095FA3268E2
:1036C800BAF8003052683648D25CFE2A01D100238D
:1036D8000CE0FF2A02D104F0D5FD08E0D9F800601B
:1036E8000A2111FB0262C8F80020013303802B78FD
:1036F800590703D52B4B08221A856DE0009A1268EA
:10370800D2075EBF164A43F001031370264B224AC4
:103718001B781F075EBF2B7823F001032B70234B08
:103728001B6813F0040F02D02149098851B92149B7
:10373800098809B19E0705D41F4B1B88003318BFA1
:103748000123DBB3022313702B7823F001032B70C2
:1037580039E000BF68000020D8280020580F00205A
:10376800D22F0020B82F0020F42A0020201000209B
:10377800F82A0020082B002058180020407E050059
:1037880018100020AC0F002030160020D82B002085
:103798002816002024160020002C0020882F002046
:1037A8002C1600200004004800280020A40F002048
:1037B800CC2F002086270020CE2F00202978C8078C
:1037C80058BF022313700BF07FFAB44B1B68C01A62
:1037D800002801DB0BF008FAB14F0CF023F93E7812
:1037E800002E00F0AC80AF4B1A689846002A00F013
:1037F800BD86D8F800000BF009FB002800F0B6865B
:10380800A84BA94C18680BF0FEFA092801D03F28EC
:1038180052D14FF0000A2668DFF8C892554636B1F3
:10382800A248D9F8001032460FF042FC10B9CA4637
:1038380005B94D469E4B09F110099945EFD3EDB1F5
:10384800D5F800C0DAF8009023681CF803E019F8EE
:103858000300704512D15A1C944958B92D2B09D828
:10386800DFF844E2CEF800204FF0200E01F803E024
:10387800885403E001F803E02260E5E723680BB110
:10388800554510D08B480AF083FC554507D855F8A4
:10389800100B0AF07DFC09200AF072FCF5E7864857
:1038A8000AF076FC002623689E42A2D27F4B985DE0
:1038B8000AF066FC0136F6E72368002B40F03C86E8
:1038C800042840F05E86794803F0D8F800F04EBE30
:1038D800D9F80000DFF8ECA10BF098FA28B3DAF871
:1038E80000000BF090FADBF8003093F8481002461D
:1038F800A9BB24286CD1012283F84820DBF80030CA
:10390800DFF8E4A193F84820062AE1D193F84900AA
:1039180000F0C2FE8346002800F083800AF08CFB8A
:10392800D8F80030002283F84820644B93F83730E9
:10393800002B40F0EF854C36982E00F01786604B30
:10394800F21892F84A100129F5D1DFF89C81F35852
:10395800C8F800205B4AC34613609146B8E70129BE
:1039680004D14D2814BF00220222C5E7022904D140
:103978003C2814BF00220322BEE703290CD14028AB
:103988004FF0000102D983F84810B7E75871197150
:10399800D97198710422AFE7042906D1997983F87F
:1039A80049004A409A710522A6E70529A6D1587907
:1039B80019798842987906D950409871481C18712D
:1039C8000B441A729AE790420CBF0622002293E732
:1039D8002B783D495B0791D42328DAF8003013D1BE
:1039E8000090012038702F48039103603348036327
:1039F80036480AF0CDFB30480AF0CAFB0399009A12
:103A08000B7843F002030B70314B1B681B78934211
:103A180001BF304B304A1A60304B04BF304ADA607D
:103A28006CE7DAF8002092F849304A2B00F06D85EF
:103A380000F28580332B00F0718421D8292B00F007
:103A4800F68309D8252B00F0CE83272B00F0D183ED
:103A5800232B40F0928569E22D2B00F0F98307D8DB
:103A68002B2B40F08A850AF0BBFA607100F04DBD3F
:103A78002F2B00F0BF84312B00F0D18400F07DBDE6
:103A88003E2B00F03D8146D8372B00F07A842DD8A4
:103A9800352B00F0868200F070BD00BF042C00209A
:103AA800D32F0020D4280020EC150020BC150020BE
:103AB80024500108776901087C690108580F002023
:103AC80038160020D0280020D22F0020AC69010829
:103AD800C01E0020FC9F0020EFBEADDE00ED00E020
:103AE8000400FA05544E0108CC280020392B00F0B8
:103AF8008D833C2B40F04185DFF81894D9F800A05D
:103B08000AF06EFA8AF80000D9F80030187809F03F
:103B180065FC00F0FABC432B00F0118405D8412B5A
:103B280040F02B854FF00009FDE3442B00F0AC84F6
:103B3800482B40F0228502F06FFD00F0E6BCD02B48
:103B480000F02F835FD8CA2B00F0E38016D84E2BE5
:103B580000F0B683C82B00F0A2804C2B40F00D85F6
:103B68000AF03EFA84F8D6010AF03AFA84F8D70146
:103B78000AF040FAA4F8D80100F0C7BCCD2B00F039
:103B88001B8304D8CC2B00F0348200F0F6BCCE2B7B
:103B980000F01B83CF2B40F0F0840AF02BFA6FF46F
:103BA800AF6E00EB0E039BB2C62B98BFA4F896012C
:103BB8000AF020FAA4F840010AF01CFAA4F842011D
:103BC8000AF018FAA4F844010AF014FAA4F8D80183
:103BD8000AF006FA0AF004FA0AF002FA0AF000FA01
:103BE80084F885010AF0FCF984F892010AF0F8F9E2
:103BF800C84BD3F800900AF0FDF900EB80004000B4
:103C0800A9F8620002E3D82B00F015810FD8D32B56
:103C18003FD003D8D22B29D000F0AFBCD42B00F072
:103C28004782D62B40F0A9844FF0000935E2F22BE9
:103C380000F08C8212D8EF2B40F09F84DFF8D492EA
:103C4800D9F800A00AF0D6F9AAF86600D9F80090C9
:103C58000AF0D0F9A9F8640000F057BCF32B00F083
:103C68001884FA2B00F0BB8200F087BC2B7803F095
:103C7800040303F0FF09002B40F047840AF0B0F971
:103C8800022884F8B00740F29282A34B83F8B097D9
:103C98008DE20AF0AFF9A14B988600F036BC92F895
:103CA80005904FEA5909B9F1120F03D904F01EFD26
:103CB80000F02BBC4FF0000ACA4507D20AF09AF967
:103CC80007AB23F81A000AF1010AF5E74A46002370
:103CD8004B4507DA07A931F81300914921F8130079
:103CE8000133F5E7122A05D08D4B002123F8121075
:103CF8000132F7E7894B012283F8362000F005BC32
:103D08000AF06EF984F8E0010AF06AF984F8DF0134
:103D1800FBE3804B1A681278022A824699466FD1D3
:103D2800D9F800B00AF05CF907EE900AF8EE677A65
:103D3800B2EE048AC7EE887A0BEB8A0BCBED087AD1
:103D4800D9F800B00AF04CF907EE900A9FED757AA1
:103D5800F8EE677A0BEB8A0BC7EE877ACBED0B7A16
:103D6800D9F800B00AF03CF907EE900A9FED6E7A98
:103D7800F8EE677A0BEB8A0BC7EE877A0AF1010A2D
:103D8800BAF1030FCBED0E7ACAD1BAF1070FD9F801
:103D980000B01CD10AF024F907EE900AF8EE677A11
:103DA800C7EE887ACBED117AD9F800B00AF018F985
:103DB80007EE900AF8EE677AC7EE887ACBED127AAA
:103DC800D9F800B00AF00CF98BF84C0012E00AF0B0
:103DD80007F9D3448BF80100D9F800B00AF000F9CC
:103DE800D3448BF80B00D9F800B00AF0F9F8D344A3
:103DF8008BF815000AF1010ABAF10A0FC5D184E35C
:103E0800D9F800B00AF0ECF8D3448BF80100D9F8DF
:103E180000B00AF0E5F8D3448BF80B00D9F800B0ED
:103E28000AF0DEF8D3440AF1010ABAF10A0F8BF856
:103E38001500E5D169E38246DFF8D8909FED3A8A0C
:103E4800D9F800B00AF0D6F807EE900AF8EE677ACB
:103E58000BEB8A0BC7EE887ACBED087AD9F800B05D
:103E68000AF0C8F807EE900AF8EE677A0BEB8A0BAF
:103E7800C7EE887ACBED0B7AD9F800B00AF0BAF819
:103E880007EE900AF8EE677A0BEB8A0BC7EE887A92
:103E98000AF1010ABAF1030FCBED0E7ACCD1BAF1CF
:103EA800070FD9F800B01CD10AF0A4F807EE900A61
:103EB800F8EE677AC7EE887ACBED117AD9F800B0B8
:103EC8000AF098F807EE900AF8EE677AC7EE887A53
:103ED800CBED127AD9F800B00AF08CF88BF84C00C8
:103EE80012E00AF087F8D3448BF80100D9F800B043
:103EF8000AF080F8D3448BF80B00D9F800B00AF028
:103F080079F8D3448BF815000AF1010ABAF10A0FBF
:103F1800C5D1FAE2E80F0020D0160020580F002083
:103F2800F42900200000C84200007A440AF058F83A
:103F3800132883463FF6BAAEDFF870A3DAF800908C
:103F48000AF04EF80023D44A0C2101FB0322117A0F
:103F5800814222D10FFA8BFB09EB8B09137889F880
:103F680085300AF03DF889F886000AF039F889F8B2
:103F780087000AF035F8C94BC94A1A6089F88800E1
:103F8800C84BDAF8000018600021853004F00AF9FF
:103F9800C54B80F001001870B7E201331C2BD2D159
:103FA80084E60AF01DF80B2882463FF67FAEBF4B29
:103FB800D3F800900AF014F803283FF677AE0623EA
:103FC80003FB0A9989F8DA000AF00AF889F8D5009B
:103FD8000AF006F889F8D6000AF002F889F8D7003E
:103FE80009F0FEFF89F8D80009F0FAFF89F8D9002E
:103FF8008BE25379092B7FF659AE019BD3F80090D9
:1040080009F0EEFF019B89F80000D3F8009009F051
:10401800E7FF89F8010009F0E3FF019B64281B68AA
:10402800A8BF6420187109F0DBFF019B64281B6896
:10403800A8BF6420587109F0D3FF019BFF281B68B3
:10404800A8BFFF20987109F0CBFF019B6428D3F823
:10405800009028BF642089F8070009F0C1FF019B80
:1040680089F80200D3F8009009F0BAFF019B89F89B
:104078000300D3F8009009F0BDFFD8F80030A9F884
:104088000A005B790A2B40F24082894BD3F80090F2
:1040980009F0A6FF89F8080037E209F0ABFF854B65
:1040A80023F8190009F10109B9F1080FF5D12CE23B
:1040B80053790F2B7FF4FAAD09F092FF0728814658
:1040C8003FF6F4AD029BD3F800A009F093FF0E234E
:1040D80003FB09F9CA44029BAAF82501D3F800A0FA
:1040E80009F088FFCA44029BAAF82701D3F800A068
:1040F80009F080FFCA44029BAAF82901D3F800A05E
:1041080009F06EFFCA44029B8AF82B01D3F800A07D
:1041180009F066FFCA44029B8AF82C01D3F800A074
:1041280009F05EFFCA44029B8AF82D01D3F800A06B
:1041380009F056FFCA44029B8AF82E01D3F800A062
:1041480009F062FFD144C9F82F01DEE109F048FF08
:104158000F2881463FF6AAADC9EBC90909F040FF0F
:1041680004EB090303F1D00983F8D00009F038FF04
:1041780089F8010009F034FF89F8020009F030FFDE
:1041880089F8030009F02CFF89F8040009F028FFDA
:1041980089F8050009F024FF89F806000AF0E4FF11
:1041A800B3E12B78580700F1B08109F061F905F007
:1041B80021FF05F0DDFFA8E12B78590700F1A58163
:1041C8003D4B4FF4C8721A809FE12B785A0700F1D3
:1041D8009C813A4A137843F00403137095E12B78D5
:1041E8005B07E4D5C9E1A06009F00EFF05F0D0FE39
:1041F8008BE109F0FFFEA4F8580109F0FBFEA4F8D2
:104208005A0109F0F7FEA4F85C017EE109F0E8FE26
:1042180084F87A0109F0E4FE84F87E0109F0E0FEF2
:1042280084F87D0109F0DCFE84F87F016DE109F076
:10423800E1FEA4F8800109F0DDFEA4F8820109F08E
:10424800CFFE84F8840109F0D5FEA4F886015CE16C
:1042580009F0C6FE84F8900109F0CCFEA4F89A0192
:1042680009F0C8FEA4F8960109F0C4FEA4F8980164
:1042780009F0B6FEDAF8003084F891015B79082B72
:1042880040F2438109F0B6FEA4F89C0109F0B2FEA1
:10429800A4F89E0139E100BFD44C01084C0F00205E
:1042A80010180020500F00200A000020E80F0020FE
:1042B80028100020B228002086270020002800208F
:1042C80092F805900323B9FBF3F9B9F1120F3FF601
:1042D800EDACDFF8C0A34FF0000BCB4580F01581A3
:1042E80009F07EFE8AF8A00109F084FE40F2ED2371
:1042F800984205DD40F6CA039842A8BF184601E077
:1043080040F2EE20A0F2EE2019230BF1010B90FBF6
:10431800F3F00AF1020A8AF89F01DEE709F060FE6D
:1043280084F89201F1E009F05BFE04EB090309F15E
:104338000109B9F1080F83F88801F4D1E5E009F023
:104348004FFEC4F808B0607109F05EFE05F020FE6B
:1043580009F046FE84F8900109F04CFEA4F85801D3
:1043680009F048FEA4F85A0109F044FEA4F85C01DB
:1043780009F040FEA4F8800109F03CFEA4F882018F
:10438800C3E053794FF0070AB3FBFAF2C2EBC2025B
:104398009A1A12F0FF0F7FF489ACB3FBFAFA0AF10C
:1043A800FF3A5FFA8AFABAF1FF0F00F0AE8009F01F
:1043B80017FE5FFA80FB4FFA8BF003F089FD814608
:1043C80000283FF473AC80F800B009F013FEA9F898
:1043D800020009F005FE89F8040009F001FE89F8D9
:1043E800050009F0FDFD89F8070009F0F9FD89F8D5
:1043F8000600D4E7DFF89C9209F1400A09F0FAFDBB
:10440800A9F8A80209F0ECFD89F8AA0209F0E8FD6C
:1044180009F1040989F8A702D145EFD175E009F03F
:10442800DFFD1F2881463FF641ACD8F800305B79A4
:10443800082B7FF43BAC09F0DDFD09F18A0904EB98
:10444800890A00F03F00AAF8020009F0D3FDBAF883
:104458000230800100F4FE501843AAF8020009F067
:10446800BFFD000104F8290009F0BAFD14F829304D
:1044780000F00F00184304F8290009F0B1FD8AF88C
:10448800010001F03BFE40E0714B012283F8372028
:104498003BE009F0A5FDFF28824622D100238DF8D4
:1044A8001B309DF81B30072B14D89DF81B00694A58
:1044B8009DF81B3052F8300002EBC30301215B6802
:1044C800994089B2042203F01FFC9DF81B30013388
:1044D800DBB2E4E760484FF40041002203F014FC2B
:1044E80013E007283FF6E2AB002009F0C9FD09F008
:1044F800A3FDD9F800000AF083FC18B932200AF0AD
:104508000AFCF6E7504603F00DFC002009F0B8FD60
:10451800FFF704BA514B98590AF072FC18B93220C7
:104528000AF0F9FBF6E70AF0DFFD05F039FD4C4B20
:104538004C4ADA60FFF7FFB90C2824D00A282BD19F
:10454800494D4A4809F024FE284623210EF099FDDA
:1045580008B1401B20602368002B40D142482360EB
:10456800002130220EF057FD3B787BB9404B9B6809
:10457800002B67D03F48984764E004F0B7F8FFF78E
:10458800CDB90C2804D13C4809F002FE3B480DE0A7
:104598007F2812D1FFF72DB90D28D1D07F2809D156
:1045A800013B314A364823600021D15409F0F0FD1F
:1045B800FFF71FB92F2B3FF61CA9A0F12002D2B29A
:1045C8005E2A3FF616A913B920283FF412A95A1CEF
:1045D8002260254AD05409F0D3FDFFF70AB95A1EC4
:1045E800A95C202901D11346B6E71F4A23600021A0
:1045F800D154244B244DD3F800A0D5F800B0DFF8EF
:10460800689058460EF04BFD0646324648465946D5
:104618000EF04EFD1D4A28B919F8063053445B7850
:10462800590703D010359542E7D306E0954204D2E6
:10463800701CEB684844984702E0154809F0A8FD4B
:1046480000238BE711B0BDEC028BBDE8F08F00BFF3
:10465800580F0020E87401080008004838160020A8
:1046680000ED00E00400FA05BC1500208F77010872
:1046780008270020900F0020816901087C69010843
:10468800A86901086C000020544E01082450010854
:104698008C690108D01600202DE9F0472DED028B1A
:1046A8004728A0B0044600F05D8600F2CE802E2890
:1046B80000F00C8667D8222800F0B98423D8032894
:1046C80000F03A8214D8012800F02B82022840F02A
:1046D8007E86042009F0D4FC432009F09EFC4C207F
:1046E80009F09BFC462009F098FC4C2000F0C0BD66
:1046F800042800F02B82052840F069861A2009F06A
:10470800BFFC002432E2282800F0798515D8242837
:1047180000F06085262840F05A86C34C062009F030
:10472800AFFCB4F8580109F0AEFCB4F85A0109F02E
:10473800AAFCB4F85C0100F0ACBD2A2800F0728530
:104748002C2840F04486B84C0C2009F099FC94F8C9
:10475800900109F062FCB4F89A0109F094FCB4F8ED
:10476800960109F090FCB4F8980109F08CFC94F8D3
:10477800910109F052FCB4F89C0109F084FCB4F8EA
:104788009E0100F086BD3A2800F0DE821DD834284C
:1047980000F06F840DD8302800F0AE85322840F044
:1047A8001686012009F06CFC9F4B93F8920100F0EB
:1047B8005FBD362800F07085382840F00886042050
:1047C80009F05EFC984C00F00BBD402800F05385C2
:1047D80011D83B2800F024843D2840F0F885924CFD
:1047E800022009F04DFC94F8E00109F016FC94F859
:1047F800DF0100F03DBD452800F0D68500F2A18517
:10480800422840F0E485884C102009F039FC607992
:1048180009F003FCA06809F03FFC94F8900109F046
:10482800FCFBB4F8580109F02EFCB4F85A0109F061
:104838002AFCB4F85C0109F026FCB4F8800109F000
:1048480022FCB4F8820100F024BD6F2800F0CF826A
:1048580000F2F280662800F0C58100F2BE804D2883
:1048680000F0E68415D8492800F0BA824B2840F0B9
:10487800AE856D4C042009F003FC94F8D60109F0CC
:10488800CCFB94F8D70109F0C8FBB4F8D80100F0C4
:1048980000BD642800F08381652840F09885634C4A
:1048A8000B2009F0EDFB208809F0EDFB6268604BF6
:1048B8009A420CBF2089608980B209F0E4FBE36862
:1048C800C3F3C000C3F38002800040EA4200C3F390
:1048D80040021043C3F3401240EAC20003F0100341
:1048E800184309F0D0FB228A6369247E02F008018C
:1048F80003F4475949EA010903F4804149EA0109E7
:1049080003F4004149EA010903F4803149EA010945
:1049180003F4003149EA010903F4802149EA010955
:1049280003F4002149EA010903F4801149EA010965
:1049380003F0007349EA0303DFF8F89099F8009050
:1049480012F0010FC9F3800914BF4FF002084FF0AD
:10495800000843EA090312F0020F43EA080314BFF0
:104968004FF0040C4FF0000C12F0040F43EA0C0C4B
:1049780014BF4FF0100E4FF0000E12F0400F14BF8E
:10498800202700274CEA0E0E12F0100F14BF4FF428
:10499800007600264EEA070712F0200F14BF4FF4E6
:1049A800806500253E4312F4807F14BF4FF40060F9
:1049B8000020354312F4007F14BF4FF4001100218A
:1049C800284312F4806F41EA000114BF4FF080635E
:1049D8000023002019430346F1E0692800F097817D
:1049E8000AD8672800F01E81682840F0F08410205B
:1049F80009F046FB002482E16D2800F09B8100F25B
:104A0800C1816C2840F0E384084C062009F038FB8B
:104A1800B4F86C0009F037FBB4F86E0009F033FB0A
:104A2800B4F8700000F035BCD0160020980F0020B4
:104A380000540040D22F0020772800F084834BD800
:104A4800732800F0A0833CD8702800F002827228F6
:104A580040F0BD84BF4C162009F012FBB4F8960153
:104A680009F011FBB4F8400109F00DFBB4F842015C
:104A780009F009FBB4F8440109F005FBB4F8D801C2
:104A880009F001FB002009F0C8FA002009F0C5FA76
:104A9800002009F0C2FA94F8850109F0BEFA94F8EA
:104AA800920109F0BAFA002009F0B7FAAA4B1B6D77
:104AB8000A20B3F9623093FBF0F080B209F0E3FA10
:104AC8008EE3742800F00683752840F080842F2038
:104AD80009F0D6FAA14C9BE2A02800F06D830AD811
:104AE800782800F0AB807B2840F071843C2009F0E6
:104AF800C7FA002436E2F12800F0DB80FE2800F037
:104B08004D83F02840F06384934C042009F0B8FAF0
:104B1800236DB3F8660009F0B6FA236DB3F86400A4
:104B2800B7E3032009F0ACFA002009F076FA204632
:104B380009F073FA0D209BE309F0A2FA012009F0AD
:104B48006CFA0B2009F069FA002091E3062009F0BD
:104B580097FA522009F061FA4D2009F05EFA4420D4
:104B680009F05BFA4F2009F058FA23E37C4B185DF3
:104B7800013409F052FA0B2CF8D10024794B185D56
:104B8800013409F04AFA082CF8D10024764B185D54
:104B9800013409F042FA072CF8D100F016BC0720BE
:104BA80009F06EFAE72009F038FA6A4B587909F0EB
:104BB80034FA002009F031FA042000F004BCA342C2
:104BC8000AD26A4A9D5C012202FA05F50D421CBF11
:104BD8009A4010430133F2E709F05EFA5D4B93F80F
:104BE800B00745E3122009F04BFA614B1B88B3F577
:104BF800806F8CBF082601260025574C04F134032A
:104C080033F9150090FBF6F0013580B209F03BFA54
:104C1800032DF2D1608F09F036FAA08F09F033FA2C
:104C2800E08FBFE2102009F02BFA0024514B185DE9
:104C3800013409F0F2F9102CF8D1C6E3702009F01C
:104C48001FFA0026444D0E242B6D7443234401366D
:104C5800B3F8250109F017FA2B6D2344B3F827019F
:104C680009F011FA2B6D2344B3F8290109F00BFA66
:104C78002B6D234493F82B0109F0CFF92B6D2344B6
:104C880093F82C0109F0C9F92B6D234493F82D01F1
:104C980009F0C3F92B6D234493F82E0109F0BDF9EF
:104CA8002B6D1C44D4F82F0109F0F6F9082EC9D150
:104CB8008BE37020274C09F0E3F904F1700594F8B0
:104CC800D00009F0AAF994F8D10009F0A6F994F8EF
:104CD800D20009F0A2F994F8D30009F09EF994F8EB
:104CE800D40009F09AF994F8D50009F096F9073438
:104CF80094F8CF0009F091F9AC42E0D165E31E4B7E
:104D0800185D013409F089F9102CF8D15DE31B4DC9
:104D18002878400000F0FE0009F0B2F900242B7852
:104D28009C4280F05283164B33F8140009F0ABF91B
:104D38000134F4E7084C062009F0A2F9606F09F085
:104D4800ABF9B4F87800A4E2042009F099F9024B11
:104D5800D86F38E3D0160020980F0020A34C010824
:104D68000F6801081B680108F3670108B10F0020EC
:104D78000C000020D80F0020EC0F0020B81E0020E7
:104D8800AC2B0020072009F07BF9CC4BCC4C1888C1
:104D9800FF28A8BFFF20C0B209F03FF9D4F880006F
:104DA8004FF6FF75A842A8BF284620EAE07080B2F7
:104DB80009F069F9B4F8840009F065F9C14BD4F831
:104DC800880093F885313BB10A235843A842A8BF0D
:104DD800284620EAE07001E000F30F0080B258E2B4
:104DE800022009F04DF9B64BB3F88C0051E2B44CEF
:104DF8000B2009F045F9D4F89030187809F00DF92E
:104E0800D4F89030587809F008F900262546D5F8E6
:104E18009030AB4C33440136187909F0FEF8032E74
:104E2800F5D1D4F89030D87909F0F7F8D4F8903063
:104E3800987809F0F2F8D4F89030D87809F0EDF8BD
:104E4800D4F89030588909F01EF9D4F89030187ABF
:104E58000EE29B4C1E2009F013F9236D1B78022BE0
:104E68004FF000056BD1236D03EB850393ED080A22
:104E7800B2EE048A20EE080A0EF0DCFA80F308008D
:104E8800C0B209F0CAF8236DDFED8F7A03EB850312
:104E980093ED0B0A20EE270A0EF0CCFA80F30800F7
:104EA800C0B209F0BAF8236DDFED887A03EB850309
:104EB80093ED0E0A20EE270A0EF0BCFA80F30800E4
:104EC800C0B2013509F0A9F8032DCCD1072D236D07
:104ED80023D193ED110A20EE080A0EF0ABFA80F305
:104EE8000800C0B209F099F8236D93ED120A20EE7C
:104EF800080A0EF09FFA80F30800C0B209F08DF896
:104F0800236D93F84C3000EE103AB8EE400A0EF0DC
:104F180091FA80F30800C0B20BE02B44587809F0EE
:104F28007CF8236D2B44D87A09F077F8236D2B444D
:104F3800587D013509F071F80A2DC7D145E2236D76
:104F48002B44587809F069F8236D2B44D87A09F076
:104F580064F8236D2B440135587D09F05EF80A2D5D
:104F6800EDD132E2564D9FED598A2B6D03EB840348
:104F780093ED080A20EE080A0EF05CFA80B209F0F8
:104F880082F82B6D03EB840393ED0B0A20EE080ADD
:104F98000EF050FA80B209F076F82B6D03EB84031B
:104FA80093ED0E0A20EE080A0EF044FA013480B29E
:104FB80009F069F8032CD5D1072C2B6D16D193ED88
:104FC800110A20EE080A0EF035FA80B209F05BF8F3
:104FD8002B6D93ED120A20EE080A0EF02BFA80B220
:104FE80009F051F82B6D93F84C000BE023445878E6
:104FF80009F049F82B6D2344D87A09F044F82B6D51
:105008002344587D013409F03EF80A2CD4D1DCE160
:1050180014F8010F002800F0D88108F0FEFFF7E728
:10502800012009F02DF8264B1B6D187820E150203F
:1050380009F026F80025224B1C6D254B04EB85044E
:105048000C2194F8852001FB0233013593F83800D0
:1050580008F0E3FF94F8860008F0DFFF94F8870073
:1050680008F0DBFF94F8880008F0D7FF142DE2D190
:10507800ABE1482009F004F80025114B1C6D06230C
:1050880003FB0544013594F8DA0008F0C6FF94F8EC
:10509800D50008F0C2FF94F8D60008F0BEFF94F8D7
:1050A800D70008F0BAFF94F8D80008F0B6FF94F8D3
:1050B800D90008F0B2FF0C2DDFD186E1A02B00202B
:1050C800980F0020D01600200000C84200007A4443
:1050D800A44C01084FF0000801260027CB4B1A7E8C
:1050E800974227DA19330024FA5CC94D0C2305F1DD
:1050F80030016343595C914207D12B44586B0DF042
:10510800CEFF82462EB9B14605E001341C2CECD105
:105118000EE080440CE0D1450ADA0C2303FB04536B
:105128005B6B13F8090008F078FF09F10109F2E751
:105138000137D3E7002E00F048815FFA88F008F0C5
:105148009FFF0026C9E7B14D287E08F099FF00248B
:105158002B7E9C4280F03981AE4BE65C0021AC4846
:105168000C2200F1300702FB01F3DA5DB24205D1EF
:10517800034493F8380008F050FF02E001311C297D
:10518800EDD10134E4E7082008F07AFF0124E0B209
:10519800013408F042FF092CF9D116E1082008F083
:1051A8006FFF002008F06FFF002008F06CFF002060
:1051B80008F069FF00206CE00C2008F061FF964BB6
:1051C800186808F069FF954B186808F065FF944B5C
:1051D8001868F8E0042008F053FF924B9868F2E052
:1051E80094F87A0108F019FF94F87E0108F015FF89
:1051F80094F87D0108F011FF94F87F0138E0894C9C
:10520800072008F03DFFB4F8800108F03CFFB4F82F
:10521800820108F038FF94F8840108F0FEFEB4F823
:10522800860136E0012008F02BFF7E4B58791FE0FD
:105238007D4C7E4D207800EB4000C0B208F020FF86
:10524800002623789E4205F1020580F0BE8015F8FD
:10525800020C08F0E2FE15F8010C00EB800000EBF0
:10526800800000F2EE2080B208F00DFF0136E8E77A
:1052780008F0D3FEA9E0082008F002FF0024694BDB
:105288002344013493F8880108F0C7FE082CF6D1AE
:105298009BE008F0F8FE98E05C4B624C93F89400B1
:1052A800C0EBC000C0B208F0EBFE04F1280594F88A
:1052B800F00100235E4AD25C904200F08A800C33F1
:1052C8003C2BF7D10834AC42F1D17EE04020554C5C
:1052D80008F0D6FE04F14005B4F8A80208F0D3FEA1
:1052E80094F8AA0208F099FE043494F8A70208F08A
:1052F80094FEAC42F0D168E0E0204A4C08F0C0FED1
:1053080004F18005B4F82A0200F03F0008F0BBFE63
:10531800B4F82A02C0F3861008F0B5FE94F8280203
:10532800000908F07AFE94F8280200F00F0008F04F
:1053380074FE043494F8250208F06FFEAC42E1D103
:1053480043E03C4C0D2008F09BFE06F0FEFD08F003
:1053580064FEA08808F0A0FE206908F09DFE01F018
:1053680055F830E008F050FE0546842008F088FE25
:10537800284608F091FE2F4B1C6905F18003A342D3
:105388008CBF641B802401F0F9F828462246694640
:1053980006F010FE00240546AC4216DA1DF804009B
:1053A80008F03BFE0134F7E7132008F069FE0024FB
:1053B800214B185D013408F030FE0B2CF8D1002089
:1053C80008F06AFE002008F067FE012018E00020BF
:1053D80016E008F022FEB4F8F20108F054FE94F842
:1053E800F40108F01AFE94F8F50108F016FE94F896
:1053F800F70108F012FE94F8F60108F00EFE61E7D6
:1054080020B0BDEC028BBDE8F08700BF980F0020EC
:10541800A44C0108B10F0020ACF7FF1FB0F7FF1F25
:10542800B4F7FF1FD0160020B81E00207018002007
:10543800C41E00200C0000200F68010810F80A3C68
:105448000133DBB20A2B84BF10F8131C044A00F89E
:105458000A3C82BF002322F8113000F80A3C70474A
:10546800182A0020334A136C90681944081A40F629
:105478008C23984270B513469160D06051603BD937
:10548800127893F945108A4210460BD1111F08294A
:1054980008D893F84610182901D8013103E083F899
:1054A800442002E0002183F8461093F94440214942
:1054B800A24219D191F84740B4B10C31002494426A
:1054C80006DA1D4D51F8046F25F814600134F6E72B
:1054D8000C2805D01849002421F810400130F7E7BE
:1054E800164801780131017083F845200022012116
:1054F8001A7083F8471070BD92F84710C9B1A0F22E
:10550800EF2440F2DA518C4208D811780B2905D8DB
:105518000B1D0131117042F8230070BD002283F881
:105528004720074B03F13002002143F8041F934240
:10553800FAD170BD08010020182A0020ED050020CE
:1055480014010020024A136C013319441164704796
:1055580008010020024B53F820301B68196070477F
:105568001C2C0020064B53F820301A681B89A1F523
:105578007A7159434FF47A7391FBF3F111607047D4
:105588001C2C0020054B98420CBF054A054A13887D
:1055980001339BB213800020704700BF00540040C5
:1055A800A00F0020A20F0020F0B5046D86682368C4
:1055B80023F0010323608379054613F0020F407935
:1055C8000CBF4FF0000E4FF4005E13F0040F14BF31
:1055D8004FF48067002710F0010F14BF0421002149
:1055E8008307206820F001002060626822F440529E
:1055F8004EEA02026260226822F4B05323F00C03E0
:1056080048BF41F008013B430B432360A36895B0B2
:1056180023F44073A360684603F028FA284B9C42A1
:1056280001D10C9B0EE0274B9C4201D10D9B09E058
:10563800254B9C4201D10E9B04E0244B9C420CBF9D
:105648000F9B109B2268A879170448BF5B00B3FB27
:10565800F6F206FB1233B3EB560F236828BF01326C
:105668001E0441BF4FF6F073C2F34201134041EAF2
:1056780003026B7992B213F0020FA28100F00101CC
:1056880014BF4FF400320022DC0748BF42F48032D6
:105698002B6D11B159680A4302E0596821EA0202E8
:1056A8005A609A6801074CBF42F0080222F00802CB
:1056B8009A601A6842F001021A6015B0F0BD00BF86
:1056C800003801400044004000480040004C0040C1
:1056D8001FB50123ADF808300023ADF80C30ADF844
:1056E8000A30094BADF804101B78ADF80620012BE1
:1056F80008BF032301A908BFADF80C3003F0F3F885
:1057080005B05DF804FB00BF0401002038B510F8AF
:105718000E2C50F8043C044652B9012200F80E2C15
:1057280020F80C1C997A18680222BDE83840CFE7A7
:1057380030F80C2C20F80A1C891A89B220F8081CA9
:10574800074A10F80F0C002522F8101004F80E5C18
:105758001868997A2A46FFF7BBFF04F8065C38BD3B
:10576800182A0020044B53F820301BB107289CBF8F
:105778001B681960704700BF30020020074A136891
:105788009B060AD5064B00211970064908684FF692
:10579800FE7303400B6020235360704700000240F3
:1057A800D12F00201C0002402DE9F047664D2B68E0
:1057B80066490A78581C02F0FF068E460AB103466D
:1057C800F6E72B60687BAB6895F80C80AA7B3746B8
:1057D80039B2202900F09B80DFF880C10CEB8103EF
:1057E8003CF82110DC789B78C3F1FF039BB2002BB7
:1057F80065D0C3F1FF0363434FF03C0C1B12B1FBB0
:10580800FCF9B9F1050F5DD8DFE809F0030B1A2997
:105818003A4AE01ADAB24143B1FBFCF01044C0B294
:1058280051E0B1FBFCF00CFB101189B2DAB2C1F106
:105838003C01E31A4B432046B3FBFCFC94442CE0A8
:10584800B1FBFCF00CFB10115FFA83F8E21A89B285
:105858004A43B2FBFCF24244D2B2204632E0B1FBEA
:10586800FCF90CFB191189B25FFA83F8E01AC1F14F
:105878003C014843B0FBFCF04044C0B2224621E062
:10588800B1FBFCF80CFB1811D8B289B2E31A01FB82
:1058980003F2B2FBFCFC224684445FFA8CF412E06B
:1058A800B1FBFCF80CFB181189B2D8B2C1F13C016C
:1058B800E31A4B43B3FBFCF20244D2B203E02246A4
:1058C800204600E044464FEA042C4CEA004C4CEADF
:1058D800020C172306F117014FF0010808FA03F824
:1058E800C91A18EA0C0F89B2DFF8748014BF4FF098
:1058F80011094FF0090913F1FF3308F80190E9D2B3
:1059080018360137B6B2BFB2114BA04660E7AA738A
:10591800AB60104AE98001238EF800300E4985F803
:105928000C8040F22A336873AE80536000234B62C8
:105938000B889BB243F001030B80136843F001030B
:105948001360BDE8F08700BF30100020D12F002081
:105958003C1000201C000240002C0140940D002047
:105968009002002073B506460D46002401232A88BC
:10597800A34013421AD0AA78009302F003038DF8CB
:105988000430EB78022B03D0032B0CBF0323012335
:105998008DF805303046C2F301136946C2F381021F
:1059A8008DF806308DF8072008F0C6FF0134102C5A
:1059B800DCD102B070BD2DE9F04F734EF57B074680
:1059C8000C4687B011469A4600686B1C91462246E1
:1059D8004FF0020BF37306F053FB3B897868ADF880
:1059E800043001A98DF806B08DF807B0FFF7BAFFAB
:1059F8000023ADF80A30ADF81230ADF81630702338
:105A08000193BA7A3C68CDF80CA0012306F110087E
:105A18002D01ADF808304FF48073A844ADF810B0EC
:105A2800ADF814300C2A7ED8DFE802F0077D7D7DC2
:105A38000F7D7D7D387D7D7D5E00204601A902F0C9
:105A4800D7FFA36943F0080326E0236A4F4823F0F1
:105A580010032362236A6168A26922F0807222F42B
:105A6800E642844242F4E04206D000F500608442F7
:105A780002D043F0300307E023F0E00321F4406153
:105A880043F0300341F480616160A261C4F838A03A
:105A98002362A36943F40063A36144E0236A3B489B
:105AA80023F480732362226A6168E369844223F0E5
:105AB800730343F0700306D000F50060844202D0FF
:105AC80042F4407207E022F4606221F4405142F44B
:105AD800407241F480516160E361C4F83CA02262E5
:105AE800E36943F008031DE0236A284823F4805340
:105AF8002362226A6168E369844223F4E64343F43B
:105B0800E04342F4405203D000F50060844201D1E2
:105B180041F480416160E361C4F840A02262E36916
:105B280043F40063E3613A7B3B681AB15A6C42F470
:105B380000425A641A8892B242F001021A80BA7A74
:105B48000C2A18D8DFE802F0071717170B171717D2
:105B58000F1717171300721903F134010AE07219AD
:105B680003F1380106E0721903F13C0102E07219F1
:105B780003F14001116135444046A5F818906B6166
:105B880007B0BDE8F08F00BF30100020002C0140A6
:105B9800F8B53A4E3A4C4000C7B24FF42045306849
:105BA800C4F8D050D0F818E01EF4004F05D0AE4627
:105BB800013DBEF1000FF5D116E0D0F804E0314DFB
:105BC8000EEA050545F490353D4345604FF4204500
:105BD800C4F8D050D0F818E01EF0020F2DD1AE4610
:105BE800013DBEF1000FF5D1C4F8D0501FE02946A1
:105BF800013D0029F8D081694906F8D5C4F8D0508C
:105C080020494568294041F0007141F4105141EAAA
:105C18000241394341604FF42041A2B1306885699F
:105C28006D071ED411F1FF31F9D2C4F8D010FFF777
:105C3800A9FC003018BF0120F8BD4FF4204581624F
:105C4800C4F8D050D7E73068C4F8D0100B46826942
:105C580092060CD41A46013B002AF8D1C4F8D03079
:105C6800E5E7416A03F8011B013AD2B2D3E7C4F869
:105C7800D0302023C3610120F8BD00BF9C0F002055
:105C880030100020009800FC400070B5C5B23248C2
:105C9800324B00684FF42044C3F8D040866936047C
:105CA80004D52646013C002EF8D113E046682C4C5A
:105CB800344044F0807444F490342C4344604FF4EE
:105CC8002044C3F8D0408669B60729D42646013C4B
:105CD800002EF8D1C3F8D0401CE02146013C002931
:105CE800F8D081690E06F8D544681D49214041F075
:105CF800007141F48031294341604FF42041C3F8D9
:105D0800D0108469A40711D40C460139002CF8D1AD
:105D1800C3F8D010FFF736FC003018BF012070BD63
:105D28004FF420448162C3F8D040DAE782624FF42E
:105D38002042C3F8D0208169890606D41146013A69
:105D48000029F8D1C3F8D020E4E7C3F8D0202023F5
:105D5800C361012070BD00BF9C0F002030100020DF
:105D6800009800FC426A806A131A584258417047EA
:105D78004171704743799B070AD5436A8269D154B8
:105D8800436A01690133B3FBF1F201FB1233436249
:105D98007047427902F0020202F0FF0342B1036940
:105DA800426A806A013BDBB2101A23EA000070479E
:105DB80018467047437913F001031FBFC36803F106
:105DC800FF32C369006A1DBF181A1040C0B21846D6
:105DD8007047437913F0010310B504460DD0FFF75F
:105DE800E9FF58B1236A6269E168D05C0133B3FB0B
:105DF800F1F201FB1233236210BD184610BD90F872
:105E08003B3210B57BB990F83A3290F83942A34248
:105E180009D2B0F8401201229A400A430133A0F88F
:105E28004022DBB2F3E710BD38B50D4B0D4D1A8A91
:105E38000D4B1968498811421C4603D008F044FFED
:105E4800286007E008F040FF2B68984282BFC01A1C
:105E5800064B186023685868BDE8384002F07EBCDD
:105E68000004004808110020580700200000002006
:105E780038B5A0F513746379A579DB0745D594F88F
:105E8800383205F00105EBB1226B1068C36A5B0874
:105E9800436294F83C3223B1B4F842320133A4F897
:105EA8004232917A6A0006F02EF8012384F83B32D8
:105EB800002384F8393284F83A3284F83832A4F866
:105EC800403238BD94F83B32012B04BF94F8393284
:105ED80084F83A322046FFF792FF94F83B22236B6E
:105EE8003AB9012284F83B221868997A05FA02F235
:105EF80007E0002284F83B2295421868997A08BF87
:105F08000222BDE8384005F0FEBF38BD10B5A0F547
:105F1800127494F83C22BAB9A36A616A994228D0EB
:105F2800591CA069A162C35C2069DBB25B0043F421
:105F380000738142A4F83E324FF00A0384F83D32E0
:105F480028BFA262012312E094F93D327BB1B4F874
:105F58003E124B08A4F83E32204601F0010105F03C
:105F6800E5FF94F83D32013B84F83D3201E084F8C6
:105F78003C3294F83832002B4FD194F8393201333F
:105F8800DBB2092B84F8393203D12046BDE8104032
:105F980035E70A2B41D194F83B322BB9B4F840329B
:105FA80043F00103A4F840326379D9071CD5B4F84B
:105FB8004002820501D4C30705D4B4F84432013342
:105FC800A4F8443210E0E36AC0F347000BB19847E5
:105FD8000AE0E3696269D054E369E1680133B3FB1D
:105FE800F1F201FB1233E361012284F8382294F8BC
:105FF8003B220023012A84F839320ED1A27984F891
:106008003B32236B12F0010F1868997A0CBF0222F9
:106018000022BDE8104005F076BF10BD10B54B88D2
:10602800DC0641BF2F4B14791B6853F8244044BF4A
:106038002D4B43F820404B889B0641BF294B547990
:106048001B6853F8244044BF274B43F820404B8833
:106058001C070ED5254B0C781B78B3EB141FA1BF7A
:10606800204BD4781B6853F82440A4BF1E4B43F838
:1060780020404B889B070ED51D4B0C781B78B3EB43
:10608800141FDFBF174B54781B6853F82440DCBF3C
:10609800154B43F820404B88DC070FD5154C0B787F
:1060A800247803F00F03A342DFBF0E4B14781B685C
:1060B80053F82440DCBF0C4B43F820404B885B0767
:1060C8000FD50B780C49097803F00F038B42A1BF59
:1060D800044B92781B6853F82220A4BF024B43F864
:1060E800202010BDF0150020940D0020471F00202F
:1060F800451F0020441F0020461F0020254A26482F
:1061080026490023F0B5156803700B711C461A4622
:106118002E1976884EB92F5D3FB9037000230A7196
:106128004B7107781C461A460CE0360548BF013209
:1061380004F1040403F1010348BFD2B2802CDBB29E
:10614800E6D1EAE7E0B2B8420CD215F82400060915
:106158009E4200F00F00A8BF731C9042A8BF421CCB
:106168000134EFE78A714B71C2F3470102F0010273
:106178000A444C1E0A490B480A70C3F3470203F04D
:106188000103134404700849501E084A087013702C
:10619800F0BD00BFF41500203C1F002008110020AE
:1061A800461F0020441F0020471F0020451F0020D5
:1061B8002DE9FF47704B714933F9103004462BB96C
:1061C80002280CD06E4B1B88980708D06D4B002214
:1061D80023F814206C4B1B8821F81430C8E031F8E0
:1061E80014301BB9694A02EB8402936001339BB2F5
:1061F80021F814301BB2002B18DD022C634A6448C6
:1062080009D11669B0F90450202095FBF0F505FB7B
:10621800006010610AE002EB840230F914509668BD
:10622800802095FBF0F505FB00609060594F3868B9
:1062380090F85E20934240F09B80544ADFF84481F6
:1062480002EB840200EB040E022C956895FBF3F335
:106258009EF85750936008BF5E424FF0000221F845
:10626800142007BFB6B214219EB20A21002D7DD09A
:10627800002E7BD038F81420002A77D00FFA86F940
:106288000FFA82FCE14571D089EAE9728CEAEC7A6E
:10629800A2EBE972AAEBEC7ACAEB0202B9F1000FA1
:1062A80012B209B2DFF8F89003DDBCF1000F03DC8D
:1062B80020E0BCF1000F1DDA8A420BDD022C90F8B9
:1062C8005A2002D102F580720EE039F814104032DB
:1062D8000A4419E049428A4218DA022C11D190F88E
:1062E8005A20C2F57F42C032B9F804100A44A9F80E
:1062F80004200BE0002AB8BF52428A4206DD022C75
:1063080004D039F81420203A29F8142039F9142037
:106318009EF8549092114A4503DBAA42A8BF2A4628
:1063280091461D4A126812031FFA89F508D51420F0
:1063380001A98DF804400293ADF80C5002F084FED8
:10634800164B1B7873B12AB207EE902AF8EEE77A5B
:10635800B2EE047AC7EE877A3B6803EB8403C3ED99
:10636800087A03E03B68234483F8019028F8146016
:1063780004B0BDE8F08700BF94260020BC070020C9
:10638800A80F0020B6070020AE0700200811002043
:10639800D20F0020A8070020A82B0020AC0700205F
:1063A800B0070020094A13781844C0B210F0800FD3
:1063B80018BF803810701346054A19781378994227
:1063C80001BF00231370014A137070472D28002065
:1063D8002C28002010B50A4B0A4A1B7842609C18EA
:1063E800094A046012789A4225BFD31A0B60C3F198
:1063F800800300232EBF4B600B604A6010BD00BFB6
:106408002D2800202E2800202C2800201FB56846A3
:1064180002A9FFF7DFFF044B02981B6803440398A7
:10642800184405B05DF804FBE00500202DE9F04FA5
:1064380089B0824601930023029103929946039AF8
:10644800934205DA029A52F8232001339144F6E781
:10645800019B4D46002B56D105F077FD002852D1FF
:1064680001987CE002223F4E8DF81C201A0C4FF454
:1064780080578DF81D2006201A0A8DF81E208DF8E9
:106488001F3005F087FD3785062001F023FF364BC6
:10649800B76101221A700020378507A9042201F08C
:1064A80041FF029FD04626464FF0000B039B9B45B9
:1064B8001EDABC4657F8042B4FEA8B03002A47D054
:1064C800B24235D332465AF80310CDF814C0002032
:1064D800049301F027FF049BDDF814C05AF8032049
:1064E80032444AF80320DCF800309E1BCCF80060E8
:1064F8001C4B4FF480529A611C4A13682D1B1C4494
:10650800019B14604BB345B3184B1B68DCB22A19C6
:10651800B2F5807F164AD2688CBFC4F580742C46C9
:1065280093429FD3134A00231370134A137014E045
:106538000020D8F8001001F0F5FE57F8043CD8F810
:106548000020F61A1344C8F80030002347F8043C2A
:106558000BF1010B08F10408A8E7C5EB090009B025
:10656800BDE8F08F00040048DD050020E0050020AC
:10657800100000202C2800202D28002030B50B4CBE
:106588000B4D22782B789A4285B00CD0684602A928
:10659800FFF720FF0123684602A90222FFF746FF02
:1065A80000232B70237005B030BD00BF2D280020BC
:1065B8002C28002030B50E4D0E4C2A7823789A42AC
:1065C80085B011D0684602A9FFF704FF002302A98D
:1065D80002226846FFF72AFFFFF7E4FE20782B78AF
:1065E8001B1A5842584100E0012005B030BD00BFD9
:1065F8002D2800202C280020054A064B10781B78EF
:1066080083422EBF181AC0F18000C018704700BF1F
:106618002D2800202C28002038B50E4C4FF480552A
:1066280045F2082005F0B6FC2585062001F052FE4B
:10663800094BA56101221A70C720258501F04AFE81
:10664800064AA56100231370054A1370054A1360B2
:1066580038BD00BF00040048DD0500202C280020BC
:106668002D280020E0050020FFF7DEBBFFF7DCBB8C
:10667800FFF7DABB2DE9F04F544D1E464FF4147363
:1066880005F11404434385B080469146E718A246B5
:1066980010B92B444E4A03E0012805D14D4A2B443A
:1066A8005A641032C3F848214FF4147303FB08F3FB
:1066B800EC180AEB030203F59C7347486061343217
:1066C80053442164A262E36200224FF0010B4FF4AD
:1066D8008071D4F8483121620320626322636162C9
:1066E800E263A26384F8502284F84CB284F84D2205
:1066F800A4F85622A4F85822C4F81C906076A6760E
:1067080084F85A8204F5A27258681B8901924FF0E6
:10671800020C03A9ADF80C308DF80EB08DF80FC03F
:10672800CDF800C0FFF71EF9636CDDF800C0597B97
:1067380058681B898DF80E1003A9ADF80C308DF838
:106748000FC0FFF70FF95946384605F0EFFB322026
:1067580008F0E1FA019A214BD2F804B0B3FBF9F141
:10676800B1F5803F03D3012BF8D95B08F6E74FF466
:10677800147404FB08F805EB0809584689B2482246
:1067880008F5127805F0CAFC0AEB0804144BC9F89E
:106798005C3200225846214605F016FDD9F84450CF
:1067A80016F0010F0CBF022200222868A97A05F012
:1067B800AAFB0C4BC9F860322846211D002205F0BF
:1067C80003FD384605B0BDE8F08F00BF0811002072
:1067D800D0660108F0660108304E010800A24A049C
:1067E800155F0008795E000803460A4690F84602DD
:1067F800D96A9B793EE700BF38B500240B4D605934
:10680800254407F0C5FC696811B1094803F08FFAFF
:10681800A96811B1074803F08AFA0748103407F04D
:10682800B7FCB4F5E87FE9D138BD00BF544E010884
:10683800C66A0108CC6A01088F77010870B5054659
:1068480028460CF02CFC064658B91A4B1A485A79B7
:106858001A4B03EB8203BDE87040D3F8CC1103F068
:1068680066BA2846164932460CF022FC60B915482B
:10687800154C07F08DFC54F8041F19B1134803F0A8
:1068880056FAF8E7124805E00024124B53F8241092
:1068980021B91148BDE8704007F07ABC2846324655
:1068A8000CF006FC01340028EFD1024B0B4D5C7153
:1068B800C6E700BFD0160020D26A0108544E01086E
:1068C800DE6A0108E36A010820500108F66A010837
:1068D8008F77010824500108FA6A0108AB6901089A
:1068E800F0B585B004460CF0DAFB082826D1621E04
:1068F800E01D1F4912F8013F09681944497801F061
:106908000301022908BF203B82421370F1D12546BA
:1069180004F1080715F8016B164831460CF0B1FB75
:1069280020B1284631460CF0ACFB10B100F02CFF2A
:106938001CE0BD42EED1204601F068FE0E4807F08B
:1069480027FC00230D4A1A4404A992F888210A4416
:106958000849595C02F80C1C0133082BF2D10023BA
:1069680007488DF80C3001A903F0E1F905B0F0BD36
:106978006C0000202D750108096B0108D016002055
:10698800337601082DE9F04105460CF088FB2E4BC3
:1069980004469E6888B92D4807F0FAFB2C4B53F83B
:1069A800241041B10123A340334202D0294803F007
:1069B800BEF90134F2E7284821E028462749224653
:1069C8000CF076FB58B92648264C07F0E1FB54F842
:1069D800041F0029EFD01F4803F0A9F9F7E72B7827
:1069E8002D2B03BF013504F1FF344FF001084FF0A0
:1069F80000080026164B53F8267027B91A48BDE838
:106A0800F04107F0C5BB2846394622460CF050FB3A
:106A1800B8B90120B040030601D51448EFE7B8F132
:106A2800000F03D003F0ACFA114802E003F0B0FA0B
:106A3800104807F0ADFB39460F48BDE8F04103F0B8
:106A480076B90136D6E700BFD01600200F6B0108D3
:106A58008C500108F66A01088F770108DE6A010880
:106A6800196B010888500108FA6A0108256B0108AA
:106A7800336B01083C6B01083276010810B50848F1
:106A880007F086FB074B00241C701C63064B1C7028
:106A980008F04EFB07F02EFD044B1C6010BD00BF34
:106AA800446B0108BC150020D32F0020D4280020F7
:106AB80070B5064600240B4BE518AA8816420AD082
:106AC800E158094803F033F92846002107F0EDFAA8
:106AD800064807F05DFB143440F6CC339C42EAD1FB
:106AE80070BD00BF645A0108706B01088F770108F8
:106AF80008B5084803F01BF9FFF78EFD05F025FAE5
:106B080018B9642008F007F9F8E70348BDE8084019
:106B180003F00DB97A6B0108876B01082DE9FF4175
:106B28000A48068885684488B0F80480C768FFF773
:106B38006DFCCDF800800290019731462A46234625
:106B4800034803F0F4F804B0BDE8F0811000002019
:106B58008F6B0108F0B504788BB005460CB10024A2
:106B680036E04B4B19680E2303FB041101F59070B6
:106B7800B1F92951B1F92521B1F92731009591F8D9
:106B88002C51019591F82D51029590F90B00039025
:106B980001F594713F4891F906100491214601349A
:106BA80003F0C5F8082CDCD170E02D2B14D1072C8C
:106BB8001BDC28460CF0CAFA0AAB661C03EB44043B
:106BC80024F8100C15F8013F303B092BFAD934464C
:106BD8002B78002BE9D104E0A3F13002092A09D867
:106BE800E5E7082CBDF8182009D00BB0BDE8F04047
:106BF80000F0CABD202BF8D101352646E7E7072A61
:106C0800F3D8BDF81A00224BA0F2EE2189B240F267
:106C1800DC55A9421B68E8D8BDF81C10A1F2EE2487
:106C2800A4B2AC42E1D8BDF81E6004B237B2A742A4
:106C3800DBDB0DB2AF42D8DCA542D6DBBDF8247051
:106C480007F16404A4B2C82CCFD8BDF826E00FFA27
:106C58008EF4112CC9DCBDF82050B42DC5D8BDF870
:106C68002240B42CC1D812B24FF00E0C0CFB0233E8
:106C7800A3F82501A3F82711A3F8296183F82C515B
:106C880083F82D4183F82B7183F82EE10BB0F0BD0A
:106C9800E80F0020EC6B0108F0B504468FB02046E1
:106CA8000CF0FDF9C5B225BBAF48B04C07F070FA3F
:106CB80094F8D21009B9AE4854E049B294F8D020FB
:106CC80094F8D130009194F8D310019194F9D4102C
:106CD800029194F9D510039194F8D6100491A5481F
:106CE8002946013503F023F8102D04F10704DFD1FC
:106CF800E1E72046A04905220CF0DAF90546B8B9C3
:106D080029469E4870220CF086F99D4B1968284642
:106D18000E2303FB001301300022082883F82F21DB
:106D280083F8302183F8312183F83221F0D119E139
:106D38002046944904220CF0BBF905462046002D54
:106D48004AD120210CF09DF9002800F00B81461C47
:106D580030460CF0A4F92C4607468B4B53F82450C8
:106D68002DB98A480FB0BDE8F04002F0E0BF3046C8
:106D78002946FAB20CF09CF901340028EDD17B4A7F
:106D880002F170011646002382F8D63082F8D2301C
:106D980082F8D13082F8D03007328A42F3D17C4968
:106DA80001EBC40191F89022934210DAD1F8947261
:106DB800C3EBC302B0183A4400F1D0011768C0F819
:106DC800D0709088888092798A710133E7E72946E4
:106DD800704802F0ACFF96E06F4907220CF068F9A2
:106DE80005462046002D4AD120210CF04AF90646D6
:106DF8000CF055F9C4B274BB684802F098FF2146FC
:106E08006748013402F093FF0E2CF8D1584802F07D
:106E18008EFF00246348214602F089FF0025584A66
:106E2800614811680E2202FB04120123D2F82F21B7
:106E38005E49AB4013425E4B05F1010508BF194698
:106E480002F075FF0E2DEAD14948013402F06FFFB8
:106E5800082CDFD186E0304656490CF07BF92C46E9
:106E6800002852D0022C55D00CF070F906AB5149CD
:106E780043F8240000200CF06DF90134F0E74D4987
:106E88000CF068F9002460B1082C3ED00CF05EF9D3
:106E980006AB484943F8240000200CF05BF90134A4
:106EA800F1E7082C31D1069B0F2B2ED8DDF81CE01A
:106EB800BEF1070F29D8089F0D2F26D8099E06F185
:106EC8006402C82A21D80A9DFF2D1ED80B98642871
:106ED8001BD80C99642918D8884216DA0D9C032C03
:106EE80013D8224AC3EBC303134483F8D0E083F8D2
:106EF800D17083F8D26083F8D35083F8D40083F834
:106F0800D51083F8D6402C4CC9E60FB0BDE8F04048
:106F180000F03ABC069B072B20D807990D291DD8ED
:106F28000278722A0DD06E2A18D1154A12680E20DE
:106F380000FB032301228A40D3F82F1121EA020221
:106F480009E00F4A12680E2000FB032301228A4041
:106F5800D3F82F110A43C3F82F2101E000F014FCE5
:106F68000D4C9CE60FB0F0BD146C0108D016002043
:106F78008F7701083F6C01085B6C0108A01700209F
:106F8800E80F0020616C010824500108FA6A010822
:106F9800544E0108666C01080C6C0108D06A01089F
:106FA800726C01084B760108776C0108FD790108BD
:106FB8009D7A01087B6C0108AB6901082DE9F7434C
:106FC800047805468CB9324D95F8AB12B5F8A8226D
:106FD80095F8AA322F4800912146013402F0A7FE05
:106FE800102C05F10405EFD14EE00CF0AFF80F2896
:106FF800044636DC284620210CF043F8264EE4B23D
:10700800D6F83480451CA400002728460CF09EF8CA
:107018005FFA87F9B9F1010F83B208D0B9F1020F0D
:107028000BD0B3F5B47F24D2726B13530AE0FF2B55
:107038001FD8736B2344987004E0FF2B19D8736B27
:107048002344D87028462C210CF01BF8054608B1BB
:10705800013502E0B9F1020F0BD10137032FD4D16A
:1070680012E00E4800210F2203B0BDE8F04300F003
:1070780008BB08EB0400002104220BF0CCFF03B08E
:10708800BDE8F04300F080BB03B0BDE8F08300BF6B
:10709800D01600207D6C0108BC150020916C0108F9
:1070A8002DE9F04304788FB00546002C59D17C4B6C
:1070B8000021142209A807AED3F838800BF0ABFFE3
:1070C8000722304600210BF0A6FF05A80023A700E1
:1070D800059308EB070583801A467249B5F802E064
:1070E80031F813C01CEA0E0F0AD00DF1380C0E311E
:1070F80002F1010E6244595C02F81C1C5FFA8EF220
:107108000133072BE9D100210B46674AB5F802E0A5
:1071180011F802C01CEA0E0F0AD00DF1380C063225
:1071280003F1010E63448A5C03F8242C5FFA8EF3A2
:1071380001310629E9D118F807305C498DE841008A
:107148006A78029209A81A0903F00F0301F0ACF952
:107158002146574809AA013402F0E9FD202CA6D19E
:107168009BE00BF0F3FF1F28044600F389802846B4
:107178002021E4B20BF085FF1F2C02D900F004FB9C
:107188008BE0474B9B6B03EB8404451C0021204696
:1071980004220BF040FF0027464B09AE3046002181
:1071A8000A2217F803905FFA87F80BF034FF0023E0
:1071B80015F8012B32B10A2B04D04A4502D0F254FB
:1071C8000133F5E74A4561D108F1FF33032B09D8AC
:1071D800DFE803F0100502420DF1230037E00DF15E
:1071E80023011FE030460BF0B1FF2378C0B243EA19
:1071F800001006E030460BF0A9FF237800F00F00DE
:107208001843207034E00133062B0BD02A4800F2D3
:107218007B369E5D9642F6D1034493F875236388C6
:107228001343638011F8012F12B30023EEE70133F3
:10723800072B0CD0204A02F26E369E5D8E42F6D1A4
:1072480002EB4303B3F8602363881343638010F8A9
:10725800011F69B10023EDE730460BF077FF0F28D7
:1072680004DC30460BF072FF607001E000236370AD
:107278000137052F90D10124FEF740FF6CB97DE757
:107288000E4800211F2200F0FCF906E020460021EC
:1072980004220BF0C0FE0024EEE70FB0BDE8F08337
:1072A800BC150020B4510108C9510108976C0108A8
:1072B800A66C0108D5510108544E0108916C0108CB
:1072C8002DE9F0412DED048BB1498AB004460BF04D
:1072D800ABFEB049002820460CBF012607260BF05C
:1072E800A3FEAD490028204608BF02260BF09CFEED
:1072F800002808BF0426F10740F1F080A748A84CF1
:1073080006F046FF002006F04BFDA64806F040FFB9
:10731800A54806F03DFF6279A44BA54803EB82031C
:107328002546D3F8CC1102F002FDA24802F0FFFC7A
:107338004FF00008274695ED048AB5EE408AF1EE35
:1073480010FA04D19C4802F0F2FC002570E09B483A
:10735800D5ED059A95ED069AD5ED078A414602F0D6
:10736800E6FCB5EEC08AF1EE10FA02D5202006F050
:1073780007FFB0EE480A06A802F06EFB01469048E7
:1073880002F0D5FCF5EEC09AF1EE10FA02D52020F5
:1073980006F0F6FEB0EE690A06A802F05DFB0146AB
:1073A800874802F0C4FCB5EEC09AF1EE10FA02D597
:1073B800202006F0E5FEB0EE490A06A802F04CFBD4
:1073C80001467F4802F0B3FCF5EEC08AF1EE10FAF0
:1073D80002D5202006F0D4FEB0EE680A06A802F016
:1073E8003BFB08F101080146764802F0A0FCB8F121
:1073F8000C0F05F110059ED1A4E749B294F8D020EE
:1074080094F8D130009194F8D310019194F9D410E4
:10741800029194F9D510039194F8D61004916A4812
:107428002946013502F083FC102D04F1070403D02E
:1074380094F8D2100029E0D16448654C06F0A8FE03
:10744800D7F8088054F8041F19B1624802F06FFC9D
:10745800F8E70D46604B53F8254054B10123AB4083
:1074680013EA080F03D05D48214602F060FC01359D
:10747800F0E75B4806F08CFE21467B180AAA93F8D1
:1074880088311344574A8A5C03F8102C01310829C3
:10749800F3D1002306A954488DF8203002F047FCA8
:1074A800524806F075FE524800F026FD514806F095
:1074B8006FFE4F48FFF7F4FD4F4806F069FE4C4851
:1074C800FFF77CFD4D4802F032FC4020FFF7F0FA50
:1074D8004B4806F05DFE464800F080FBB20739D500
:1074E800484806F055FE484806F052FE404806F067
:1074F80097FC464806F04CFE3D4800F0CFF844485B
:1075080006F046FE3A4800F0BBFA424802F00FFC8B
:10751800374800F03FF9404806F03AFE3448FFF794
:1075280019FB00270E257D4300243C4AD26B2A44D0
:107538000123D2F80A20A34013421ED101340E2C95
:10754800F3D10137082FEDD12C4802F0F0FB802051
:10755800FFF7AEFA730716D5314806F019FE314821
:1075680006F016FE224806F035FC244802F0DFFB40
:107578004FF48070FFF79CFA05E0394622462A4806
:1075880002F0D5FBDAE70AB0BDEC048BBDE8F08168
:10759800B26C010801710108B96C0108BF6C0108DF
:1075A800D0160020CD6C0108DF6C0108544E01088C
:1075B800EB6C0108F66C0108036D0108106D0108F9
:1075C800CF6A010833760108286D0108186D010893
:1075D80088500108476D01088C500108556D010855
:1075E800626D01082D7501086E6D0108776D01083F
:1075F800AB690108866D0108926D01088F77010853
:10760800A06D0108AD6D0108C06D0108CE6D0108BF
:10761800D86D0108E76D0108F56D0108BC1500205B
:10762800016E0108126E0108246E0108F8B50446BF
:107638000E4617460025204620210BF022FD044661
:10764800D0B1013420460BF081FDB0F5617F05DB38
:1076580040F634039842A8BF184601E04FF4617021
:10766800A0F56170192390FBF3F00DB9307000E0BC
:1076780070703B7801333B700DB90125DBE720467C
:10768800F8BD30B505460C46134629462246024841
:10769800BDE8304002F04BBB0C7401087FB504789C
:1076A8000646E4B9354B1B6803EB8403192193F8AC
:1076B800870093F8886093F8852093F886304FF414
:1076C800617511FB005011FB0651009001912C4887
:1076D8002146013402F02BFB142CE3D14BE00BF0D4
:1076E80035FD1328054641DC244B701C1C682021FD
:1076F80000238DF80F300BF0C4FC2035064670B11E
:10770800013630460BF022FD1A289FBF04EB850393
:1077180058719DF80F30013398BF8DF80F303046FF
:1077280020210BF0AEFC064670B1013630460BF056
:107738000DFD0D289FBF04EB850398719DF80F3050
:10774800013398BF8DF80F3004EB85043046E11DF6
:107758000DF10F02FFF76AFF9DF80F30042B0AD0D6
:10776800601D002104220BF056FC04E005480021AE
:107778001322FFF786FF04B070BD00BFE80F00209A
:107788002B740108916C0108014806F001BD00BF87
:1077980040740108F8B50478064674B9304DB5F858
:1077A800C421B5F8C6312F482146013402F0BFFA8A
:1077B800042C05F10405F2D1F8BD2B490BF034FC7B
:1077C800A8B9274B4FF47A714FF4FA62A3F8C411A1
:1077D800A3F8C621A3F8C811A3F8CA21A3F8CC11AD
:1077E800A3F8CE21A3F8D011A3F8D221F8BD3046D2
:1077F8000BF0ACFC032805462BD8304620210BF0B3
:1078080040FC044630B1013420460BF09FFC0126B1
:10781800074600E00646204620210BF032FC10B94E
:10782800BDE8F840B0E701300BF090FC012EF7D12D
:10783800A7F2EE2240F2DC539A42F1D8A0F2EE22EF
:107848009A42EDD8064B703503EB85039F80D880AC
:10785800F8BD064800210322BDE8F84011E700BF43
:10786800D01600204E7401085B6C0108B578010839
:107878002DE9FF4104780546002C39D17348744D31
:1078880006F086FCD5ED047AF5EE407AF1EE10FAB2
:1078980000F0D88021466F4802F049FA95ED040AB5
:1078A800684602F0D9F801466B4802F040FA95EDB7
:1078B800050A684602F0D0F80146674802F037FA30
:1078C80095ED060A684602F0C7F80146624802F0DC
:1078D8002EFA95ED070A684602F0BEF80134014613
:1078E8005E4802F024FA0C2C05F11005CAD1A9E073
:1078F8005B4905220BF0DCFB40B9554B03F1C00294
:10790800002143F8101F9342FAD19BE028465549BD
:1079180004220BF0CDFB04462846002C40D1202140
:107928000BF0AFFB002800F08D80451C28460BF0BB
:10793800B6FB07464C4B53F824601EB94B4806F07B
:1079480027FC7FE028463146FAB20BF0B1FB013440
:107958000028EFD13E4B03F1C0029E46002143F8B8
:10796800101F9342FAD1424B03EBC4029846D2F857
:1079780004C0BCF1000F04D131463E4802F0D7F9EB
:1079880057E0002718F834309F42F5DA3B010EEB38
:10799800030563440FCB103585E80F000137F1E785
:1079A8000BF0D4FB0B28064647DC284620210BF0B9
:1079B80068FB054650B10135284601F0C3FF244B4A
:1079C80003EB061383ED040A012400E0044628466D
:1079D80020210BF056FB054648B10135284601F039
:1079E800B1FF1B4B03EB061383ED050A0134284650
:1079F80020210BF046FB054648B10135284601F029
:107A0800A1FF134B03EB061383ED060A0134284646
:107A180020210BF036FB10B9FFF7B6FE12E001305B
:107A280001F090FF0A4B032C03EB061686ED070ABC
:107A3800F2D11148FFF71CFF04E0104801210C2285
:107A4800FFF71FFE04B0BDE8F08100BF61740108B4
:107A5800D01600207C74010882740108337601086E
:107A68005B6C0108616C010824500108FA6A01087E
:107A78003C730108666C0108AB690108916C010848
:107A8800F0B5047887B006461CBB514B196806232D
:107A980003FB0411192091F8D65091F8D77091F88A
:107AA800DA2091F8D5304FF4617610FB056510FBAC
:107AB80007600095019091F8D8000290D0314548B0
:107AC800497A03912146013402F031F90C2CDCD1BA
:107AD8007CE00BF03BFB0B28044672DC3C4B701C33
:107AE8001D68202100238DF817300BF0CAFA0646CE
:107AF80080B1013630460BF029FB03289FBF0623CF
:107B080003FB045383F8DA009DF817309CBF013358
:107B18008DF81730304620210BF0B3FA074680B1B4
:107B2800013738460BF012FB0D289FBF062303FBD5
:107B3800045383F8D5009DF817309CBF01338DF8A6
:107B4800173006266643A9193846D6310DF11702B3
:107B5800FFF76CFD20210BF094FA074670B101374E
:107B680038460BF0F3FA14289FBF9DF817307619A2
:107B7800013386F8D80098BF8DF817303846202191
:107B88000BF07FFA78B101300BF0E0FA0D289FBFB7
:107B9800062303FB045383F8D9009DF817309CBFD4
:107BA80001338DF817309DF81730062B0ED00622BA
:107BB80002FB04500021D5300BF02DFAFFF7E4FD4D
:107BC80004E0054800210B22FFF75BFD07B0F0BD7C
:107BD800E80F002086740108916C01082DE9F3472D
:107BE800047807464CB9204601A900F02DFD013460
:107BF800FFF7F4FF122CF6D179E00BF0A7FAC5B223
:107C0800112D6FD8781C20210BF03BFA394C3A4FD4
:107C180005F1D006034614F8168030B9A8F102021F
:107C2800D2F1000848EB020843E000F1010A597854
:107C380038460BF026FA60B1032D8CBF03230023CE
:107C4800C01B3B4453FA80F090F80490B9F1030F3D
:107C580002D1FFF799FD4AE0A9F10203D3F1000828
:107C680050464FF0200148EB03080BF00AFAD8B150
:107C7800B8F1000FEDD001300BF068FA40F2ED23B7
:107C880080B2984205DD40F6CA039842A8BF18465C
:107C980001E040F2EE2004EB4603A0F2EE201922A8
:107CA80090FBF2F0587002E0B8F1000FD1D104F85F
:107CB800169014F81630FA5CB8F1000F0DD00D4B81
:107CC8000E4803EB46062946737840F2EE24192540
:107CD80005FB034302F02BF809E02946084802F0A7
:107CE80026F804E0074800211122FFF7CAFC02B079
:107CF800BDE8F087D016002098520108A674010844
:107D0800B8740108B578010807B50123ADF8041067
:107D180001A98DF806208DF80730FDF723FE03B082
:107D28005DF804FB2DE9F041054672B64FF0904628
:107D38004FF480614FF4007731853046042237854F
:107D4800FFF7E2FF304639460122FFF7DDFF2C48F6
:107D580050F8354000EBC500236842680125510002
:107D680005FA01F848EA030395402360A561B76165
:107D78004FF090431B8A5E05FAD4236848EA030350
:107D880023604FF090434FF40072A9B221851A8501
:107D98000822C3F8182440F605564FF090473B8A4E
:107DA800580503D4002EF8D0013EF6E7A561204619
:107DB8000422FFF7A9FF96B14FF090431A8A5205A3
:107DC800DBD5228A92B215420E4A4FF400704FF06A
:107DD800080115BF9861188591611185ECE7094B79
:107DE8004FF400710822B96138469A610222FFF700
:107DF8008BFF62B60A20BDE8F04106F08CBF00BFD9
:107E0800E874010800040048002208490C2303FB19
:107E180002135968814204D10022C2621A725A6060
:107E280070470132052AF0D1704700BFC41E0020F8
:107E38002DE9F74389469DF8288011461A469DF892
:107E48002C30064600250C2068431D4FC419C05726
:107E5800B04202D1207A20B12DE00135052DF2D1B2
:107E680029E0022E0FD005DC56B1012E23D1009354
:107E780014480AE01E2E0ED01F2E1CD101200AE045
:107E88000093114801E011480093434604F0DCFADE
:107E9800044638B90FE0FEF7EDFB036841469B69DD
:107EA800044698470C2303FB05752671204685F880
:107EB80008906C6000E0002003B0BDE8F08300BFCC
:107EC800C41E002000440040003801400048004023
:107ED80010B5084B1968002201EBC20393F9024060
:107EE800844201D1981C10BD0132052AF4D100202A
:107EF80010BD00BFC01E0020F0B5027887B08AB957
:107F08004A4C04F1280694F8F021002348495956B0
:107F180050B281426ED00C333C2BF7D10834B442B6
:107F2800F1D181E0002204920592451C0BF00EF974
:107F3800C4B260B2FFF7CCFF074618B18DF8104005
:107F4800012400E00446284620210BF09AF8054653
:107F580038B1013528460BF0F9F80134ADF81200B4
:107F6800E4B20026284620210BF08BF8B0B3451C5C
:107F780028460BF0EBF800222E4951F822308342B4
:107F88005FFA82FE04D00132082AF5D1002300E00E
:107F9800734651F82320824220D1022E0FD0032E9F
:107FA80012D05A1E012ED2B204D0042A13D88DF84A
:107FB80014300EE0042A0ED88DF8153009E0052B90
:107FC80009D88DF8173004E09A1E052A03D88DF8D1
:107FD80016300134E4B20136042EC3D1052C04D87E
:107FE80007B0BDE8F040FFF7CFBB04AB03CB386068
:107FF800796019E094F8F5010E4B94F8F45153F8B0
:108008002000B4F8F221009094F8F70153F820000A
:10801800019094F8F60153F82000029053F82530A7
:10802800054801F084FE79E707B0F0BDD0160020BE
:10803800C41E002064570108C774010838B143887A
:1080480011EA030003D08B420CBF012002207047C5
:1080580030B50A4B0A491C680A78042A0AD813461C
:1080680004EBC303551CEAB29D882842F5D00A7078
:10807800981C30BD0A70002030BD00BFC01E002013
:10808800FC150020014B00221A70E1E7FC150020C6
:108098002DE9F047877890F803C0214DBBB2C7F1AE
:1080A800640E03EB83065C42C3F178005FFA8EFE30
:1080B8007600CCF16408A4B280B2A3B20FFA83F9B7
:1080C800B9F1000F05DC002B14BFBA464FF0010AC6
:1080D80000E0F24613FB03F303FB0CF21AFB0AF36E
:1080E80092FBF3F3434403FB09F30A2293FBF2F3F5
:1080F80033449BB225F8023FB1F800904A880A340D
:10810800C9EB020AA4B21AB202FB0AF24FF47A735C
:10811800844292FBF3F34B442B80CED1BDE8F08729
:10812800FC15002010B544780078002202FB02F309
:10813800193B634303F6C413534340F6C411434346
:1081480093FBF1F3034921F812300132072AEDD1EC
:1081580010BD00BF161600200430114B33F9100073
:10816800B0F5617F10B506DB40F63303984202464E
:10817800A8BF1A4601E04FF461720C78192340F247
:10818800833013FB0404944207DA497813FB010394
:108198009342B4BF0020012010BD002010BD00BFD5
:1081A800AC2B002010B500F1500302788A4203D1AD
:1081B8008478C278944204D304309842F5D10020E0
:1081C80010BD012010BD0B4B1B6813F4805F0A4BD8
:1081D800B3F9063005D0C089421A934207DD084436
:1081E80000E0008A8342B4BF0020012070470120CC
:1081F800704700BFA82B0020AC2B00201FB5094BEF
:108208001B681B030AD58DF8040001230D2001A962
:108218008DED030A8DF8053000F016FF05B05DF806
:1082280004FB00BFA82B00201FB5084B1B681B03CD
:1082380009D58DF80400029100230D2001A98DF8BD
:10824800053000F001FF05B05DF804FBA82B002005
:1082580010B540001428A8BF14200023084A0221A2
:1082680099540B4499181424834201F8014CF5DB06
:10827800FF21D1540F20BDE8104006F0EFBC00BF2D
:10828800E828002010B5002006F06CFD054B0024FE
:108298001C7006F0A9FC044B83F82840DC621C869D
:1082A8005C6310BD002C0020FC150020084BDA6828
:1082B800D10709D4DA68D20608D4DB6813F0040FB2
:1082C80014BF032004207047012070470220704724
:1082D8000020024040F2E9330F4A1289920704D481
:1082E800013B9BB2002BF7D10BE00C4A40F2E9337B
:1082F800107009490989C9070AD4013B9BB2002BB0
:10830800F7D1074A138801339BB21380FF207047C7
:108318001078C0B2704700BF003800400C380040E9
:108328003416002030B5174B9B894FF47A733AB353
:1083380011B10D78013107E0FF2505E0013B9BB243
:108348004FF6FF74A3420FD00E4C2489A407F5D52D
:108358000D4C25700B4D2D89ED070BD4013B9BB2BD
:108368004FF6FF75AB42F5D1084A138801339BB22B
:10837800138005E0247808B104700130013AD6E78B
:10838800012030BD003800400C3800403416002071
:108398000C4B0D49DA684378D243C2F30222C2F18A
:1083A8000402934002781B010A44DBB282F80033CE
:1083B80003780122580903F01F0302FA03F341F876
:1083C8002030704700ED00E000E100E0036823F092
:1083D8001F0202F1804202F5823270B503F01F01DC
:1083E8001468012303FA01F124EA0101116002680B
:1083F8002A4C22F01F0502F01F02295903FA02F243
:1084080021EA02022A510279016802F1804221F030
:108418001F0402F5823201F01F01155903FA01F118
:108428002943115102681E4D22F01F0402F01F0259
:10843800615903FA02F221EA020262510268194CF8
:1084480022F01F0602F01F02315903FA02F221EA54
:108458000202417932511029026812D122F01F011B
:1084680002F01F024E5903FA02F232434A510268DF
:1084780022F01F0102F01F020859934003430B51D9
:1084880070BD01F1804122F01F0001F5823102F038
:108498001F020C58934023430B5070BD0404014045
:1084A800080401400C0401400EB40FB507490190BF
:1084B80006AB01A8064A039301F04CFB019B00227E
:1084C8001A7004B05DF804EB03B070478D9800088B
:1084D800976C010810B50446B0F9000005F0B7FB29
:1084E800B4F9020005F0B3FBB4F90400BDE810408C
:1084F80005F0ADBB10B50446006805F0A8FB606840
:1085080005F0A5FBA068BDE8104005F0A0BB2DE96B
:10851800F74F0120FFF7B6FD002480B3012C2ED8B9
:108528004FF04C09174E09FB04FA06EB0A0808EB52
:108538000907BD7815B10134E4B2EEE790F90030CF
:1085480090F804E01846104B03228DE8240001211E
:108558002A4653F82E30FFF76BFC834658B1301D7E
:10856800504429464A460AF056FD01231C44C8F8DF
:1085780004B0BB70E4B20120FFF76AFDCDE703B099
:10858800BDE8F08F341600206457010808B52A2288
:10859800114800210AF03FFD104B00221049515CA0
:1085A80083F8F01104200521013283F8F5018A428D
:1085B8004FF0000083F8F41183F8F70183F8F611FF
:1085C80003F10803EAD1074B0122A3F88E225222B5
:1085D80083F88A2208BD00BFBE180020D0160020EC
:1085E800287501083416002010B5FFF75FFE4FF418
:1085F8003024012806D11CB1FFF758FE013CF8E7EA
:10860800052010BD002C08BF052010BD70B506461A
:10861800441E14F8011F89B1094D28460AF031FD9E
:108628000028F6D005F1080398423FBF054B401BD0
:10863800C018A31B38BF80F82432EAE770BD00BF1A
:108648002D75010834160020031EB8BF2D2210B561
:10865800B8BF58420C46B8BF01F8012B0A2201F0F6
:1086680065FA00230370204610BD07B51B4B03F6BF
:108678008402C3F8802893F82C225AB1012A14D115
:10868800032183F88618072183F8882883F8871838
:108698000C2208E0022183F88618032183F8882831
:1086A80083F88718072283F884280D4B0D4A1A602F
:1086B8004020FFF7E7FC70B10122002390F9000089
:1086C80040218DE80C00084A4FF4E133FFF7B0FB76
:1086D800003018BF012003B05DF804FB34160020F9
:1086E8002000002019E60008ADE70008012000215D
:1086F80005F0A8BCF0B5184A92F88938D2F88C78F9
:108708001546042B11D807EBC3025E1C941CF6B265
:1087180009D013469288D10705D5104203D008E046
:108728000131052908D13346EBE785F8893800205F
:10873800F0BD93F802E00021074C0C2204F5096C07
:1087480002FB01F31CF803209645E9D1234484F881
:108758008968D3F89408F0BD3416002020F01F0172
:10876800012300F01F00024A83408B50704700BF6E
:108778001404014000230360436083608381036124
:1087880043618361C36103624362836270478A689D
:10879800036810B50C6A14430A6914434A69144300
:1087A8008A691443CA6914434A6A14438A6A23F4D7
:1087B800FF4323F070032243134303608B89436014
:1087C8000B6883604B68C36010BD02684FF6FE7388
:1087D800134003600023036043608360C360294B38
:1087E800984201D1284A27E0284B984201D1264ACD
:1087F8002AE0274B984201D1234A2DE0254B984285
:1088080001D1214A30E0244B984201D11E4A33E07D
:10881800224B984204D11C4A536843F470032EE05B
:108828001F4B984204D1184A536843F0706326E0FE
:108838001C4B984204D11C4A536843F00F031EE0B6
:108848001A4B984204D1184A536843F0F00316E0D3
:10885800174B984204D1144A536843F470630EE0EE
:10886800144B984204D1104A536843F4704306E00D
:10887800114B984204D10C4A536843F47023536057
:10888800704700BF08000240000002401C00024080
:108898003000024044000240580002406C00024090
:1088A8008000024008040240000402401C04024008
:1088B80030040240440402405804024001F003031B
:1088C80001F0FC0101F1804101F5803110B59B00F8
:1088D8008C680F229A4024EA02028A608A689840CB
:1088E80002438A6010BD0A888B88F0B54C880E89CF
:1088F800CD88C2B9026A22F0010202628269016A65
:1089080022F0F3021A4342EA061344F0010421F06C
:108918000A02144383610462836923F00C038361B0
:1089280083691D431FE0042A016A1ED14FF6EF72C6
:108938000A4002628269016A1B0222F4734243EA16
:1089480006332401134344F010044FF65F720A40C3
:10895800A4B2224383610262836923F44063836182
:10896800836943EA05258561F0BD082A1DD14FF6C4
:10897800FF620A400262C269076A4FF60C71114031
:108988004FF2FF523A4042EA042443EA06130B43EB
:1089980044F480749BB2A4B2C3610462C2694FF606
:1089A800F3731340C361C3691FE04EF6FF720A40B8
:1089B8000262C169026A40F6FF470F4045F6FF713F
:1089C80011401A0242EA063341EA04343B4344F4B4
:1089D80080549BB2A4B2C3610462C2694FF2FF33F0
:1089E8001340C3612D02C369ADB21D43C561F0BD1B
:1089F800036A23F001030362036A70B5446882695D
:108A08000D6822F4803222F0730215438A8923F01C
:108A1800020313438A881343134A90420FD002F586
:108A2800006290420BD002F54062904207D002F5F6
:108A38008062904203D002F5806290420DD1CA89CB
:108A4800CE8823F0080313430A8A24F4407414439D
:108A58004A8A23F00403334314438A6844608561D7
:108A68004263036270BD00BF002C01409B4A5368FB
:108A780003F00C03042B2DE9F04105D0082B06D098
:108A880097490160B3B916E0954B036012E053684B
:108A98005468C3F38343991CE30349BFD36A914BDA
:108AA8008F4C03F00F0344BF0133B4FBF3F34B4384
:108AB800036000E0002351688B4FC1F30311394470
:108AC8000D790168EDB221FA05F444605668C6F3E1
:108AD80002263E44367924FA06FEC0F808E05668B5
:108AE800C6F3C2263E443679F6B2F440C460D2F8E2
:108AF8002C80C8F3041808F00F0C07EB4C0C18F086
:108B0800100FBCF814C01FFA8CFC07D0BCF1000F82
:108B180004D0B3FBFCFCC0F810C000E00161D2F83F
:108B28002CC0CCF3442C0CF00F0807EB48071CF0C2
:108B3800100FBF8ABFB204D01FB1B3FBF7F747616C
:108B480000E04161176BFF065ABF654F876181617D
:108B5800176BBF065ABF624FC761C161176B7F06AB
:108B68005ABF5F4F07620162176BFF0506D599422E
:108B780004D1AE4202D14F00476200E04462176B55
:108B8800FF0406D5994204D1AE4202D14F00876254
:108B980000E08462176BBF0506D5994204D1AE4246
:108BA80002D14F00C76200E0C462176B7F0506D58B
:108BB800994204D1AE4202D14F00476400E04464B8
:108BC800176B3F0506D5994204D1AE4202D14F003A
:108BD800876400E08464176BBF0406D5994204D10A
:108BE800AE4202D14B00C36400E08464156B3B4B7A
:108BF800AD0701D1046315E01C6B04F00304012CDC
:108C080001D101630EE01C6B04F00304022C02D1B5
:108C18004FF4004305E01B6B03F00303032B01D162
:108C28002F4B0363146B2D4B14F4403F02D1C0F853
:108C380034E018E01C6B04F44034B4F5803F01D1F3
:108C4800416310E01C6B04F44034B4F5003F02D1DA
:108C58004FF4004306E01B6B03F44033B3F5403F89
:108C680001D11F4B4363146B1C4B14F4402F02D1EA
:108C7800C0F838E018E01C6B04F44024B4F5802FE9
:108C880001D1816310E01C6B04F44024B4F5002F7B
:108C980002D14FF4004306E01B6B03F44023B3F505
:108CA800402F01D10E4B8363146B0C4B14F4401FFF
:108CB80002D1C0F83CE021E01C6B04F44014B4F588
:108CC800801F01D1C16319E01C6B04F44014B4F592
:108CD800001F0BD14FF400430FE000BF001002400B
:108CE80000127A0000093D00200000201B6B03F4ED
:108CF8004013B3F5401F01D1134BC363126B134BE1
:108D080012F4400F03D1C0F840E0BDE8F0811A6BBF
:108D180002F44002B2F5800F02D10164BDE8F0818F
:108D28001A6B02F44002B2F5000F02D14FF400436F
:108D380006E01B6B03F44003B3F5400F01D1024B6F
:108D48000364BDE8F08100BF00127A000010024001
:108D58002F4B304A1B68126810B51A602E4A1168EA
:108D6800596051689268DA602C4A996011681961F3
:108D7800516892689A612A4A59611168D9615168A3
:108D880092685A62274A196211881985518859854B
:108D98009188D288DA85244A99851188198651885C
:108DA800598692889A86214A1188D98651881987C6
:108DB8001946928821F83A2F1D4A107800228242DB
:108DC80006DA1C4C34F8124021F8024F0132F6E75B
:108DD800194A1288A3F86420184A1288A3F8662052
:108DE800174A12689A66174A3B21126892FBF1F2F9
:108DF800B2F5967FC8BF4FF0FF32DA66124A128882
:108E0800A3F87020114A5289A3F85E2010BD00BF54
:108E1800082E0020B82F0020E4260020F02600208D
:108E2800FC26002094260020D20F0020CC0F002022
:108E38004C2C0020EC0F0020102B00207C0F002071
:108E48002C070020000000201C100020D80F002054
:108E5800A0F17D03012B70B504460D460A4E05D8D6
:108E680030687D2105F0D5FF84F020043068214664
:108E780005F0CFFF35B12B881C4404EB142404F013
:108E8800FF042C8070BD00BF840D002010B50A4C73
:108E98005E280146206805D15D2105F0BAFF2068EB
:108EA8003E2105E05D2903D105F0B3FF20683D218F
:108EB800BDE8104005F0ADBF041F00202DE9F843C0
:108EC8000E4B93E8800305460E460024B44213DA9D
:108ED8007B1933F9140008EB050333F9142009EB67
:108EE800050333F914301344022293FBF2F3C01A3A
:108EF80004F0ADFE0134E9E7BDE8F883082E002050
:108F080010B5104B93F8D837012B014612D10E4AF1
:108F18000E4C1078431CDBB213701B0644BF0023B1
:108F280013702154FDF768FB3F2809D9BDE81040AC
:108F3800FDF740BB064BBDE81040186805F069BF57
:108F480010BD00BFD01600202C2800202E2800209D
:108F5800EC2D00207FB5264C264E274D2749284A60
:108F6800284B20B128480088B0F5805F32D230887D
:108F78001F4E91F820101278ADF8040028788DF86B
:108F88000600351D8DF807108DF808201B788DF820
:108F9800093001A8294606220AF022F830B30198C0
:108FA800BDF808307060AB805320FFF7A9FFA08898
:108FB80004F03DFEA07904F03AFEE3790193237AA8
:108FC800029301A8637A039304F0A0FD0E4B0022DC
:108FD8001A800BE03088A08091F820102878127849
:108FE8001B78A071E17122726372DDE704B070BD75
:108FF800041F0020A80F002000280020DC2B0020E0
:10900800400E0020EE0E0020982F00200A4A1388F8
:1090180001331380094A136801331360084A13881F
:1090280001339BB2202B01BF00231380054A13880C
:1090380008BF013313807047982F00207C2F002031
:10904800802F0020822F002038B5294B1B78083B41
:10905800012B05460C464AD84520FFF751FF284604
:10906800FFF74EFF0E2D33D003D83DB10D2D07D09D
:1090780038BD142D20D0FF2D32D038BD20682BE00C
:10908800637820789BB180F08000FFF739FFA568EE
:10909800E8B2FFF735FFC5F30720FFF731FFC5F347
:1090A8000740FFF72DFF280EFFF72AFF04E0FFF720
:1090B80027FF606804F0CBFD2078FFF721FF606888
:1090C80004F0C5FD2489E0B2FFF71AFF200A0BE07F
:1090D800206804F0ACFD6068BDE8384004F0A7BD26
:1090E800044804F0B8FD0020BDE8384008E738BD62
:1090F800EA2D0020427501082DE9F04FB54BB64F17
:109108001A8889B01C46002A40F0A280B7F8D60712
:10911800B24E42F20103C11A48424841FFF71AFF12
:10912800FFF716FE34684920FFF7EAFEAC4B2546E8
:10913800186804F07CFD55F8040B04F078FD284607
:10914800FFF7D8F904F11000FFF7D4F904F11C096E
:109158004FF01008A34D01232A6803FA08F31342BD
:1091680003D0D9F8000004F072FD08F10108B8F145
:10917800130F09F10409EDD104F12800FFF7AAF94A
:10918800B7F84031B4F92E00C01A04F050FD2B682E
:10919800DA0408D5944BB4F864001B88181AC0F395
:1091A8000D0004F044FD2B689B0403D5B4F8660059
:1091B80004F03DFD2B68180502D5A06E04F047FDAC
:1091C8002B68590402D5E06E04F041FD2B681A049F
:1091D80003D5B4F8700004F02AFD04F13000A0466D
:1091E800FFF778F904F13600FFF774F9B7F8403162
:1091F80038F93C0FC01A04F01AFD01277B4B1B7885
:109208009F4208DA38F9020FB4F93C30C01A04F06A
:109218001EFD0137F2E72B689B0505D5B4F95E0002
:10922800A0F2DC5004F013FD326871487260B2603D
:10923800121A91106F4A4A43531C032293FBF2F20D
:1092480002EB42029A1A742303FB0203336084E19F
:10925800694B6A4A1B6811688B4206D008A900202E
:1092680041F8203D1360FFF7EFFE97F8D6172388E3
:1092780097F8D7070B44013BB3FBF0F200FB12331E
:109288008B4280F06A81554C0120FFF763FEFFF79F
:109298005FFD502026686568FFF732FEA2682368E4
:1092A80010681B68626803441068A3EB400004F070
:1092B800CEFC6A6873689B1A0093AA68B3689B1A05
:1092C8000193EA68F36868469B1A0293FFF712F95C
:1092D8002A6933699B1A00936A6973699B1A019317
:1092E800B369AA6968469B1A029304F00FFC06F159
:1092F8001C0B05F11C091027A0463A4901230A68EE
:10930800BB4013428A4606D0DBF80000D9F800308B
:10931800C01A04F09CFC0137132F0BF1040B09F160
:109328000409EAD106F1260005F12601002330F9E7
:10933800022F31F9024F121B4DF823200133042B61
:10934800F5D1032200275DF82230BF00FFB26BB1D0
:1093580003F108010F2902D847F0010706E080331E
:10936800FF2B94BF47F0020747F0030712F1FF32C3
:10937800E9D23846FFF7C4FD0024EB46A14607F0C2
:109388000303022B10D0032B17D0012B4BD1B9F1BB
:10939800000F42D0DBF8000000F00F002043FFF779
:1093A800AFFD4FF000093EE0B9F1000F0CD0DBF83B
:1093B8000000C0F3031020432DE0B9F1000F1FD1C6
:1093C8009BF80100FFF79CFD9BF80000FFF798FD54
:1093D80029E000BF802F0020D0160020082E002092
:1093E8007C2F0020742F0020702F00204C2C002090
:1093F800142E002035C2724F882F0020842F0020A1
:10940800DBF80000C0F303302043FFF779FDDBF8F9
:109418000000C0F30710FFF773FDDBF800402401DC
:10942800E4B24FF001090BF1040B04AB9B454FEA82
:109438009707A4D1B9F1010F02D12046FFF760FDCB
:10944800DAF8003013F480541FBFB6F86420B5F87A
:109458006410521A009218BF01249F040AD508AA62
:1094680002EB8401B5F86600B6F86620121A41F8D6
:10947800202C0134180508D508AA02EB8400A96E2F
:10948800B26E521A40F8202C0134590408D508AAA3
:1094980002EB8400E96EF26E521A40F8202C013477
:1094A8001A040BD508AB03EB8402B5F87010B6F8B4
:1094B80070305B1A42F8203C013400E0E4B1012C22
:1094C80003D1009804F0C3FB16E0631E00205DF88A
:1094D80023204000C0B20AB140F0010013F1FF336D
:1094E800F5D2FFF70DFD00275DF8270008B104F05D
:1094F800AEFB0137A742F7DB30200321FFF7DEFC84
:1095080036200321FFF7DAFC164B3C201978FFF7C9
:10951800D5FCDAF800309B0506D5B6F95E00B5F93A
:109528005E30C01A04F093FBD8F800200E48D8F833
:109538000430C8F80420121A91100C4AC8F80830F0
:109548004A43531C032293FBF2F202EB42029A1A9B
:10955800742303FB0203C8F8003004F0C5FA09B00D
:10956800BDE8F08F4C2C0020142E002035C2724F1D
:109578002DE9F74F0E9F4D4CC2EB030B0D9BFF1AC5
:109588006368002914BF4FF006094FF0040901333E
:109598008246164634D122684A4580F08280DFF838
:1095A8002881019158F8220009F079FD0B3004F068
:1095B8003BFA0199054608B1012073E022683C484E
:1095C800032A98BF514658F8222004F0D7FB394A9D
:1095D8001368181A6368106001336360364B9D7214
:1095E8000EE00D9A92B103FB07F20D99895C0122F6
:1095F8008A40324909680A4208D1636801336360C6
:1096080063680C9A294D9342EBDB32E003FB0BF5C0
:10961800236806EB050A2BB9705909F040FD00F1E3
:10962800050801E04FF00308404604F0FDF9002862
:10963800C2D1204A204B1068C8EB000010609A7A0B
:109648001AB12C20FFF75CFC01E001229A72236812
:1096580043B9705904F0FFFA9AF904104B1CCCD0A6
:10966800174803E09A4417489AF8041004F086FB58
:10967800C3E710D1012004F0D7F960B90D4A136887
:109688000A20013B1360FFF73BFC2B6801332B607A
:109698004FF0FF336B60206848452CBF0020012045
:1096A80000E0002003B0BDE8F08F00BF902F00203D
:1096B8004D7501088C2F0020041F0020742F0020F6
:1096C8005C7501084B7601088457010830B585B0F0
:1096D80004AC002524F8025D0091ADF8060021468F
:1096E8001020FFF7B5FB9DF806002146FFF7B0FBF9
:1096F8009DF807002146FFF7ABFB9DF800002146C7
:10970800FFF7A6FB9DF801002146FFF7A1FB9DF896
:1097180002002146FFF79CFB9DF803002146FFF756
:1097280097FB9DF80E00C043C0B22946FFF790FB97
:1097380005B030BD10B5054C206805F067FB18B1C1
:10974800206805F060FBF6E710BD00BF5C0D002047
:1097580030B50028104C114AB8BF40423C2590FB58
:10976800F2F304FB030068430D4D90FBF2F22D6801
:109778002D7B25B903EB830303EB830301E0C3EBE4
:10978800031302EB83030B8004FB02024FF47A738A
:1097980092FBF3F24A8030BD806967FF809698009B
:1097A800140D002010B50446C0B2FFF76FFBC4F3D8
:1097B8000720BDE81040FFF769BB024B5E2118681F
:1097C80005F027BB041F002038B5064C05465E216E
:1097D800206805F01EFB20682946BDE8384005F0E2
:1097E80018BB00BF041F0020F0B50124B0FBF4F53E
:1097F8008D4201D34C43F9E70026D4B1B0FBF4F510
:1098080004FB1500B4FBF1F41EB9002D01DC002C9B
:10981800F3D1092D03F1010EEFB204DD002A14BFC4
:109828003725572500E030253D441D700136734625
:10983800E3E71C70F0BDF0B50124B0FBF4F58D42F0
:1098480001D34C43F9E70026D4B1B0FBF4F504FB8F
:109858001500B4FBF1F41EB9002D01DC002CF3D186
:10986800092D03F1010EEFB204DD002A14BF3725DC
:10987800572500E030253D441D7001367346E3E767
:109888001C70F0BD03685A1C0260197070472DE9FE
:10989800F843089E002B07468846144614BF4FF02D
:1098A80030094FF02009334613F8012B0AB9254631
:1098B80003E0002CFBDD013CF6E7002D04DD384613
:1098C8004946C047013DF8E724EAE4743546A01B41
:1098D800284415F8011B11B13846C047F7E7BDE821
:1098E800F883024B186805F094BA00BF880F00206F
:1098F80090ED017A07EE901AB5EE407AF1EE10FA83
:1099080001BFF8EEE77A9FED0E7A67EE877AB7EE39
:10991800007A04BFC7EE277AC0ED017A90ED017A8C
:10992800D0ED007A30EE877A30EE670AC0EE870A0B
:10993800E0EE807AB0EE670AC0ED007A704700BFAB
:10994800DB0FC94010B50278202A034600F1010058
:10995800F9D0092AF7D02D2A03D10346BFEE000A11
:1099680004E02B2A08BF0346B7EE000ADFED387A79
:109978001A46134612F8010BA0F13001CCB2092C9B
:109988000AD807EE101AB8EEC77AF2EE046AA7EE04
:10999800A67AF0EE477AECE72E2816D1F2EE046AA2
:1099A8001146B0EE666A0B4611F8012B303AD0B278
:1099B80009280AD807EE102AB8EEC77A87EE267A61
:1099C80066EE866A77EE877AEDE71A7802F0DF02AC
:1099D800452A35D15A782D2A02D10233012004E0D4
:1099E8002B2A14BF013302330020013B002213F855
:1099F800011F3039CCB2092C03D80A2404FB021207
:109A0800F5E7B2F59A7F28BF4FF49A721346B7EE7E
:109A1800007A072B05D9DFED0F6A083B27EE267A77
:109A2800F7E702F007032BB1F2EE046A27EE267A75
:109A3800013BF8E7F0EE476A20B1C7EE877A03E00A
:109A4800F7EE006A67EEA67A20EE270A10BD00BF7F
:109A58000000000020BCBE4C30B52DED028B87B055
:109A6800B0EE408A0C220021054603A809F0D3FA7B
:109A7800B5EEC08ADFED2A7AF1EE10FACCBF38EEE7
:109A8800278A38EE678ADFED277A28EE278A694623
:109A9800FDEEC87A17EE904A84EAE470A0EBE47011
:109AA800FEF7D2FD002CACBF20232D2368468DF88D
:109AB8000C3009F0F4FA012807D130238DF80D3065
:109AC8008DF80E308DF80F300CE0022805D13023C8
:109AD8008DF80D308DF80E3004E0032804BF3023D4
:109AE8008DF80D30694603A809F0BCFA03A809F0FF
:109AF800D6FA0338C4B2224603A9284609F0FCFA6C
:109B080000232B552846084909F0ACFA03AB284630
:109B1800191909F0A7FA284607B0BDEC028B30BD29
:109B28006F12033A00007A448075010870B5064642
:109B380015460846B6FBF2F414B12046FFF7F6FFC7
:109B480005FB1464024B1B5D00F8013B70BD00BFB0
:109B5800827501082DE9F04F814689B08A4616467C
:109B68001C4600253178002900F0DD80252902D027
:109B78000136484675E07278302A08BFB278A2F1FB
:109B8800300319BFB71C4FF0000BF71C4FF0010B47
:109B9800092B4FF0000819D8A2F13003D9B20929CE
:109BA80005D80A2202FB083817F8012BF4E7A2F1BE
:109BB8006103052B02D8A2F1570305E0A2F1410386
:109BC800052B03D8A2F137030A2BEADD6C2A31D121
:109BD8003A78642A07F1010600F083800BD8252A19
:109BE8003DD003D8002A00F09E80BBE7582A0CD04D
:109BF800632A19D0B6E7732A22D002D86E2A37D042
:109C0800B0E7752A5CD0782AACD1271D2068A2F16C
:109C1800580462424FF01001624155E02CD9582A8D
:109C280032D0632A2AD13E4648462178271DD0479C
:109C380001350FE0642A64D00ED9732A14D13E4648
:109C4800236800934846514642460023FFF71FFE0B
:109C5800271D05443C4685E7252ADFD13E46484670
:109C68002521D04701357DE70AD86E2A06D13E4620
:109C7800236804341D6075E7002A54D03E4671E716
:109C8800752A26D0782AF9D1A2F1580304F1040CD8
:109C98005A422068CDF80CC04FF010015A4105AB6C
:109CA800FFF7A2FDDDF80CC03E46644605AB009305
:109CB8004846514642465B46FFF7E9FD054451E7F1
:109CC8002068271D0A21002205ABFFF7B4FD3C469A
:109CD800ECE704F1040CCDF80CC020680A2100223E
:109CE800DDE72068002804F1040708DA2D238DF841
:109CF800143040420DF115030A210022E5E705ABB7
:109D0800FAE72068002804F1040C0ADA2D238DF8FC
:109D1800143040420DF11503CDF80CC00A21002281
:109D2800BEE705ABF8E7284609B0BDE8F08F0FB4E9
:109D380013B50B4904AB08680A4953F8042B0968A2
:109D48000193FFF707FF0446074B186805F058F81A
:109D58000028F9D0204602B0BDE8104004B0704792
:109D6800DC000020D8000020880F002080EAE07383
:109D7800A3EBE0738B4206DB002801DD401A704735
:109D880002D00844704700207047B0EEE06AF0EE59
:109D9800C05AB4EEE56AF1EE10FAD4BFF0EE656A87
:109DA800F0EE466AF5EE406AF1EE10FA0BD0B4EE2A
:109DB800E56AF1EE10FA54BFF0EE657AF0EE467AF5
:109DC800C7EEA66A01E0DFED206ADFED207A9FED9D
:109DD800207A9FED205AA6EEA77ADFED1F7AE7EEEC
:109DE800267A9FED1E7AA7EEA67ADFED1D7AE7EEBA
:109DF800267AF4EEC65AB1EE677ADFED1A7AA6EE45
:109E0800A75AF7EE007AE5EE267AF1EE10FAC7EED9
:109E1800277AC8BF9FED147AF5EEC00AC8BF77EE5F
:109E2800677AF1EE10FA48BF9FED107AB5EEC00AD6
:109E380048BF77EE677AF1EE10FA48BFF1EE677A1D
:109E4800B0EE670A704700BF0000000039094E3DB8
:109E5800E3B59EBE69A2163E88FA16BE45FE7FBFD0
:109E6800A7DFA8B499FB243FDB0FC93FDB0F4940AC
:109E7800FDEEC07A17EE903A2033402B43D8DFED41
:109E8800237AB4EEE70AF1EE10FA04DDDFED207A6A
:109E980030EE670AF3E7DFED1F7AB4EEE70AF1EE7A
:109EA80010FA04D5DFED1A7A30EE270AF3E7DFED72
:109EB8001A7AB4EEE70AF1EE10FA04DD30EE670A1A
:109EC80037EEC00A0AE09FED157AB4EEC70AF1EE44
:109ED80010FA44BF30EE270A37EE400A60EE007AE7
:109EE800DFED0F6A9FED0F7AA7EEA67ADFED0E6A17
:109EF800E7EE876A9FED0D7AA7EEA67A20EE276A2D
:109F0800A6EE070A70479FED060A7047DB0F494027
:109F1800DB0FC940DB0F49C0DB0FC93FDB0FC9BFEF
:109F28000000000092E741B99730083C15A82ABE06
:109F3800DFED027A30EE270A9AE700BFDB0FC93F50
:109F4800064B1A8822EA0000904210B518801C4679
:109F580002D00120FEF77CF9208810BDA80F002050
:109F6800064B1A881043904210B518801C4602D040
:109F78000120FEF76DF9208810BD00BFA80F002052
:109F8800024A936823EA000090607047D0160020C8
:109F9800024A936818439060704700BFD0160020AB
:109FA80008B5104B1A780023D9B2914207D20E494E
:109FB80051F823100968002008600133F4E73220C3
:109FC80004F0A9FE094B1B685A0309D5084B9B6886
:109FD8005B0305D440F2DC50BDE8084004F09BBEAA
:109FE80008BD00BF4C2C00201C2C0020A82B0020F2
:109FF800D01600202DE9F34104F0E0FD454A6F2317
:10A00800137040F2E4735380BE231371EF2382F878
:10A01800E037002382F8E13719461646F25C01332F
:10A02800514040F2E4729342F8D13A4B83F8E11779
:10A03800394B1A69120604D5384A5A6002F1883237
:10A048005A6004270020013F17F0FF0750D0324B19
:10A058003422DA60002444B1002356F804800193C6
:10A06800FEF7C2FA0428EED117E0FEF7BDFA04287D
:10A07800E9D1294D2B6943F002032B61284B6B6111
:10A088002B6943F040032B61FEF7AEFA2B690428D5
:10A0980023F002032B61DFD0D5E71F4D2B6943F076
:10A0A80001032B6104F1006303F5FC331FFA88F206
:10A0B8001A80FEF799FA042810D11A4B2344019309
:10A0C800019B4FEA1848A3F80080FEF78DFA2B6928
:10A0D800042823F001032B6105D0B4E72B6923F092
:10A0E80001032B61AFE7043440F2E4739C42B2D120
:10A0F800094A1369042843F08003136102D103F06D
:10A1080094F910B9052004F033FE04F043FD02B0C1
:10A11800BDE8F081D01600200020024023016745E9
:10A1280000F8010802F8010810B50E4C2068FDF788
:10A13800F9FF2068047A002202FB02F3193B63430B
:10A1480003F6C4135343192193FBF1F3064921F88D
:10A1580012300132072AEFD10449BDE81040FDF75B
:10A1680097BF00BF28100020580F002010180020AB
:10A178002DE9F04103F059F910B9042004F0F8FD75
:10A18800AA4CAB4D04F01AFDAA4940F2E4722046ED
:10A1980008F036FF94F8B037022B84BF002384F808
:10A1A800B03794F8B0274FF4CC7101FB02F303F5F4
:10A1B8003A7023442044286093F84803022801FB9E
:10A1C800024284BF002083F8480392F848339A4A31
:10A1D80013700C2202FB0343984A03F2B273136014
:10A1E800A26846F2090313401BB94FF40050FFF769
:10A1F800CFFEA368D80703D54FF40050FFF7C0FE81
:10A20800A368590409D50820FFF7BAFE4FF4005097
:10A21800FFF7B6FE0120FFF7B3FEA3681A0706D5BD
:10A228004FF40050FFF7ACFE0120FFF7A9FEA3682A
:10A238009B0402D54020FFF7A3FE012284F81922CF
:10A2480094F8DE21794B2AB193F8E22112B1002269
:10A2580083F8E2217A4B7B4E1E604FF0000C674674
:10A2680004EB0C03B3F8F2E14FEA5E0101F0773139
:10A278004FEA9E0303F03333C1EB0E00C11A4FEAD5
:10A28800DE0303F01133CB1A03EB23131EF001088E
:10A2980003F00F324FF0FF0392FBF3F3C3EB0323FA
:10A2A80018BF0137A2EB030318BFFFB2012B0ADD69
:10A2B800022B40F0B880B8F1000F00F0B4801EF017
:10A2C800BC0F00F0B0800CF1080CBCF1280FC7D10E
:10A2D800013F012F00F2A780FFF726FF302200215F
:10A2E80059485A4F08F097FE594BD5F800801F601F
:10A2F800584B002108F18500C3F80080FDF752FF94
:10A30800554B80F001001870544B07F128021A6071
:10A31800534B07F1D8021A6098F8000003F05EF872
:10A32800504B94F8D601DFED506A07F196021A6097
:10A3380064214E4BC82211FB00225A6000229A6009
:10A34800DA601A615A619A61DA6183F8202083F829
:10A358002120474B07F12E021A602B68454A93EDDE
:10A368001B7A03F225111160434A03F2951111601B
:10A37800424A07F108011160414A1760414A07F152
:10A38800A201116067EE266A3F4A07F1AC01B6EEFA
:10A39800007A116087EE267A3C490E60B4F86411A1
:10A3A800101D07EE901AB4F86611F8EE677AC2ED40
:10A3B800027A07EE901A93F86810117193F88410D6
:10A3C800517194F8E1111174F8EE677AB3F822111B
:10A3D800C2ED037A07EE901A2D49F8EEE77A086085
:10A3E800536182ED077A9FED2B7AC7EE277A03F146
:10A3F800700191612849294A0B6029499FED297A02
:10A4080067EE877AC2ED007A03F174020A60264982
:10A4180003F21D130B60254B1F60254BBDE8F0416F
:10A428001A6004F0B7BBFEF7B1F855E7D016002064
:10A43800E80F002000F80108B028002028100020AC
:10A44800A42B002058180020180F002010180020F6
:10A458004C0F0020500F00200A0000202027002069
:10A46800BC050020A82F0020DB0F4940DC2B002072
:10A4780088270020F8150020C4080020682D002037
:10A488006C2D0020D8070020101F00209C080020F9
:10A49800042800200000614450070020D407002051
:10A4A800440700204C3D0F44C4070020CC0700207F
:10A4B8003C06002008B5FFF79DFDFFF759FE012077
:10A4C800BDE80840FDF7C4BE2DE9F74FA44C04F0E1
:10A4D800FBFB26686568A768861BF643451BC71BF8
:10A4E800ED43FF43F60F8046ED0FFF0F2EB93FB93E
:10A4F800002D00F07E82B9462CE04FF0000929E0DB
:10A50800B14627E003EB8A0BBBF8023019050ED4DD
:10A5180013F4805F1DBF934A9BF801101268924A9A
:10A52800924B14BF52F82120126843F82A20BBF836
:10A538000230DA0516D49B050AD58D4B1B7813F02B
:10A54800040F0CBF8B4A8C4A884B126843F82A20A8
:10A5580009F10109207B89495FFA89FA82450B686C
:10A56800D0D320E050465946854AFBF757FD854B26
:10A578001B88580603D550465946834A10E01907E8
:10A5880003D550465946814A0AE09A0703D55046F2
:10A5980059467F4A04E0DB07DAD57E4A50465946D9
:10A5A800FBF73CFDD4E7DFF804E20093BEF9063080
:10A5B8007822A3F57A7353434FF47A7293FBF2F33C
:10A5C80003F22B1301930022F3465FFA82FE8645BD
:10A5D80017D2009B03EB820EBEF802E01EF4806FD8
:10A5E8000DD0DFF88891019B39F822E040F2671A14
:10A5F8009E449EFBFAFC0AFB1CEE29F822E001327D
:10A60800E3E74DB308F5C333A0336360637B544A73
:10A6180013BB9373604B1B6813F0020F0AD0DFF86B
:10A6280090E19EF800E0BEF1000F03D04FF0010E5C
:10A6380082F80EE0DA0506D5584BDB781BB1A37B10
:10A6480043F00203A3734A4B1B7813F0050F02BFB4
:10A65800A37B43F00403A37394F80EE0BEF1000F4C
:10A6680003D13F4B5B7B002B4FD094F80DC01CF0FF
:10A67800010FACF10C031DD1BCF1030F07D8DFF8B3
:10A68800E8903C4A1EF0040F08BF4A4600E0364AEC
:10A69800ACF1040CBCF1070F05D8DFF818C11EF0A7
:10A6A800010F18BF6246DBB2032B0ED81EF0020F53
:10A6B8003B4B06E0DBB2032B06D82F4B2A4A1EF091
:10A6C800020F18BF1A4600E0274A4FF0000C5FFA45
:10A6D8008CF383420DD20B6803EB8C035B881B065B
:10A6E80042BF224BD2F8009043F82C900CF1010C99
:10A6F800EDE785B1BEF1000F08D0637B184A01333E
:10A70800DBB2142B06D1002304E025B1637B002BB8
:10A71800F3D100E05373002E50D0224AB2F9025010
:10A72800B2F90020002DB8BF6D42002A4FF0320365
:10A73800B8BF524295FBF3F592FBF3F2EDB2D3B2F8
:10A74800AB4238BF2B46184A13B192FBF3F300E033
:10A75800134643442360E37B014A6BBB01232CE08F
:10A76800301F0020F0150020A0670108940D00207C
:10A77800D22F0020B0580108A0580108F415002075
:10A788009C570108A80F0020A2570108A8570108E4
:10A79800AE570108B4570108A82B0020DC2B002075
:10A7A800B858010894260020400D0300AC2B002067
:10A7B800D8280020C05801080023D3738E4D8F4B32
:10A7C8002D78E27BADB9002F00F00E818C4B267BF3
:10A7D8001A788C4B8C4D93F800C08C4BD3F800E062
:10A7E8000B6802F004020021D2B203EB86060F4682
:10A7F800B5E01AB9864A1A61002508E0854AFAE7E1
:10A808000A68AB00D6187688760604D40135EBB210
:10A818008342F5D3D7E7804EB6F90060192E25DDBF
:10A8280012F803E094F814C026690EF00F09E14508
:10A838000CDCDFF8C8C19CF815C0BCEB1E1FDEBFDE
:10A84800DFF8D8E1D6F800C043F80EC012F803E0EC
:10A8580094F816C00EF00F09E14533DBDFF89CC110
:10A868009CF815C0BCEB1E1F2CDC26E0193629DA33
:10A8780012F803E094F814C026690EF00F09E145B8
:10A888000CDCDFF878C19CF817C0BCEB1E1FA2BF18
:10A89800DFF888E1D6F800C043F80EC012F803E0EC
:10A8A80094F816C00EF00F09E1450BDBDFF84CC138
:10A8B8009CF817C0BCEB1E1F04DBD6F800E0574E0F
:10A8C80043F806E0544EB6F90260192E1BDD12F863
:10A8D80003C094F814E026690CF00F09F1450CDC6C
:10A8E800DFF8189199F81590B9EB1C1FDEBFDFF857
:10A8F8002CC1D6F8009043F80C90D25C02F00F0CF3
:10A90800F4451EDD82E7193680DA12F803C094F8A0
:10A9180016E026690CF00F09F1450CDBDFF8DC9036
:10A9280099F81590B9EB1C1FDEBFDFF8F0C0D6F818
:10A93800009043F80C90D25C02F00F0CF445FFF63F
:10A9480065AF94F817E0BEEB121FA2BF334A366812
:10A958009E505BE75888000504D404330435B3429D
:10A96800F8D122E04AB101EB0C0A06209AFBF0F973
:10A9780000FB19A001280DDC01E057B9012793F865
:10A9880001900EEB89003EF829A090F80290C0785B
:10A9980003E01746002081468246013125F802ACC3
:10A9A80085F800906870C9B2D7E7164A1378013B5A
:10A9B80013F0FF0308BF06231370114B1B785B07C6
:10A9C80041BFBBF90630A3F57A7303EBC3034FF419
:10A9D8007A7243BF93FBF2F30133DBB20123104ACF
:10A9E80092FBF3F34344A36003B0BDE8F04FFAF7DA
:10A9F800DBBE03B0BDE8F08F400E0020301F002002
:10AA0800D22F002054000020960D0020F0150020C1
:10AA1800BC580108A067010894260020940D002066
:10AA2800400D03002DE9F04F2DED0A8B87B08346CA
:10AA3800039390F85030029101925BB1322BA8BF7A
:10AA4800322307EE903AB8EEE7BADFEDD67A87EE12
:10AA58008BBA01E09FEDD4BAD44BDFEDD5BA1B8891
:10AA6800D44CDFF86493002B08BF012307EE903A1B
:10AA7800B8EEE79A238869EE2BBA13F0020F3BEE83
:10AA88002BBA8BEE8BBA26D0B9F90030B9F902206F
:10AA980083EAE37182EAE270A1EBE371A0EBE27072
:10AAA80088420546B8BF0D46B5F5E17F16DA8842FB
:10AAB800DFEDC1AA05DD002AD8BF524207EE902A71
:10AAC80004E0002BD8BF5B4207EE903AF8EEE77A35
:10AAD800C7EEAAAA04E0DFEDB9AA01E0F7EE00AAE2
:10AAE800DFEDB69AB64A59464FF0000AB0EE69AAA9
:10AAF800B448B54D30F81A00B4F800E003B207EED8
:10AB0800903AF8EEE77AB5EE047A67EE877A35F987
:10AB18001A309FEDAE7AFDEEE77A06EE903AF8EE3F
:10AB2800E77A1EF0030F5FFA8AF64FEA4A0767EEE4
:10AB3800877AF8EEE66A6FD036EEA67A019BBDEE0C
:10AB4800C77AC3F1000817EE105A454503DBAB423C
:10AB5800A8BF2B4698469E4D039B7D5F9FED9D5A4F
:10AB6800C5EB080833F91A509BF81C30454407EE2A
:10AB7800105A0AEE103A9BF80830B8EEC76A07EE8A
:10AB8800103AB8EE477AB8EE4AAA26EE077AF1EEFE
:10AB9800045A27EE057A6AEE255ABDEEC77A17EEF3
:10ABA800108AB1EE657ABDEEC7AA1AEE103A98453A
:10ABB80008DBBDEEE5AA1AEE103A4345A8BF4346A6
:10ABC8000AEE103A844D05EB8A0595ED007AA6EE5B
:10ABD8002B7ABBEE0E6AB4EEC67AF1EE10FAB8EE36
:10ABE800CAAA09D4B3EE0E6AB4EE467AF1EE10FAA8
:10ABF800C8BFB0EE467A01E0B0EE467A85ED007A3D
:10AC08009BF8123009EE903AF8EE699A27EE297A05
:10AC1800DFED729A67EE299A1EF0010F50D100B24B
:10AC28000028B8BF4042B0F5206F02DD0020106058
:10AC380025E09FED6B6A4B7826EE867A06EE103A91
:10AC4800B8EE466A87EE066A92ED007A36EE676AD3
:10AC5800A6EE2B7A9FED636AB4EEC67AF1EE10FA8F
:10AC680009D49FED616AB4EE467AF1EE10FAC8BFD6
:10AC7800B0EE467A01E0B0EE467A82ED007ACB7A01
:10AC880092ED007A08EE103AB8EE488A1EF0020FEC
:10AC980028EE077A9FED558A27EE088A14D076EEBB
:10ACA800CA6AB0EE4A7AAAEEA67A38EE698AF0EE57
:10ACB800476AB0EE697AAAEE887AB0EE478A03E06E
:10ACC800B0EE698AF0EE4A6A49489FED4A6A1AF876
:10ACD8000030059207EE103AB8EEC77A4FEA8A08B4
:10ACE80027EE677A051D4544E7EE066A049195ED5F
:10ACF800007AC5ED007A37EEC77A00F10C0587EEC9
:10AD08002B7A454414301AF80030D5ED007A37EE26
:10AD1800677A08EE903AEBEE077AF8EEE88AC5ED26
:10AD2800007A67EEA87ADFED348A344D67EEA88A98
:10AD380036EE880AB0EE66CA30EE680A08F07AFB8A
:10AD4800E85320880499059A10F4006F08D02C481D
:10AD58000078400704D53046FBF72AFA059A04998B
:10AD68002848294FFDEECC6AFDEEC87AF1EE688AD4
:10AD780016EE903A17EE906AFDEEE88A48F8003031
:10AD880048F8076018EE903A204E049648F80630C6
:10AD9800043201318046BAF1000F3BD14FF0010A6D
:10ADA800A6E600BF83F9223EAF4C593C980F00201D
:10ADB800BD378635A80F00200000E14300000000E1
:10ADC800481F0020D20F002094260020CDCC4C40F4
:10ADD800041000206F12033C541F00200AD7A33D23
:10ADE8000000A043000040C3000040430AD7233CB2
:10ADF8005C1F0020A69B443BF7CC9238DC26002041
:10AE0800D22F0020E4260020F0260020FC26002077
:10AE180000803B45BDEEC99A5FED037A9BF853600D
:10AE28009049DFF864A219EE103A23F0030309EE03
:10AE3800103A029BB8EEC99A9B7989EE279AB5EE2B
:10AE4800000A002E6DD0B9F904209BF80300002AEF
:10AE5800B8BF52425A43844B92FBF3F364336422E3
:10AE6800434393FBF2F308EE903AB1F9043007EE4E
:10AE7800903AF8EEE77AF8EEE88A27EE800A08F0CA
:10AE8800D9FA07EE900AF8EEE77AB9F9043067EED6
:10AE9800A88ADFED767AC8EEA78A80EAE072A2EB8C
:10AEA800E072B2F5207F07EE903AF8EEE77A77EE97
:10AEB800E88A05DC83EAE372A2EBE372642A03DD25
:10AEC8000023CAF80830A2E003EB83031A019BF8B9
:10AED800033092FBF3F31B1A07EE903AF8EEE77A89
:10AEE800DAF8083067EE897AFDEEE77A17EE902AED
:10AEF8001A441346B2F57A5F5D4AA8BF4FF47A53F5
:10AF08009342B8BF1346CAF808307D2293FBF2F388
:10AF18009BF80D2053439B1107EE903AB8EEE78A51
:10AF280075E0544A5B00B2F90490283303FB09F931
:10AF3800B1F9043007EE903AF8EEE77A4FEA69196A
:10AF480027EE800A08F076FAB9F1000FC0EB090085
:10AF580007EE900AB8BFC9F10009B9F1320FB8EE8F
:10AF6800E77A02DDCAF808601BE09BF80D3007EEAF
:10AF7800903AF8EE677ADAF8083067EE277A67EEE3
:10AF8800897AFDEEE77A17EE902A13443A4A9342FB
:10AF9800A8BF1346394A9342ACBFCAF80830CAF86A
:10AFA8000820DAF808305B13B3F5807FA8BF4FF4A8
:10AFB80080736FF0FF029342B8BF134607EE903AD2
:10AFC800B8EEE78AFDEEC77A9BF8032017EE903AB1
:10AFD80053439B1107EE903A294B1B78032BF8EE4D
:10AFE800E78A14D9BBF84E20B2F5FA7F0FD2FDEEEE
:10AFF800E87A534217EE901A994204DB914217EE11
:10B00800903AA8BF134607EE903AF8EEE78A78EE32
:10B01800887AFDEEE77ACDED017ABDF80430AB8091
:10B028001BB200EE103AB8EEC00A08F003FA238803
:10B03800A8801A0506D5134B1B785B0702D502209A
:10B04800FBF7B6F8FDEEE88ABDEEC88A049AC8EDAB
:10B05800028A002387ED028A936007B0BDEC0A8B51
:10B06800BDE8F08FD20F00200CFEFFFF0000A042C9
:10B0780080C1FFFF94260020FEFFFF0F020000F0B2
:10B088004C2C0020D22F0020AC2600202DE9F04FB8
:10B0980087B000260593BA4B0491B3F90270B3F94F
:10B0A80000300292002FB8BF7F42002BB8BF5B422E
:10B0B8009F42B8BF1F46B7F5FA7F8046A8BF4FF436
:10B0C800FA770090B3460196B2463446AD4B1988DC
:10B0D80011F003023DD0AA4B33F91400029B400043
:10B0E8005B4298424FEA440503DB029B8342A8BFB8
:10B0F8000346A5482D5E05985B1B30F914501D4486
:10B1080098F8083064206B4393FBF0F398F81C0020
:10B118006FF0040A0AFB00FA534504DB00EB800ACF
:10B128009A45A8BF9A46994850F824302B4442F2D1
:10B138001075AB42A8BF2B46954DAB42B8BF2B4606
:10B1480040F8243098F8120043431B13012A019356
:10B1580038D08B4B8F4833F914B0009B50F824E05B
:10B1680093F801C08C4B33F9145085EAE573A3EBCF
:10B17800E573B3F5206F4FEA840616DC0BEB8B03FF
:10B188001A0192FBFCF3042295FBF2F55D1BAE4419
:10B19800BEF57A5FA8BF4FF47A5E804B9E45ACBF80
:10B1A80040F824E040F8243002E0002340F824303E
:10B1B80083597D2693FBF6F6009BDB7A7343402682
:10B1C80093FBF6F6880711D50198C7F5FA7307FBC4
:10B1D8000BF907FB06F54FF4FA7103FB0A9903FB19
:10B1E800005599FBF1F295FBF1F505E0C9074DBF54
:10B1F800019D35465A465246630069490393664B9A
:10B20800605C33F814E020310FFA8EF34FF0040C31
:10B2180093FBFCF909FB00F06FF04F0990FBF9F97B
:10B22800914431F9142021F814E098F850109B1A31
:10B2380093FBFCF379B107EE903A5A485A4BB8EEB3
:10B24800E70AD3ED000A00EBC400FEF751FBFDEE60
:10B25800C07A17EE903A554A554912F804C0039837
:10B2680003EB430309EB05020CFB03F34FF0200C3F
:10B2780093FBFCF3D21A4252424A1288120508D5AF
:10B288004C4A1278500704D520460393FAF790FFEA
:10B29800039B494A49494A4841F824905B4242F88D
:10B2A8002430009B40F82450013300930D4681461A
:10B2B8000CB901240AE7324B3648B3F90410049B51
:10B2C80086689B790F335B004B435B113249002B37
:10B2D8004FF00404B1F9041091FBF4F1A3EB010160
:10B2E800B8BF5B42322B98F80D400BDC354B04FBA2
:10B2F8000164A342A8BF2346334CA342ACBF83607A
:10B30800846001E000238360304B98F803401B7889
:10B318004C43032B4FEAA4140CD9B8F84E30B3F5BC
:10B32800FA7F07D259428C4203DB9C42A8BF1C46D5
:10B3380000E00C46866846F34F36B6F5807F6FF01E
:10B34800FF03A8BF4FF480769E42B8BF1E46184B35
:10B35800A11999800B4B1B88190508D5154B1B782B
:10B368005B0704D502200092FAF722FF009AAC602E
:10B378000023C9F80860936007B0BDE8F08F00BFEC
:10B3880094260020A80F002004100020741F00201D
:10B39800F0D8FFFFAC260020D20F002080C1FFFFAD
:10B3A8005C1F0020C4260020A8260020701F002053
:10B3B800DC260020D22F0020FC260020E4260020D6
:10B3C800F0260020FEFFFF0F020000F04C2C0020AA
:10B3D8002DE9F04F87B080460493A94B03911C8850
:10B3E800029204F00204A4B294B1A64BB3F902404D
:10B3F800B3F90030002CB8BF6442002BB8BF5B42E1
:10B408009C42B8BF1C46B4F5007FA8BF4FF4007437
:10B41800C24600259B4B9C4E33F915E09B4B33F8F5
:10B4280015300193BDF9040056F8253080EAE0771D
:10B43800A7EBE0770421B7F5206F90FBF1F189B213
:10B448004FEA450B4FEA4E0C0AB24FEA85090FDC6A
:10B45800C2EB0C021344B3F57A5FA8BF4FF47A53DA
:10B468008B4A9342ACBF46F8253046F8252002E0C7
:10B47800002346F8253056F809709AF80B30804AB0
:10B48800FF115F4312889AF80130960703FB0CF30B
:10B498004FEAA7174FEAA31340D0029A4FEA4E0E7D
:10B4A8005242964503DB029A7245A8BF7246794E0E
:10B4B800DFF814E23BF90660961B049A32F915206E
:10B4C800164459F80E2042F2107C32446245A8BF57
:10B4D8006246DFF8F8C16245B8BF624649F80E20F7
:10B4E80098F808E00EFB06F698F81CE00EEB8E0EB6
:10B4F800F611CEF1000C664503DB7645A8BF76460B
:10B50800B44698F8126072431213BF1ACCEB0303C7
:10B518006743634302EB67270CEB63235E4A565D80
:10B52800243211FB06F6A3EBA6163BF9023098F875
:10B538005010C01A042390FBF3F0BDF804302BF828
:10B54800023079B107EE900A544B5548D3ED000A02
:10B55800B8EEE70A00EBC500FEF7CAF9FDEEC07ABF
:10B5680017EE900A4F4B504A5B5D00EB4000584382
:10B578004311F119C91A2BF802104149088810F42F
:10B58800006F8B460AD049490978490706D52846ED
:10B5980005920193FAF70CFE059A019B4448454928
:10B5A80049F80060444E49F801705B4249F806309A
:10B5B8000AF1010A074689460DB901252AE7314BE8
:10B5C80098F80D00B3F90410039B9B790F335B00C7
:10B5D8004B435B112D49002BB1F904104FF00405C2
:10B5E80091FBF5F52849A3EB0505B8BF5B42322B63
:10B5F8008C680BDC314B00FB05408342A8BF034637
:10B608002F488342ACBF8B60886001E000238B60C9
:10B6180098F803305D432B4B1B78032B4FEAA51595
:10B628000CD9B8F84E30B3F5FA7F07D258428542A4
:10B6380003DB9D42A8BF1D4600E005468C6844F325
:10B648004F34B4F5807F6FF0FF03A8BF4FF48074C8
:10B658009C42B8BF1C462B199380BBF800301A05D2
:10B6680006D5124B1B785B0702D50220FAF7A0FD1E
:10B678000023BD60C9F80840B36007B0BDE8F08F8B
:10B68800A80F002094260020AC260020D20F00200E
:10B6980080C1FFFF041000205C1F0020A8260020A6
:10B6A800C4260020701F0020DC260020D22F002096
:10B6B800E4260020F0260020FC260020FEFFFF0FD5
:10B6C800020000F04C2C0020741F0020F0D8FFFF6F
:10B6D8002DE9F04F2DED028B85B000260293A44B87
:10B6E8000192B3F90270B3F900300090002FB8BF8F
:10B6F8007F42002BB8BF5B429F42B8BF1F46B7F5D9
:10B70800FA7F8346A8BF4FF4FA77B046B146B246EF
:10B718003446984B1B8813F0030045D0022C43D0C5
:10B72800934A32F91410019A4900524291424FEA61
:10B73800440503DB019A8A42A8BF0A468E4935F9B7
:10B74800019002999BF81C5031F91410C9EB0202C0
:10B7580002EB01099BF8081001FB09F2642192FB36
:10B76800F1F16FF0040202FB05FA514505DB05EB28
:10B7780085029142A8BF11468A46804D804A55F8F5
:10B78800241042F2107E49447145A8BF7146914287
:10B798009BF81290B8BF114609FB01F9012845F83A
:10B7A80024104FEA293942D0764D714935F91450A1
:10B7B800009A754831F9148092F801E050F8242075
:10B7C80085EAE576A6EBE576B6F5206F4FEA8401C3
:10B7D80020DC022C18D008EB8800000190FBFEFE4C
:10B7E800042095FBF0F5C5EB0E0E02EB0E0CBCF534
:10B7F8007A5F6548654DA8BF4FF47A5CAC45ACBF2D
:10B8080041F800C00D5007E088EAE876A6EBE87634
:10B81800642EE0DD002545505B48009A09587D26D6
:10B8280091FBF6F6D17A7143402691FBF6F69D0717
:10B8380012D5022C10D0C7F5FA7307FB06F507FBE3
:10B8480008F103FB0A114FF4FA7003FB095391FB4B
:10B85800F0F193FBF0F508E0D80704D5022C02D0EC
:10B868004D46514601E035464146464B33F91400F2
:10B87800042390FBF3F34648205C022C03FB00F3FF
:10B888006FF04F0093FBF0F30B444FEA440C08EEC3
:10B89800103A0ED13F4B4048D3ED000ACDF80CC00A
:10B8A800B8EEC80A1E21FEF723F8DDF80CC0BDEE7D
:10B8B800C08A344B39493CF803003CF901302CF874
:10B8C80001009BF850100FFA80FEC3EB0E034FF0F7
:10B8D800040E93FBFEF399B107EE903A30482D4BD6
:10B8E800CDF80CC0B8EEE70AD3ED000A00EBC400AF
:10B8F800FDF7FEFFFDEEC07ADDF80CC017EE903ABA
:10B908002849294811F804E018EE102A03EB4303EC
:10B9180051190EFB03F34FF0200E93FBFEF3C91AE7
:10B928002CF8001013490988090508D51F4909781A
:10B938004A0704D5E0B20393FAF73AFC039B1C4983
:10B9480018EE102A41F824201A4941F824501A49BF
:10B958005B4241F82430009B01340133032C0093EF
:10B968007FF4D7AE05B0BDEC028BBDE8F08F00BF09
:10B9780094260020A80F002004100020741F002027
:10B98800F0D8FFFFD20F0020AC26002080C1FFFFB7
:10B998005C1F0020A8260020A0260020841F00206D
:10B9A800C4260020701F0020DC260020D22F002093
:10B9B800E4260020F0260020FC2600202DE9F04F88
:10B9C80087B06D4C02916D4922880E68B4F810E07A
:10B9D800B4F80CC0C2EB26135200C2EBE602B4F96D
:10B9E80002605B435643B4F904201B1353439B1373
:10B9F80003EBE62606EB86038033B6F5FA384FEA02
:10BA0800E6774FEA232347F1FF3904934B68B4F9EB
:10BA180008200393A8FB08AB08FB09F30BEB430BC7
:10BA2800E3890593D31708FB03F10546B4F90A0027
:10BA3800A66102FB0911A8FB02230B44C1171F03CF
:10BA48000AFB01F300FB0B33AAFB000116031944A0
:10BA580047EA1257020A42EA016292194FEA212381
:10BA6800E6887B41003243F50043A2FB060106FB52
:10BA780003114B100093CB170193DDE90023134307
:10BA88006DD00FFA8EF0BDF91460C1170AFB01F1F1
:10BA9800AAFB002300FB0B11F7170B4408FB07F167
:10BAA80006FB0911A8FB06670F4479047004801887
:10BAB80041EAD6315941039BC3F5801E7246D3171C
:10BAC8000FFA8CF8002212184FEACE764FEAC377A5
:10BAD8004FEAC8034B4147EA5E07B61A67EB03070C
:10BAE80040F63543A6FB030103FB0711DDE90023FC
:10BAF80004F0BAFAB4F916204E13470B47EAC147C7
:10BB080002FB06FED31707FB03EEA2FB07237344D1
:10BB1800564307FB0366A2FB07233344560E46EA47
:10BB2800C3168219B4F914604FEA636741EB07033F
:10BB38007143F71700FB0717A6FB00013944C60C31
:10BB480046EA413692194FEAE1474FEA1221B4F921
:10BB580012207B4141EA036113010B4400E00023FA
:10BB68000DB11B0A2B60029B13B11A46049B13608C
:10BB780007B0BDE8F08F00BF680200208C1F0020CE
:10BB880070477047054B1A7A02F0FF0122B1012273
:10BB9800027000221A727047017070478C1F0020D3
:10BBA80037B5104B04465D68187806216A46A847E1
:10BBB800A8B19DF800209DF8013043EA02232380B4
:10BBC8009DF802209DF8033043EA022363809DF824
:10BBD80004209DF8053043EA0223A380012003B026
:10BBE80030BD00BF5402002013B5104B04465B68FB
:10BBF8003B2006216A469847A8B19DF800209DF889
:10BC0800013043EA022323809DF802209DF8033087
:10BC180043EA022363809DF804209DF8053043EA37
:10BC28000223A380012002B010BD00BF54020020EF
:10BC380007B5F7216B4606227620F9F7A9FF9DF88C
:10BC480000309DF801100C4A1B0343EA01139DF8CC
:10BC5800021043EA111353609DF803309DF8041055
:10BC68001B0343EA01139DF8051043EA11131360FF
:10BC780003B05DF804FB00BF8C1F002030B50546FB
:10BC88000C461346294622466820BDE83040F9F79D
:10BC98007FBF7620F4213122F9F7F6BF03460A4622
:10BCA80068201946F9F7F0BF094B1B681869094B5A
:10BCB80020F01F0210B5D258012400F01F0304FA27
:10BCC80003F31A4203D0FCF749FD034B1C7210BD65
:10BCD80060020020140401408C1F0020F0B5314D93
:10BCE8006B7A85B0002B5BD12F4C2368002B57D083
:10BCF8001A682E4E12B171690A4372619A88ADF8BA
:10BD08000020022298688DF80320694600228DF8E9
:10BD18000220F9F727FEB36943F00103B3612368F2
:10BD2800187B197DFCF7CAFD22689368188A9388E6
:10BD380018402AD1567D1E4A536811464BB3D36822
:10BD480033B303F015F823681869FCF707FD236877
:10BD58001B69029308230DEB0300002701268DF8C9
:10BD68000D308DF80C708DF80E60FCF72FFB2368F2
:10BD78008DF806705B7D8DF8043001A803238DF8DB
:10BD880005308DF80760FCF703FB01236B7207E0B1
:10BD9800012301EBC3020748506001F83360D2E782
:10BDA80005B0F0BD8C1F002060020020001002408A
:10BDB8000C2C0020B1BC000870B50446FFF78EFFBC
:10BDC800B4F5807F0ED0BB2C0ED8612C0ED8292C50
:10BDD8000ED8132C0ED8092C0ED8002C14BF06250B
:10BDE80000250AE0002508E0012506E0022504E018
:10BDF800032502E0042500E00525154C8021A368F1
:10BE08006B209847642002F086FFA36803216B200B
:10BE18009847104AA3681178192098470F2002F014
:10BE28007AFFA36829461A209847A36818211B207F
:10BE38009847A36810211C209847A368022137203F
:10BE48009847A36838200121BDE87040184700BF13
:10BE5800540200208402002008B5FFF73FFF074B7B
:10BE68005B7813B1012B03D008BD4FF4006201E0E9
:10BE78004FF48052024B1A8008BD00BF51020020C7
:10BE88000C0000202DE9F0410369C76805460E46FD
:10BE98001F40002F35D0B7FA87F24FF00043D34048
:10BEA800DB432B611F40A2F11B03042BF1D8DFE811
:10BEB80003F0221F1C190300746A24B1013C0023FB
:10BEC800A4B2736201E0EC6AA4B2D6F82080B8F19B
:10BED800000FDED0D8F80030404621469847D8F801
:10BEE8000480F4E73068696B07E07068A96B04E0C8
:10BEF800B068E96B01E0F068296C036889B298477B
:10BF0800C7E7BDE8F0811FB50123ADF80830ADF8EB
:10BF18000410002301A9ADF80A30ADF80C30ADF8D3
:10BF28000620FCF7E0FC05B05DF804FB8379DB072D
:10BF3800D0F8343144BFB1FA81F149095A681B89F4
:10BF480009B19361704713857047104B73B5187822
:10BF58001C4698B105230E4D8DF800304FF48056DD
:10BF680000238DF8013001A82E8569460222FCF7CE
:10BF7800D9F9AE619DF8050000F0010000F001005C
:10BF8800207080F0010002B070BD00BFDD05002008
:10BF980000040048064B70B51D6806461C46FFF7AE
:10BFA800D4FF18B923685B1BB342F8D970BD00BF32
:10BFB800D82B0020F7B503238DF80430030C8DF837
:10BFC80005308DF80700030A06200F4614468DF841
:10BFD8000630FFF7DFFF78B1084D4FF4805601A90E
:10BFE80004222E850020FCF79DF9384600212246C0
:10BFF800FCF798F9AE61204603B0F0BD0004004894
:10C00800014802493EE700BF00480140402D00209A
:10C018000148024936E700BF00400140F02C0020EB
:10C02800014802492EE700BF00080040C82C002044
:10C038000148024926E700BF00040040A02C002068
:10C048004FF0804000491DE7782C002010B5054CC2
:10C0580005482146FFF716FF04F1C8010348BDE86B
:10C0680010400FE7502C0020002C014000440140F4
:10C078000148024906E700BF002C0140502C00206F
:10C08800224B10B5224C5A43224BB3FBF2F20388E1
:10C098000139013AA04289B292B29BB20ED004F59E
:10C0A8000064A0420AD0B0F1804F07D0A4F59834BC
:10C0B800A04203D004F58064A04202D123F07003AB
:10C0C8009BB2154CA04206D004F58064A0421CBF68
:10C0D80023F440739BB203800D4BC16298420285E2
:10C0E8000FD003F5006398420BD003F540639842E4
:10C0F80007D003F58063984203D003F58063984224
:10C1080001D1002303860123436110BD40420F0083
:10C11800002C014000A24A040010004073B50546F7
:10C128000068FFF7ADFF2A6813889BB243F001034C
:10C138001380EB7A8DF804300124002601A88DF8CD
:10C1480005408DF806608DF80740FCF721F9EB7A79
:10C158001B2B0BD1192301A88DF804308DF805404D
:10C168008DF806608DF80740FCF712F902B070BD33
:10C17800134B800A984220D00AD84A3B984212D0E2
:10C188000133984211D0B0F5801F14D101207047B7
:10C198000C4B98420BD0013398420AD0023B98428C
:10C1A80009D10420704702207047032070470520FA
:10C1B800704706207047FE2070470020704700BF78
:10C1C8004B00100051001000F8B5046806462046E0
:10C1D8000F461546FFF7CCFF06284BD8B27A9108D0
:10C1E80047B902238B40D4F80CE0DB439BB203EA47
:10C1F8000E03E3600A23204A03FB001342F823706E
:10C20800043342F8235015463FB1B17AE2688908F1
:10C2180002238B409BB21343E360282202FB0052A7
:10C228002032EFF31286502383F3128803B203EB14
:10C238008303DB0003F10C011C3329442B4451F820
:10C24800047F17B117600A6804329942F7D10023B6
:10C258001360F3B283F31188282303FB0050036AA9
:10C268001BB1E36843F0010303E0E2684FF6FE7395
:10C278001340E360F8BD00BF502C0020014800F0D7
:10C288008BB800BF981F0020014800F085B800BF98
:10C29800EC1F0020014800F07FB800BF40200020BC
:10C2A800026BC168034610B5406942B11A6C8C1A1A
:10C2B800013A005D08BF0A46C0B21A6410BD1A6A86
:10C2C800805C01328A4228BF0022C0B21A6210BDC7
:10C2D800436B13B190F844007047836A406A1B1A95
:10C2E800584258417047426A816A03698A4238BF96
:10C2F800D218521A416B21B149680A44591E8A4220
:10C3080003D2013B981AC0B2704700207047036BF4
:10C3180013B15B68016C01E0C369016A8B423CBFE1
:10C32800C2689B18581AC0B27047836A8169426B09
:10C338001944D160416A99429DBF0169CB1A536083
:10C34800CB1A96BF0023536083624FF0000380F836
:10C358004430136888BF816243F00103136070475B
:10C36800436A8269D154436A02690133934228BF00
:10C3780000234362436B1BB11B68DB0705D4D4E77A
:10C38800026D136843F08003136070474171F9F739
:10C398000BB98160F9F708B9026D036B70B50446F3
:10C3A800D5699BB9A90611D5C36A1BB1908C80B217
:10C3B80098470BE0E169928C40694E1CD2B2E66165
:10C3C8004254E169E268914228BFE361616BA1B917
:10C3D8002A0612D5636AA26A9A42236D09D0501CB4
:10C3E800A669A062B25C1A852369984205D3A16246
:10C3F80003E01A6822F080021A602B0742BF236DFF
:10C4080008221A6270BD0D4B0D484FF400525A6055
:10C418000C4A11684FF6FE730B401360426B1168AB
:10C428004FF6FE730B401360426A836A9A4200D04B
:10C438007BE7012380F84430704700BF00000240CA
:10C4480040200020440002402DE9F0471E46A64B3C
:10C458008CB09842894690469DF8505040F08580AF
:10C46800A24BA34A1A60A34A5A6102F580729A61E4
:10C478004FF48072DA601A619F4A1A63143A5A6359
:10C48800A2F54842203ADA6404329A64C3F8088074
:10C4980018659A4B9A6942F480429A615A6942F047
:10C4A80001025A6102238DF80830032315F0010AAE
:10C4B8008DF809304FF000038DF80A3014BF0223BD
:10C4C80001232C078DF80B3019D54FF090444FF409
:10C4D800007701978AF001038DF80A30636A23F028
:10C4E800F0036362636A43F070036362204601A944
:10C4F80002F022FABAF1000F27D1A76125E0B007B0
:10C5080010D50CA94FF4007341F82C3D4FF0904022
:10C51800436A23F0F0034362436A43F070034362C3
:10C5280002F00AFAF10710D50CA94FF4806341F81C
:10C538002C3D4FF09040436A23F470634362436A92
:10C5480043F4E063436202F0F7F90E238DF80030FC
:10C558000022012368468DF801308DF802208DF8FD
:10C568000330624CFBF714FF0BE1654B984276D120
:10C57800644B5F4A1A604FF48072DA601A61624A4B
:10C588005A6102F580729A615C4AC3F8088018659E
:10C59800D36943F40033D36102238DF808300323B1
:10C5A80015F0010A8DF809304FF000038DF80A30B4
:10C5B80014BF022301232A078DF80B3019D54FF039
:10C5C80090444FF4804701978AF001038DF80A30B0
:10C5D800636A23F070636362636A43F0E0636362D3
:10C5E800204601A902F0A8F9BAF1000F27D1A761E6
:10C5F80025E0B30710D50CA94FF4804341F82C3D32
:10C608004FF09040436A23F070634362436A43F0FB
:10C61800E063436202F090F9F70710D50CA94FF4D4
:10C62800004341F82C3D4FF09040436A23F070439B
:10C638004362436A43F0E043436202F07DF92623F4
:10C648008DF800300022012368468DF801308DF8FE
:10C6580002208DF803302B4CFBF79AFE91E02B4B10
:10C66800984240F00F812A4B214A1A604FF4807299
:10C67800DA601A61274A5A6102F580729A611F4A84
:10C68800C3F808801865D36943F48023D361022373
:10C698008DF80830032315F0010A8DF809304FF0A2
:10C6A80000038DF80A3014BF022301232C078DF8EC
:10C6B8000B3033D5184C4FF4806701978AF001038B
:10C6C8008DF80A30636A23F470636362636A43F423
:10C6D800E0636362204601A902F02EF9BAF1000F67
:10C6E80040D1A7613EE000BF003801404020002053
:10C6F800BC57010894200020580002400010024056
:10C7080000440040EC1F0020942200200048004014
:10C71800981F00209424002000040048B0070FD57B
:10C728000CA94FF4806341F82C3D5848436A23F420
:10C7380070634362436A43F4E063436202F0FCF8C7
:10C74800F1070FD50CA94FF4006341F82C3D4F4871
:10C75800436A23F470434362436A43F4E043436209
:10C7680002F0EAF827238DF80030002201236846FA
:10C778008DF801308DF802208DF80330FBF708FEA4
:10C78800434CC4F82C900027012384F844302762D6
:10C79800E761A76267626671C4F80880A5712046E0
:10C7A800F8F702FFF20734D5236B002B2AD001A833
:10C7B800FBF7E0FFE36C01934FF480530A93802367
:10C7C8000693E368ADF8103020230993206B636962
:10C7D80002930B970597079708970397FBF7F5FFC1
:10C7E80001A9206BFBF7D3FF236B216D1A6842F078
:10C7F80001021A608A6842F040028A605B689BB254
:10C80800236406E0236D20221A621A6842F020028F
:10C818001A60B3072FD5636B43B301A8FBF7AAFFD0
:10C82800A36C01934FF480530A93802306932369E2
:10C83800ADF8103000251023606B03930B95059518
:10C84800079508950995FBF7C0FF606B01A9FBF7F1
:10C858009EFF636B1A6842F002021A60226D5D60E7
:10C868005D60936843F08003936004E0226D136871
:10C8780043F080031360226D136843F001031360D3
:10C88800204600E000200CB0BDE8F0870004004816
:10C89800981F00202DE9F04F2DED028B85B08146C1
:10C8A80003938A4B02921B889D0737D5109B8848B3
:10C8B800DC89B0F900301B1B03F2F31540F2E632B5
:10C8C800954203D8002BB8BF5B4201E04FF4FA73DE
:10C8D800B0F90220121B02F2F31440F2E63084424F
:10C8E80003D8002AB8BF524201E04FF4FA729342CB
:10C8F800B8BF1346C3F5FA73052293FBF2F30A2275
:10C90800643B534399F81C20D2105343642293FB91
:10C91800F2F3134423EAE373DBB200E064230093E9
:10C92800CB1C0193C8460025019B6A4813F8011FD8
:10C938000193022D4FEA450A06D1B0F9040001F12E
:10C948001B04444363112DE030F91520029B50006D
:10C958005B42984203DB029B8342A8BF03465E48C2
:10C9680030F90A40039830F915001B1B1844574B3F
:10C978001E88F40712D401F11B035A43B1074FEA8A
:10C9880022130FD599F812409DF9001044434C43E7
:10C99800642294FBF2F203EB221303E099F80830C7
:10C9A80043431B114D4A042432F90A2092FBF4F444
:10C9B8001C1B484B03F108026421AF5C98F8012066
:10C9C80062437A43022D92FBF1F24FEAE21208EE3B
:10C9D800102A0AD1B8EEC80A03F10C001E21D3EDC3
:10C9E800050AFCF785FFBDEEC08A3A4A3C4B98F829
:10C9F8000B601B8802F1180E03FB04F05EF825108B
:10CA0800C01206FB0016B6F5001F3649A8BF4FF442
:10CA1800001602F124008E42B8BF0E4650F82510C9
:10CA280040F82540611A1B094FF6FF70B0FBF3F37D
:10CA38004B4399F850104EF825604FEA850B761352
:10CA48009B1179B107EE903A02F13000B8EEE70A8F
:10CA580000EBC500D2ED050AFCF74AFFFDEEC07AEF
:10CA680017EE903A98F815101F4A03EB43034B430F
:10CA78005F43642397FBF3F718EE103A3F123344F1
:10CA88003B4422F80A30114B1B881A0506D5174B70
:10CA98001B785B0702D5E8B2F9F78AFB144B18EE4E
:10CAA800102A01354BF8032003F10C021833032D2B
:10CAB8004BF802604BF8037008F101087FF434AFBB
:10CAC80005B0BDEC028BBDE8F08F00BFA80F0020B9
:10CAD800AC2B00209426002004100020D20F002048
:10CAE800241000200000E0FFDC260020D22F0020C8
:10CAF800E42600202DE9F04F2DED0A8B97B011F0B8
:10CB0800FD0806460191A94C06D0A94B1B689A0757
:10CB180000F1B08000F041BCA36FA648DFF8949202
:10CB280098470028F1D0A44F94F8882048464946F1
:10CB380001F03EFF3B8804F1D802002B70D0D4F8F6
:10CB48008C301B7808EE103A04F1900A04F19C0529
:10CB5800B7F800B039F91800BBF57A7F02BF002397
:10CB6800CAF800302B61DAF800300344CAF8003004
:10CB78002B6907EE900A0133012B4FEA4801F8EEC2
:10CB8800E77A2B6106D10023C5ED017AC5ED007A5D
:10CB9800AB601BE0D5ED006A07EE103A37EEE66AA7
:10CBA800B8EEC77A86EE077A36EE877AD5ED026A4E
:10CBB80085ED017A77EEC77A85ED007AE6EE276A89
:10CBC800F0EE667AC5ED036AC5ED026A0023BBF193
:10CBD800010F29F8013053522DD12B690392012BF3
:10CBE800C3BF03F1FF3300EE103AD5ED037A9FED92
:10CBF800730A0291C4BFB8EEC00A87EE800A06F035
:10CC080063FE0299039A18EE103A5BB1F8EEC87AFF
:10CC1800B4EEE70AF1EE10FA04DD4FF47A733B80C4
:10CC280000231CE0DAF800304FF47A7003F5FA7349
:10CC380093FBF0F3535208F10108B8F1030F0AF11E
:10CC4800040A05F1140583D1BBF1010F04D158463C
:10CC5800029202F003F8029A3B88013BDFE739F8B9
:10CC6800131032F81300091A29F813100133032B93
:10CC7800F5D14AE7019B002B00F08F8394F8DE7012
:10CC88004A4D6FB1012F40F0808305F59470D5EDC2
:10CC9800486A95ED497A05F59A730021804613E1B3
:10CCA80002F012F8D5F8E8309FED457AC5F8E000B3
:10CCB800C31A07EE903AF8EE677A424BC5F8E800D7
:10CCC80067EE877A5B68C5ED397A05F1EC0098471D
:10CCD80005F1EC08002800F0F1803B4B40461A783B
:10CCE800414601F065FEB5F8F230002B42D0D5F888
:10CCF800F4103B46B4F8F22038F913702B4DB2F516
:10CD0800C87F324A04BF002042F823004FEA830E4E
:10CD180052F80E00384442F80E00002028F813009C
:10CD280021F813000133032BE4D1B5F8F230012BBD
:10CD38001BD1D5F8F8304FF4C87703F1C80292FB3D
:10CD4800F7F20A80D5F8FC20C83292FBF7F24A8045
:10CD58001F4AD5F800311288C83393FBF7F39B1AA2
:10CD68008B8030807080FDF7A5FBB4F8F230013B72
:10CD7800A4F8F230174B1B685B0740F18B80B4F8BE
:10CD880004210A4B322A27D1D3F8F4201188A3F8BA
:10CD9800061151889288A3F80A213288A3F80C2139
:10CDA8007288A3F80811A3F80E2117E09426002032
:10CDB800A40F0020D20F0020CE2F0020000000007A
:10CDC800BD378635DC280020D42F00208C27002092
:10CDD8000C000020A82B0020002A3BD0D4F8F40037
:10CDE8000023B4F8042138F913E0C64D322AC64AA4
:10CDF80004BF002142F823109F00D1597144D1513A
:10CE0800002228F8132020F813200133032B1146A1
:10CE1800E7D1B5F80431012B17D10C2085F81C2176
:10CE280085F81D3101F01AFFD5F8F430B5F8062160
:10CE38001A80B5F808215A80B5F80A219A80B5F801
:10CE48000C313380B5F80E317380B4F80431013BEE
:10CE5800A4F8043194F81E31AA4ADBB1D2F8F400E0
:10CE6800D2F81031002182F81E11322593FBF5F318
:10CE78000380D2F8143193FBF5F34380D2F81831CC
:10CE8800A24A93FBF5F312889B1A83803180718044
:10CE9800FDF710FBD4F8F420B4F8EC3011885B1AD5
:10CEA800A4F8EC305188B4F8EE305B1AA4F8EE30F0
:10CEB8009288B4F8F0309B1AA4F8F03094F8DE3079
:10CEC800013384F8DE30D9E68E4D914F05F1EC023E
:10CED80032F8112027F8112012B207EE902A8D4A55
:10CEE800F8EEE77A32F9112067EEA67A0131E0EC24
:10CEF800017A07EE902AF8EEE77A032967EE877A37
:10CF0800E3EC017AE0D105F59A7005F5A0710246C7
:10CF180002F08BF905F59A7005F5A67104AA02F0DE
:10CF280084F904A895ED390ADFF8D8A1014602F082
:10CF380095F9DDED054ADDED047A9DED065A95ED8E
:10CF4800594AD5ED583A95ED563AB6EE007A64EE60
:10CF5800874A67EE875A64EEA47A25EE075AE5EE0B
:10CF6800A57A07A80146B7EE008AE5EE057A0AAA6F
:10CF78000DAFF0EE482AE7EEC72A0AF5BC7965EE50
:10CF8800846AD5ED577AE2EEA36A25EE236AE4EEC9
:10CF9800836A23EEE57AB1EE452AE2EE276AA2EE2D
:10CFA800A76AA4EEA77A67EEE57AF1EE641AE2EED4
:10CFB800837AA1EE846AA2EE847AE1EEA37AA5EEE2
:10CFC800836AA5EE037AE2EE047A85ED576AC5ED29
:10CFD800567AB1EE466AC5ED586A85ED597AF1EE92
:10CFE800666AB1EE477A8DED097A8DED076ACDED67
:10CFF800086A02F01AF995ED560A474810A902F096
:10D008002DF907A8444913AA02F0F0F813A810A9AB
:10D018003A4602F00AF90AA8394613AA02F0E6F8D5
:10D028003D4813A93A4602F000F9D5ED5A7A9DED2C
:10D038000F7A95F86C31B4EEE77AF1EE10FACCBFBE
:10D0480043F0080323F0080385F86C31D4F87031F5
:10D058001B78F0EE489A0AF5C4753BB3DAED5D8AA1
:10D068004846B0EE680A10A902F0F8F89AED618A0D
:10D078000AF59470B0EE480A13A902F0EFF84A4690
:10D0880010A813A902F0D1F82846B0EE680A10A932
:10D0980002F0E4F8384613A9B0EE480A02F0DEF8C8
:10D0A80010A813A92A4602F0C0F807E098E807007C
:10D0B80089E8070097E8070085E80700D4ED4B7A70
:10D0C800D4ED4A6A94ED4C7A0E4D67EEA77A0023A8
:10D0D800E6EEA67AE7EE077A9FED107AF4EEC77AC5
:10D0E800F1EE10FA06DC9FED0E7AF4EEC77AF1EE57
:10D0F80010FA19D5C4F84C31C4F85031C4F8543179
:10D1080025E000BF94260020A42700200C00002062
:10D11800CC0F0020D20F0020E0570108B81E8D3F29
:10D128003D0A673F6F12833A05F5BC7005F5C47177
:10D1380005F5A67202F05AF8D5ED397A1FED070AFF
:10D1480005F5A67080EE270A014602F087F8B4F8C4
:10D158009431984D01339BB2B3F57A7FA4F894319A
:10D168002ED195ED570AD5ED566A95ED587AD5ED3D
:10D17800597A20EE000AA6EEA60AA7EE070AA7EE3D
:10D18800A70A06F0A1FB89EE800A0023A5F89431CE
:10D19800D5ED576A95ED587AD5ED597A95ED566AD9
:10D1A80060EE266A20EE077A60EE277A26EE000AFD
:10D1B800C5ED576A85ED560A85ED587AC5ED597A59
:10D1C800D4ED578A94ED59AA94ED56BAD4ED58AADD
:10D1D8009FED799A68EECA7AB7EE007AEBEE2A7A72
:10D1E80077EEA77AF4EEE97AF1EE10FA0EDCFFEEAC
:10D1F800006AF4EEE67AF1EE10FA24D4F4EE477AF7
:10D20800F1EE10FAC8BFF0EE477A01E0F0EE477A87
:10D2180017EE900A02F084FE41EC100B06F050F96C
:10D2280051EC100B02F0D0FE08EE100AB5EEC08AE1
:10D23800F1EE10FA09DD78EE497AF5EEC07AF1EEF2
:10D2480010FA10DC23E09FED5D8AF1EE487A77EE64
:10D25800C97AF5EEC07AF1EE10FAB5EEC08A13DDA0
:10D26800F1EE10FA06DD38EE499ADFED557AB4EEA4
:10D27800E79A03E09FED527AF4EEC77AF1EE10FADE
:10D288004CBF0123002312E0F1EE10FA06DD38EE60
:10D29800499ADFED4C7AB4EEE79A03E09FED497ABC
:10D2A800F4EEC77AF1EE10FACCBF0123002353B194
:10D2B800B0EE4A0AF0EE4B0AFCF767FD9FED42CA52
:10D2C80070EE008A41E02AEE8A0A6AEEAABAABEE4C
:10D2D800280AB0EE6B7A30EE000AA8EEA87AB5EE0E
:10D2E800400AF0EE007AF0EE690AF1EE10FAE7EE85
:10D2F800670AB0EE679A04D1F5EE400AF1EE10FA2B
:10D3080004D0FCF742FDB0EE40CA01E09FED2ECA02
:10D3180028EEAA0AEAEE0ABAABEE0A0AF0EE690AA1
:10D3280030EE000AEBEEC90AB5EE400AF1EE10FA4B
:10D3380004D1F5EE400AF1EE10FA04D0FCF725FD11
:10D34800F0EE408A01E0DFED208A9FED209A204D23
:10D358002CEE090A06F06EF828EE090A288006F075
:10D3680069F8DFED1C7A1C4A688068EEE78AFDEEF2
:10D37800E88ACDED018ABDF8043013F4004F18BFD8
:10D3880003F5B4731380002300E00123002284F81E
:10D39800DE20002B7FF472AC06E00023A4F8EC300A
:10D3A800A4F8EE30A4F8F03017B0BDEC0A8BBDE855
:10D3B800F08F00BF94260020DB0FC93FDB0FC9BFE9
:10D3C80035FA0E3C35FA0EBC000000004D3D0F4406
:10D3D80004100020E12E65420810002001380A4B95
:10D3E800042804D8DFE800F00507090B0D00074AF8
:10D3F80008E0074A06E0074A04E0074A02E0074A4D
:10D4080000E0074A1A60704760000020D9B600089B
:10D418009DC8000801F60008D9B3000895B00008B7
:10D428002DAA00080846FBF76BBD0F4B1A786F2A28
:10D4380017D1598840F2E472914212D11A79BE2A62
:10D448000FD193F8E027EF2A4FF000000BD113F823
:10D45800012B5040054A9342F9D1B0FA80F04009B7
:10D46800704700207047704700F80108E4FF010882
:10D478002DE9F04F2DED028BF24C85B0002140F2E2
:10D48800E472204605F0C7FDEF4B04F53A721A60C6
:10D49800EE4B00261E70EE4B04F2B2721A606F2338
:10D4A8002370022003236371FCF772FD4FF4807030
:10D4B800FCF76EFD20224FF4167384F868216E2263
:10D4C800A4F8643184F87A21FA230A22A4F8663190
:10D4D80084F87B214FF4FA732B22A4F86C3184F87A
:10D4E8007D210123212284F85E3184F8693184F892
:10D4F8006A3184F87C3184F87E2184F884312322CF
:10D50800002384F87F21C4F81C32C4F820324FF479
:10D51800C872052384F8B067A4F87061A4F86E6136
:10D52800A4F8726184F8556184F8566184F85761EB
:10D53800A4F85861A4F85A61A4F85C6184F85F61A2
:10D54800A4F88261A4F88021A4F8866184F819629D
:10D5580084F8186284F8246284F8256284F82732F3
:10D5680040F2DC53A4F8963140F24C43A4F89831C9
:10D5780040F26C73A4F89A3140F27533A4F89C31E8
:10D5880040F64303A4F89E3184F8266284F890613B
:10D5980084F8916125462346032ECCBF0122002240
:10D5A80006F1010683F8A02114BF1E220522122EBF
:10D5B80083F8A12103F10203EED140F27E42A4F8E0
:10D5C800402140F23A724FF4FA63A4F8422140F243
:10D5D8007E52A4F8C631A4F8CA31A4F8CE31A4F812
:10D5E800D231A4F84821052340F2EA5284F8E03108
:10D5F800A4F84A21C82340F2B452002601274FF468
:10D608007A7B4FF01E0840F2DC504FF0190AA4F85C
:10D61800E431A4F84C214FF4C8733222A4F8E8315D
:10D62800A4F846010390A4F84E21A4F8503184F8D8
:10D63800938184F8DF7184F8E1A184F8E27184F8B9
:10D64800E37184F8E67184F8EC7184F8926184F8E7
:10D658009461A4F8C4B1A4F8C8B1A4F8CCB1A4F8F2
:10D66800D0B184F8D46184F8DE6184F8EA61A4F862
:10D6780044B1A4F85221029284F85461FAF786FF63
:10D68800DFF8C4C12673DCF80030029A83F80B80F7
:10D698004FF05F0E83F803E04FF00F0E83F805E0BC
:10D6A8004FF0220E83F806E04FF00E0E83F810E0DC
:10D6B8004FF0350E83F81AE04FF0210E83F811E091
:10D6C8004FF0530E83F81BE04FF05A0E83F808E032
:10D6D8004FF0780E83F80AE04FF02D0E4FF028092E
:10D6E800142183F80C8083F807A04FF00A084FF044
:10D6F800640A83F814E04FF4FA7ECDF804C01F7072
:10D70800597599755A731A719F7783F8019083F840
:10D71800029083F817809E731E76DE735E7683F818
:10D72800128083F81CA083F80990A3F84EE0DFF874
:10D738003CE1C3F838E0C3F83CE0DFF834E1C3F873
:10D7480028E0DFF830E1C3F834E0DFF82CE1C3F873
:10D7580048E0DFED407A9FED408AC3ED0B7A4FF049
:10D768004B0E83F84CE04FF4E17EC3ED0C7AA3F83E
:10D778005CE0B7EE087AF1EE047A4FF0100E83F809
:10D788005EE083F8509083ED087A83ED097A83EDA3
:10D79800108AC3ED117A83F8536083F8548083F8B4
:10D7A800558083F8568083F857A083F858A083F8EB
:10D7B80059A083F85A60039884F8B4274FF0460EAE
:10D7C800042284F8BA1784F8B3E7A4F8BC0784F8ED
:10D7D800B2A784F8B56784F8B96784F8B66784F89F
:10D7E800B76784F8B86783F86820152283F874202F
:10D7F8001A4A9A671A4ADA671A4AC3F8802083F8DD
:10D808008470A3F86460A3F86660A3F86260C3ED4F
:10D818001B7A83F8709083F871901348FAF7F6FE34
:10D82800DDF804C0DCF800204FF4487382F820715A
:10D8380082F81D6182F81E6182F81F9182F82461C6
:10D848001CE000BFD0160020E80F0020B028002000
:10D8580028100020CDCCCC3E000000009A99193F3A
:10D86800F6287C3F3D0A773FA77501088FC2F53C33
:10D87800000060406666663F00004040A2F8223122
:10D88800114684F8D68184F8D781A4F8D8B184F8F1
:10D89800DA61A4F8DCA167460E2303FB06236FF0C8
:10D8A800170083F82501032083F826016FF02F0065
:10D8B80083F82701072083F828016FF0230083F8F5
:10D8C8002901052083F82A01642381F82B310136C8
:10D8D8005A2381F82C3181F82D31082E4FF0FF039F
:10D8E80081F82E3101F10E01D6D1002382F895314D
:10D8F8002E4B18EE102A45F8102F9D42F9D12C48CE
:10D908000021402205F087FB00232A4D2A4C595953
:10D918001A1904330868C2F8A802382BF5D104F59F
:10D928000A700021802205F076FB05F1380170228B
:10D9380004F50A7005F064FBF8F7E0FB4FF40020EB
:10D94800FCF726FB3E680125314604F590604FF44C
:10D95800CC7284F8D85784F8D65784F8D75705F08E
:10D968004FFB04F5C36031464FF4CC7205F048FB19
:10D97800124B1B681A68C4F8BE275A68C4F8C22735
:10D988009A68C4F8C6271A68C4F8CA275A68C4F837
:10D99800CE279A68C4F8D227022384F8E05484F882
:10D9A800783605B0BDEC028BBDE8F08F90170020EB
:10D9B80078190020EC570108D01600202810002004
:10D9C8001549D1F8883043F47003C1F88830134BF7
:10D9D8001A6842F001021A605868114A02405A60F7
:10D9E8001A6822F0847222F480321A601A6822F4CB
:10D9F80080221A605A6822F4FE025A60DA6A22F01B
:10DA08000F02DA62186B074A02401A6300229A6012
:10DA18004FF000638B60704700ED00E0001002409B
:10DA28000CC07FF8CCFC00FF38B5144B1B6898423B
:10DA380005461ADD124B93F8D84714B1012C09D0CA
:10DA480017E0104B1B68186988B1A842CCBF0120A9
:10DA5800022038BD7F280CDCF8F7CEFDC0F17F002E
:10DA6800854208DDF8F7A6FD05E0002038BD012055
:10DA780038BD022038BD204638BD00BF8C2F00209D
:10DA8800D0160020EC2D0020074B93F8D837012B37
:10DA980008D1064A064BD0681B68834234BF002071
:10DAA8000120704700207047D01600201000002089
:10DAB800E005002038B5094B93F8D85765B9084CEC
:10DAC8002068FAF7A1F9074B25601B78022B03D1D0
:10DAD800BDE83840FAF71BBD38BD00BFD01600209E
:10DAE800EC2D0020EB2D0020064B93F8D8371BB106
:10DAF800012B05D1F8F75EBD034B186801F080B91A
:10DB080000207047D0160020EC2D0020F8B5011F2A
:10DB180006460023083051F8042F02F120043F2C58
:10DB28003BD802F108040F2C06D80232032A04D984
:10DB3800002B08BF012300E002238142EBD1012B17
:10DB480030680ED0022B1AD0736803F003039B00D1
:10DB580000F0030043EA0010B36803F0030318431E
:10DB680017E000F00F0040F04000FBF7C9F9B0687B
:10DB7800736800F00F0040EA0310C0B209E000F03B
:10DB88003F0040F08000FBF7BBF93079FBF7B8F9AC
:10DB9800307ABDE8F840FBF7B3B906F10C07344614
:10DBA8003A46002552F8043D03F18001FF294FEA67
:10DBB800850510D903F50041B1F5803F02D245F043
:10DBC800010508E003F50003B3F1807F34BF45F099
:10DBD800020545F00305B242E4D165F03F00C0B24A
:10DBE800FBF78EF905F00303022B207807D0032BEF
:10DBF8000CD0012B13D1FBF783F960780FE0FBF70A
:10DC08007FF96078FBF77CF9A07808E0FBF778F9F2
:10DC18006078FBF775F9A078FBF772F9E0780434BF
:10DC2800FBF76EF9BC424FEAA505DBD1F8BD10B58C
:10DC380004467F2C06D964F07F00C0B2FBF760F978
:10DC4800E409F6E7E0B2BDE81040FBF759B9430034
:10DC580083EAE070EBE72DE9F047314B93F8D837CA
:10DC6800012B86B0074601D004464AE005F017FAB2
:10DC780003A9054606466846F8F7ACFB039B049AD9
:10DC8800029713442B443F2B059519D90023684666
:10DC980003A90322F8F7CAFB039B3BB9049B2BB9E2
:10DCA800204A13705370059BABB301E0F8F77AFB79
:10DCB800039B049A059E134433447F2B2BD8029F61
:10DCC800DFF86090CA4639461AF8024BC4F180085A
:10DCD800B04528BFB0460AEB04004444E4B24246CB
:10DCE80005F08EF9802C89F8004014D1C8EB06069F
:10DCF800504607EB0801324605F082F989F80060C2
:10DD080009E0254614F8011B21B1074B186801F0FA
:10DD180080F8F6E7ED1B284606B0BDE8F08700BF9F
:10DD2800D01600202C280020EC2D00200FB437B589
:10DD380006AC482054F8045BFBF7E2F82020FBF718
:10DD4800DFF82A4623460B4901940020FBF702FF1F
:10DD580004460A20FBF7D4F8074BC4F1FF241A68DD
:10DD680004F57F04FD3414441C6003B0BDE8304062
:10DD780004B070472DD400088C2F00200FB407B5CD
:10DD880004AB064953F8042B01930020FBF7E2FE8D
:10DD980003B05DF804EB04B0704700BF2DD4000851
:10DDA80007B5064B0093064B01930649064A074BF5
:10DDB8000748FBF7BCFF03B05DF804FB1B680108CC
:10DDC800F3670108D6750108DB7501080F680108BB
:10DDD800B075010808B5037833B90C4B0C481978AD
:10DDE800BDE80840FBF7A3BF05F0B0F902280CD83E
:10DDF800064B1870074B0C2202FB0030064B023012
:10DE08001860FCF791F90548E5E708BDB02800203F
:10DE1800E2750108801E002028100020AB69010867
:10DE280008B503783BB90B4B0B4893F8B017BDE81E
:10DE38000840FBF77CBF05F089F9022808D8054B94
:10DE480083F8B007FCF7D6F8FCF792F90348E8E73F
:10DE580008BD00BFD0160020E6750108AB690108AF
:10DE680038B5037803BB214B1B6801330F2B07D848
:10DE78001F490C2202FB03121C4695682DBB00E0CB
:10DE88001C4601340F2C01DD002400E005D8184998
:10DE98000C2202FB04129568BDB99C42F1D11548C9
:10DEA800BDE83840FBF743BF05F050F90F2804469A
:10DEB80005D80F4A0C2303FB00239D682DB9214682
:10DEC8000D48BDE83840FBF732BF084B1C60FAF735
:10DED800D9F921462A460948FBF729FF0C235C4358
:10DEE800034B185DBDE8384000F0B8BE580000206C
:10DEF800C4580108F375010809760108217601085C
:10DF080073B5037813B9F9F73FFC3DE01F4901AA3F
:10DF180005F07DF9002401462646254699B134B11D
:10DF2800012C08D1084605F011F9064603E0084619
:10DF380005F00CF905461549002001AA05F067F916
:10DF480001340146EAE70B2D02D911480C220BE0F7
:10DF5800022C10D1A6F57A73B3F57A7F07D90D484C
:10DF68004FF47A714FF4FA62F9F78BFB0CE00A4B25
:10DF780003EB45035E80084B084803EB450329463D
:10DF8800B3F90220FBF7D3FE02B070BD7B6C010829
:10DF9800916C01084C700108B028002038760108FF
:10DFA80038B50D4C23688342054606D1F9F72CFF96
:10DFB800204600214C2205F02EF8E36CAB4209D133
:10DFC8002846F9F721FF054800214C22BDE83840D2
:10DFD80005F021B838BD00BF38160020841600208F
:10DFE800034BDA69D379591C1344D171187A7047F5
:10DFF800B028002010B5FFF7F3FF84B2FFF7F0FF59
:10E0080004EB002080B210BD10B5FFF7F3FF044603
:10E01800FFF7F0FF04EB004010BD38B5054D04468E
:10E028002146286A00F0F5FEEB69987960409871FE
:10E0380038BD00BFB0280020014BDB699879ECE7B8
:10E04800B028002038B5044624200D46FFF7E5FF28
:10E058004D20FFF7E2FF002C084C14BF21203E2082
:10E06800FFF7DBFFE369002228469A71FFF7D5FF27
:10E07800E36993F84900BDE83840CEE7B0280020AE
:10E0880001460020DEE710B50446C0B2FFF7C5FF21
:10E09800200ABDE81040C0E710B5044680B2FFF77B
:10E0A800F2FF200CBDE81040EDE737B582888368A1
:10E0B800044610060D4641BF2B4991F8B0174FF49E
:10E0C800CC7000FB0133D10544BF2849097802F020
:10E0D8003F0244BF01EB410103EB8103042A12D044
:10E0E80006D8012A0DD0022A32D193F9001030E067
:10E0F800102A0AD0202A0AD0082A29D1B3F90010F8
:10E1080027E0197825E0198823E0196821E093EDC4
:10E11800000A6846FBF7A0FC01461548FBF707FE16
:10E1280005B3D4ED037A6846B8EEE70AFBF794FC2A
:10E1380001461048FBF7FBFD94ED040A6846B8EE6B
:10E14800C00AFBF789FC01460A48FBF7F0FD09E025
:10E1580000210948FBF7EBFD25B10848E168226971
:10E16800FBF7E5FD03B030BDD0160020B028002035
:10E17800CF6A0108C86A01084B760108477601088A
:10E18800024B0146586A00F044BE00BFB028002088
:10E1980010B5441E14F8011F21B1034B586A00F052
:10E1A80038FEF7E710BD00BFB028002010B503788F
:10E1B8001BB90A48BDE81040EAE704F0C7FF044667
:10E1C800082899BF2146064806480821FBF7AFFDF5
:10E1D800601EC0B2BDE81040F9F7A4BD4E76010834
:10E1E80095760108C17601082DE9F3412B4E2C4B99
:10E1F80096F828002B4D1C682B4B05EB80001A88DD
:10E208002A4BD0F8C0101B78294800914FF47A7136
:10E21800B4FBF1F1FBF78BFD26484821FBF787FD9E
:10E22800254BD3F800800027FBB205EB8302D2F818
:10E23800D010E9B101249C4014EA080F16D0220737
:10E2480014D01E4AD25C0B2000FB0323154A1C483D
:10E2580002EB8303D3F8F020FBF769FD022C05D10C
:10E2680096F8341011B11748FBF761FD0137DBE769
:10E278001548FFF78DFF154B15481A68154B9A423C
:10E288000CBF154B154B1A88154B198892B240F2E2
:10E29800E47302B0BDE8F041FBF749BDB0280020A7
:10E2A800D82B0020C4580108A02B002068000020AB
:10E2B800EC7601082F770108A40F002064000020E5
:10E2C8003F770108477701088F7701089C0F0020E6
:10E2D8004B77010800540040A00F0020A20F002037
:10E2E800980F00202DE9F0410024804625460F4E66
:10E2F800A7594146384604F011FF58B139460C4831
:10E30800FBF715FD30190021FFF7CFFE0948FFF78D
:10E318003FFF0135143440F6CC339C42E7D11DB998
:10E328000548BDE8F04133E7BDE8F081645A0108CB
:10E33800746B01088F770108FA6A01082DE9F04F1C
:10E348002DED028B83B0054604F0A9FE064620B1E8
:10E35800012818D12B782A2B15D15C48FFF718FF14
:10E3680000245B4D5B486159FBF7E1FC28193146F5
:10E37800FFF79BFE5848FFF70BFF143440F6CC33E9
:10E388009C42EED19CE028463D2104F07AFE00280C
:10E3980000F08F800346994613F8012D202AFAD001
:10E3A800441C204604F0D2FE80462046FBF7CAFAF9
:10E3B800C5EB0909B0EE408A0026DFF834A1142223
:10E3C80002FB06F40AF5D07B54F80B70384604F0CB
:10E3D80066FE03461A4628463946019304F068FE4D
:10E3E800019B00285BD15FFA89F29A4257D10AEB68
:10E3F8000402D2ED6B7AF8EEE77A0BEB0405B4EE83
:10E40800E78AF1EE10FA48DBD2ED6C7AF8EEE77A9B
:10E41800B4EEE78AF1EE10FA3FD8B2F8A431D2F898
:10E42800A82113F0200F08BF08EE108A1C0641BF70
:10E438002A4991F8B0174FF4CC7404FB0122D9058E
:10E4480044BF2749097803F03F0344BF01EB41016A
:10E4580002EB8102042B18EE100A0BD004D8013B02
:10E46800012B0ED810700CE0102B05D0202B06D0F5
:10E47800082B06D1108004E082ED008A01E082EDCD
:10E48800008A39461748FBF752FC2846002103B09A
:10E49800BDEC028BBDE8F04F07E6134803E00136F8
:10E4A800972E8AD1114803B0BDEC028BBDE8F04F1E
:10E4B8006EE6284603B0BDEC028BBDE8F04F11E7CD
:10E4C80003B0BDEC028BBDE8F08F00BF7D7701087B
:10E4D800645A0108746B01088F770108D016002070
:10E4E800B0280020927701089D770108FA6A010890
:10E4F800C458010810B50A48FFF74AFE094B5C6A80
:10E50800204600F07DFC18B90A2000F004FCF7E76B
:10E5180000F0EAFDFBF744FD034B044ADA6010BD46
:10E52800BD770108B028002000ED00E00400FA05DE
:10E5380008B50548FFF72CFEFEF79AFFFBF75AFDD2
:10E54800BDE80840D6E700BFC977010808B5044808
:10E55800FFF71EFEFBF74EFDBDE80840CAE700BF07
:10E56800DF77010803788B4286BF024B33F811002E
:10E57800002070470029002070B500221346234967
:10E5880014180C44247E83EA0423082413F4004F4F
:10E598004FEA430318BF83F4815304F1FF3418BFD3
:10E5A80083F0010314F0FF049BB2EFD10132192A62
:10E5B800E5D100F1190200F11A050A440D44167E4E
:10E5C8002A7E02EB062292B29A421ED10F4B93F892
:10E5D8003950E2B2AA4215D2431C03EB4203DBB224
:10E5E800CA1801330B44127E1B7E03EB02239BB235
:10E5F8004FF4AF6253431B1303F5487321F81430EB
:10E608000134E6E7012381F83A3070BD0029002083
:10E6180003788B420BD9074B1A78074B89001944AA
:10E62800C86B02B1400800F5777080B270470020CF
:10E63800704700BFBC1E00200029002007299DBF8D
:10E64800034B03EB8101B1F86C000020704700BF59
:10E6580000290020034B03EB4101B1F88C00C008EE
:10E66800704700BF002900200A4BDFED0B7A03EB4F
:10E67800810191ED2B7AB8EE477AF6EE046AE7EE5F
:10E68800267A82B0FCEEE77ACDED017ABDF8040077
:10E6980002B070470029002000005C44024B03EBE5
:10E6A8004101B1F8F400704700290020024B03EB48
:10E6B8004101B1F81801704700290020024B03EB13
:10E6C8004101B1F818017047002900200020704767
:10E6D80070B5334C054600F0F7FAD4F83031C4F879
:10E6E8003001C31AB3F5FA5FC4F8343182BF00238E
:10E6F80084F8383184F8393194F838312BB9A12DA0
:10E7080002BF274A012182F8391194F83911244AA5
:10E7180029B1D118EDB201330D7682F8383194F869
:10E72800385194F83A31AB4239D11D4B93F83B310B
:10E73800052B02D0062B03D02CE00020FFF71CFF8E
:10E74800637E1E2B26D100200246C1B26B1E994261
:10E7580019DA21440B7E0821DBB283EA0206F607A8
:10E7680044BF83F01803C3F3460301F1FF3154BFDC
:10E778005B0843F0800311F0FF01C2F34702ECD1BC
:10E7880001301A46E1E723441B7E9A4202D1032056
:10E79800FFF7F2FE002384F8393184F8383170BD70
:10E7A8000029002010B5044600F08EFA0F4BD3F86C
:10E7B8003C21C3F83C01821A41F288318A42C3F8ED
:10E7C800402184BF002283F8442193F8442107495B
:10E7D80013440F2AE4B218BF013283F8454112BF2F
:10E7E80081F84421012381F8553110BD002900200A
:10E7F80010B5044600F068FA0F4BD3F85821C3F857
:10E808005801821A41F288318A42C3F85C2184BFD8
:10E81800002283F8602193F8602107491344142AE1
:10E8280018BF013283F8614112BF81F860210123CA
:10E8380081F8763110BD00BF0029002038B50446A4
:10E8480000F042FA274A2749D2F87831C2F878010D
:10E85800C31AB3F57A6F84BF002382F87C3192F82B
:10E868007C3133B9A82C3BD181F87D31A1F87E31B8
:10E8780006E0022B02D181F8804101E0242B02D866
:10E88800D11881F8814192F88011164D0133023177
:10E89800DBB249008B4282F87C3118DAB5F87E3158
:10E8A800E0B283EA0020082310F4004F4FEA40004A
:10E8B80018BF80F4815003F1FF3318BF80F00100C6
:10E8C80013F0FF0380B2EFD1A2F87E0138BD013109
:10E8D8008B4201BF002385F87C31012385F87D3107
:10E8E80038BD00BF0029002010B5044600F0ECF93F
:10E8F800104AD2F8A83140F6AC51C31A8B42C4BFB3
:10E90800002382F8AC3192F8AC31D11881F8AD41CE
:10E9180023B90F2C0DD10749C1F8A8010133DBB287
:10E92800192B044982F8AC310CBF0123002381F86C
:10E93800C63110BD00290020F0B500230E681C4622
:10E948000125A54005EA060EAE452BD10F797A1EA2
:10E95800012A15D8856803229A4025EA02028260B6
:10E968004D7982689D4015438560828892B222EA7B
:10E978000E0282808A798588A2402A4392B28280D8
:10E98800032205689A40D2431540056005689F40F8
:10E998002F430760C7681740CA7902FA03F547EAA8
:10E9A8000502C2600134102C03F10203C8D1F0BD86
:10E9B80038B52DED048B4A4C0368C4F8C8318388F8
:10E9C800A4F8CC31023A0D46062A05D8DFE802F051
:10E9D8000A101822292F3500B4F8C8310B80B4F872
:10E9E800CA3113E0B4F8CA310B80B4F8C83105E075
:10E9F800B4F8C8315B420B80B4F8CA315B4205E019
:10EA0800B4F8CA315B420B80B4F8C8316B80B4F8F3
:10EA1800CC311DE0B4F8C8315B420B80B4F8CA3180
:10EA280012E0B4F8CA310B80B4F8C8310CE0B4F87D
:10EA3800C8310B80B4F8CA3105E0B4F8CA315B427A
:10EA48000B80B4F8C8315B426B80B4F8CC315B42C0
:10EA5800AB80244B1B78002B3ED1B5F9003094EDE8
:10EA6800770AD4ED747A09EE103AB5F9023008EE57
:10EA7800103AB8EEC88AB5F90430B8EEC99A28EE4B
:10EA8800000A08EE903AA7EE890AF8EEE88AD4ED73
:10EA98007A7AA7EEA80A04F0CDFC94ED780AD4EDB2
:10EAA800757A288028EE000AA7EE890AD4ED7B7AC9
:10EAB800A7EEA80A04F0BEFC94ED790AD4ED767AA4
:10EAC800688028EE000AA7EE890AD4ED7C7AA7EEC2
:10EAD800A80A04F0AFFCA880BDEC048B38BD00BFC9
:10EAE800002900205C000020094BD3F8F42113789A
:10EAF80044F6FB7103EB431300FB03135078C0EBA0
:10EB08000030B3FBF0F39078B3FBF0F080B27047BD
:10EB18000029002010B50A4C94F8F93104EB43039E
:10EB28000A22B3F8081204F5067089B2A4F8101284
:10EB380000F072F980B2FFF7D7FFA4F8A00210BD69
:10EB480000290020124930B5D1F8A43203EB400463
:10EB58000A46257E15B1022D11D00BE0022805D9F1
:10EB6800032807D1D1F8A822D20401D5D88930BD0D
:10EB7800988A30BD02EB4000B0F8AC0230BD607E30
:10EB880000EB800000EB800000F2EE2080B230BD88
:10EB98000029002008B500F097F8074B022283F8F7
:10EBA800D422D3F8D822C3F8E4220122C3F8D00231
:10EBB80083F8FD2208BD00BF0029002008B500F039
:10EBC80083F8084B022283F8D422D3F8E42200F514
:10EBD800B71000F5587002F2DC52C3F8D002C3F83F
:10EBE800E42208BD00290020104B93F80023012AD5
:10EBF80010B51C460DD008D3022A0DD10C4A938AB1
:10EC08009BB283F00803938206E0094B08229A61BD
:10EC180002E0074B08221A8500F056F800F5F420A8
:10EC280000F59070C4F8040310BD00BF002900204F
:10EC380000040048034B4FF4004208B19A61704742
:10EC48001A85704700080048034B4FF4004208B18A
:10EC58001A8570479A6170470008004810B5E0B1FE
:10EC6800134B1B6813F0020304D0124B1B78012BC3
:10EC780013D900230C225A430F4C1119125D8242FA
:10EC880003D00133102BF5D110BD0C4B186840B1DF
:10EC98004A784078824204D310BDBDE81040F9F7A5
:10ECA800F1BA074A196000231380064A136010BDA1
:10ECB800A82B002068000020C45801083016002046
:10ECC8002C1600202816002010B50A4A0A4B116895
:10ECD8009B6800BF12689142F7D1084A14684FF444
:10ECE8007A7000FB04F2D31AB3FBF4F300FB013093
:10ECF80010BD00BFD82B002010E000E0082C002039
:10ED080038B50446FFF7E0FF0546FFF7DDFF401B77
:10ED1800A042FAD338BD10B504462CB14FF47A702E
:10ED2800FFF7EEFF013CF8E710BD024A1368013314
:10ED380013607047D82B002010B5094CA36823B185
:10ED480094F90420282A00D1984723693BB1044A42
:10ED580092F90C20282A02D1BDE81040184710BDAE
:10ED6800082C0020014B1B68184700BFBC2F00204F
:10ED78002DE9F84307460B24013C35D01D4B0822EA
:10ED88009A617D1C32264FF00508DFF86890B9F8C3
:10ED980014309BB283F00803A9F814300120FFF760
:10EDA800E1FF3046FFF7B7FFB9F814309BB283F0A4
:10EDB80008030020A9F81430FFF7D4FF3046FFF706
:10EDC800AAFFB8F1000F08D0B8F10108DDD14FF45F
:10EDD800FA70FFF7A0FFFA26D7E7013DD5D14FF427
:10EDE8007A70FFF798FFC7E7034B044ADA60BDE87B
:10EDF800F88300BF0004004800ED00E00400FA05B5
:10EE080003685B6918470368DB68184703685B6831
:10EE1800184703681B6818472DE9F84FB0F9023006
:10EE2800934218BF00232DED048B18BF037005789B
:10EE380004460E469146002D40F0978007EE902A32
:10EE4800DFED7D8AF8EEE77AB6EE009A67EEA88ADB
:10EE5800DFED7A7A68EEA78AA04668EE898A2746A7
:10EE6800B0EE680AFBF704F8B0EE408AB0EE680A24
:10EE7800FBF75EF888EE000A40F2DC536365102366
:10EE8800A4F852301823A4F85030DFED6D6A60EE14
:10EE9800266AB7EE006AB0EE667AA0EE007AD0EE87
:10EEA800006A37EE067A76EE866AC6EE077A84ED51
:10EEB800046A27EE807AB0EE498A27EE007A77EE68
:10EEC800075A84ED017AC4ED025A70EE005A84EDB7
:10EED800037AB8EE007AA5EE807A27EE877A67EE95
:10EEE800A67A84ED057AC4ED067ADFED567A98EDB8
:10EEF800047A27EE277AF0EE678AB5EEC07AF1EE4B
:10EF080010FA4CBF77EE487A77EE087A013517EE9B
:10EF1800900A01F0C5F8D8ED017A67EEA87AC7E93A
:10EF28000E01F5EEC07AF1EE10FA4CBF77EEC87A12
:10EF380077EE887A08F1040817EE900A01F0B0F825
:10EF4800032DC7E9080107F10807CED1A6F2DC5363
:10EF58001B042367E3676367C4F88030A367C4F8BA
:10EF680084300123A4F802902370D4F85490B4F9A3
:10EF78005280636A276A206FE26FD4F840C0D4F8E1
:10EF88008010C4F88020C9EB060606FA08F64FEA96
:10EF9800E67B734307FB0B332667A7FB06671F4413
:10EFA800636C656F60674FEAE27B53430CFB0B3E73
:10EFB800ACFB02237344B61A67EB0307E36AA26A41
:10EFC800C4F884104FEAE07B434302FB0B3EA2FBEC
:10EFD80000237344B6185F41E36CA06CB4F9502069
:10EFE800A5674FEAE17B4B4300FB0B33A0FB010114
:10EFF8001944636B361A206B4FEAE57B05FB03F374
:10F0080000FB0B3367EB0107A0FB050119448019CE
:10F01800794100F013FE08F1FF3201239340E067C5
:10F02800C01841EBE371424600F008FEBDEC048BCA
:10F038004844BDE8F88F00BF6F12833ADB0F4940A0
:10F04800F404B53F0000804B2DE9F8430024234B1E
:10F0580093F84460E0B2B0420CD203EB8003204A3C
:10F068005B6932F810101BB10B2801D8DB68984790
:10F078000134ECE71B4B1B685B032CD500242346AB
:10F08800E2B2B24227D2DFF8549009F114074FEAEE
:10F09800840857F8242055689D4214D02846FDF767
:10F0A80067F8EFF31283502282F3128828216A6AE4
:10F0B80001FB00900132C2666A6942F001026A618E
:10F0C800DBB283F3118857F808301B6800221A60F6
:10F0D80001342B46D4E7BDE8F88300BF082C002094
:10F0E800EC0F0020A82B002008B50E4B1B6813F46A
:10F0F800805F0D4B14BFD3F86021D3F8642193F8D7
:10F10800441092880023D8B2884204D2074820F8D5
:10F1180013200133F7E7FFF797FF3220BDE80840D7
:10F12800F9E500BFA82B0020082C0020EC0F0020D8
:10F138000A4B1A680A4B30B502F48052D3F8604182
:10F14800D3F8645100230AB1A18800E0A9880548D2
:10F1580020F8131001330C2BF5D130BDA82B00205B
:10F16800082C0020B228002070B5124D002421463A
:10F1780005F26910702285F8684103F04CFF2146BA
:10F18800D5F8DC310B4A0B4493F9020080B102F246
:10F1980069141E680E5108199C8884809B798371B4
:10F1A80092F8683107310133702982F86831E7D164
:10F1B80070BD00BF082C0020094B1A680E2303FB02
:10F1C8000020437AFF2B07D0064A12789A4203D9C7
:10F1D800054A32F8130000E0808800B2704700BF8B
:10F1E800F8150020B81E0020AC2B0020D0ED024AF4
:10F1F80091ED016A90ED015A91ED027AD0ED005A35
:10F20800D1ED007A66EE646AE5EE076A27EE657A64
:10F21800C2ED006AA4EEA77A67EEC57A82ED017A9C
:10F22800E5EE867AC2ED027A7047D0ED017A91ED6B
:10F23800017AD1ED026A91ED006A37EE877AD0ED56
:10F24800027A77EEA67AD0ED006A82ED017A76EE40
:10F25800866AC2ED027AC2ED006A704790ED017AC3
:10F26800D0ED027AD0ED006A20EE077A60EE277AB8
:10F2780026EE800A81ED017A81ED000AC1ED027A5D
:10F28800704700BF2DE9F04FA7490B7813F0010F25
:10F2980087B003F0040200F06B81002A40F075810A
:10F2A800A248066816F0806640F06F81980700F162
:10F2B8005F8143F004030B709D4B9E4C9E4F1B884F
:10F2C80023803B681B0340F11E819C4B80201E70ED
:10F2D800F9F710FA08B1FEF763FEA578012D40F0A2
:10F2E8001281974B93F8D61721B193F8D7270AB113
:10F2F800914203D3012283F8D62711E096460846A7
:10F30800BEF1000F06D090FBFEFC0EFB1C0C7046F5
:10F31800E646F5E791FBF0F183F8D61792FBF0F299
:10F3280083F8D72793F8D827012A82BF844A002177
:10F3380082F8D81793F8D897B9F1000F03D0B9F12C
:10F34800010F2ED036E08020F8F79CFE804688B367
:10F358008021F8F773FE98F806207A4BE07053F88E
:10F36800223098F90000B3F5613F0CBF0222002259
:10F3780002218DE806004A468021F8F759FD724BB4
:10F3880060601B684FF4FA7203EB4303B3FBF2F3BC
:10F398001BB1402BA8BF402300E00123237258B9BA
:10F3A80008E06A4BDB682BB1FEF76EFB10B940230F
:10F3B800237201E00023A5E000211422644803F031
:10F3C8002AFE644B236203F17402E833A362624BA2
:10F3D8005B491B88A4F88831604B62621B683A68F5
:10F3E80091F8D6E791F88491C3F3800C91F89231A3
:10F3F800002B4B79A3F11907C2F3402B02F40068E4
:10F40800C2F3400AC2F3C03218BF012278427841E1
:10F41800012B14BF03460123049391F8D7375048B2
:10F4280005909E454F4B07681B7803932CBF4FF000
:10F43800000E4FF0010E691EC9B24B1E132B3BD8AC
:10F44800DFE803F00C0C0C0C0C0C0C0C0A3D9D9F17
:10F45800273335121212373D049B93E0039B8B42EE
:10F46800B4BF0023012326E03B78022B0BD107EB26
:10F47800810353ED027AF5EE407AF1EE10FA14BFEB
:10F488000123002317E07B185B79003318BF0123A1
:10F4980011E0B8F1000F04D009F1FF3043424341B5
:10F4A80000E0434603F001036CE05B466AE0134664
:10F4B80068E0734666E013B101238B401E43142DA8
:10F4C80002D80135EDB2B6E7059BC4F88C6118681F
:10F4D80019218530F8F766FE0023C4F89431A4F8A2
:10F4E8009831A4F89A31C4F8A431C4F8A8311E4B55
:10F4F800D4F8A0211B68C4F8AC3184F89001C4F892
:10F508009C210223A370184B0D4A1B6892F8E02136
:10F518004FF47A7101FB0233144A0520136007B0D7
:10F52800BDE8F04FFFF79ABBD22F0020AC0F0020A8
:10F5380008100020E82D0020A82B0020BD1E002068
:10F54800D016002064570108241000201000002065
:10F55800F42D0020142E0020102B0020A40F0020D2
:10F56800E80F00204C2C0020D82B0020100F002082
:10F578005AB9012007B0BDE8F04FF8F769BE6346F5
:10F5880000E05346002B97D19BE707B0BDE8F08F0A
:10F5980010B5154A1378590725D523F004031370BD
:10F5A800124B1B681B0319D5114CA378A3F1080251
:10F5B800012A0BD8FF200021F9F746FD0D4B1B68E7
:10F5C800C4F8AC31FEF790FA0A2306E0012B05D9FE
:10F5D8000A2B03D0FEF76EFA0123A3700420BDE8BE
:10F5E8001040FFF73BBB10BDD22F0020A82B0020F6
:10F5F800E82D0020D82B00202DE9F04F2DED088BA9
:10F60800CB4D83B0044601932B8813F0020F0AEE0A
:10F61800102AF7EE009A4CD0149BC648DE89B0F940
:10F6280000309B1B03F2F31740F2E632974203D8EF
:10F63800002BB8BF5B4201E04FF4FA73B0F9022027
:10F64800921B02F2F31640F2E630864203D8002AF3
:10F65800B8BF524201E04FF4FA7294F84C0058B324
:10F668009342B8BF1346C3F5FA7307EE903A9FED7D
:10F67800B27AF8EEE77A6423C7EE877A93FBF0F361
:10F6880007EE103A77EEE97AB8EEC77AB0EE699AE3
:10F69800A7EE879AF7EE006AB5EEC09AF1EE10FA77
:10F6A8000AD4B4EE669AF1EE10FAC8BFB0EE669AC4
:10F6B80004E0B0EE699A01E09FEDA09AA04E01F136
:10F6C8000308A3464FF0000ABAF1020F18F8010F19
:10F6D8009C4F4FEA4A09F2EE04AA0ED100F10A0142
:10F6E800B7F904009FED987A00FB01F307EE903A12
:10F6F800F8EEE77AC7EE877A51E0B8EE4A7ADFED9E
:10F708008E6A37F91A1087EE267A07EE901A1AEEE3
:10F71800103AF8EEE77A5B4227EE877A07EE903ADE
:10F72800F8EEE77AB4EEE77AF1EE10FA08D4F8EEDC
:10F73800CA7AB4EEE77AF1EE10FAD8BFF0EE477A5B
:10F74800824F37F909302F8807EE103A019BB8EE3F
:10F75800C77A33F91A3077EEC77A07EE103AB8EE5F
:10F76800C77AFB0737EE877A87EE2A7A04D5D4ED75
:10F77800117A67EE277A12E0143001FB00F307EEE6
:10F78800903ADFED716AF8EEE77AB907C7EEA67A24
:10F7980042BFD4ED126A27EE267AE7EE097A6C4961
:10F7A8006C4F31F909306C499BED08BAD1ED046A08
:10F7B8009FED6A8A07EE103AB8EEC77A684BE7EE13
:10F7C800667A1AF80330BAF1020FF0EE678A67EE2C
:10F7D8008B7A0BEE103AB8EECBBAF0EE48BA27EEB9
:10F7E8008BBA8BEE08BA09D1B0EE4B0A5D48D7ED5B
:10F7F800000A1E21FAF77CF8B0EE40BAD7ED000AED
:10F808009BED0B7A68EEA07A67EE877A96ED007A20
:10F81800A7EEAA7ADFED547AB4EEE77AF1EE10FAA1
:10F82800F0EE47AA09D4DFED517AB4EE677AF1EE2B
:10F8380010FAC8BFF0EE67AA01E0F0EE67AA89EEF9
:10F84800A08A4B494FEA8A07394491ED000AC6ED70
:10F8580000AAC1ED008A38EEC00A94F8501020EED4
:10F86800080A21B1434800EBCA00FAF741F83C4BBB
:10F87800DBED0E7A13F80A3060EE277A00EE103AC4
:10F88800B8EEC00A27EE800ADFED3B7A80EE2B8ABD
:10F89800B4EEE78AF1EE10FA09D4DFED387AB4EE67
:10F8A800678AF1EE10FAC8BFB0EE678A01E0B0EEE1
:10F8B800678A3BEE2A0A30EE080A03F0BBFD30499E
:10F8C800B0F57A7FA8BF4FF47A708842B8BF08466F
:10F8D8002C4921F8090029880A0507D52A490978F9
:10F8E8004B0703D55FFA8AF0F6F762FCBDEECBBA98
:10F8F80026491BEE103AFDEEEAAA7B50BDEEC88AF7
:10F9080023491AEE903A0AF1010A7B50214918EE70
:10F91800103ABAF1030F7B500BF1040B06F1040601
:10F928007FF4D2AE03B0BDEC088BBDE8F08F00BF0A
:10F93800A80F0020AC2B00200000FA4300000000B4
:10F94800481F002094260020000048420410002090
:10F95800D20F0020A8260020082700200000C84257
:10F968009C260020A026002000007AC300007A43CD
:10F978009C2F0020C4260020000096C30000964358
:10F9880018FCFFFFDC260020D22F0020E4260020F0
:10F99800F0260020FC260020044B00221A605A6042
:10F9A800034B00221A605A60704700BF741F002082
:10F9B800541F002010B50B4C0123E3704FF48060F6
:10F9C800022384F82030FAF7CBFA074A074BD268AB
:10F9D8001B685178642212FB013363612388013369
:10F9E800238010BDDC2B00209C2F0020D82B00206A
:10F9F800022803D0431E584258417047064B1B68E3
:10FA08001B7823B1054B1868C0F3C0407047044BFE
:10FA18001878C0F380007047BC050020AC0F0020A8
:10FA2800D22F0020674B73B51878674DFFF7E0FFBA
:10FA38002B788342044620D0C8B1644B1B68E3B1DD
:10FA480093F9000002230093614B1B685B78003335
:10FA580018BF0123019304214FF416530022F8F72D
:10FA6800E7F95C4B186040B101232B7005E0594E53
:10FA78003068F8F7C9F934602C70574B574D18782F
:10FA8800FFF7B6FF2B788342044618D088B1544B51
:10FA98001B68A3B10022012493F9000000944FF4DD
:10FAA800964301920821F8F7C3F94E4B186028B91C
:10FAB80005E04C4E3068F8F7A7F934602C704A4BD3
:10FAC8004A4D1878FFF794FF2B78834204462E4658
:10FAD80042D0002837D0464B1A68002A3CD0D37948
:10FAE80092F90000434C002B08BF02230222009227
:10FAF800002254F8233001921021F8F799F93E4B6F
:10FB08000546186040B33D4C94F84A30022B0BD0A0
:10FB180094F89620022A01D14C3405E023B1002A3A
:10FB280004F14C0418BF0024354B1C6044B1204636
:10FB380000214C2203F06FFA0223256084F84A3032
:10FB48000123337008E02C4E3068FEF729FA30683C
:10FB5800F8F75AF934602C702A4B2B4D1878FFF7B8
:10FB680047FF2B788342044629D000B3274B1B68F4
:10FB78002BB3274A93F9000012685278002A0CBF69
:10FB8800082209220323009301924FF461432021A4
:10FB98000022F8F74DF91F4B186080B11E4A012367
:10FBA80013702B701D4B1A681D4B1A6007E0194E15
:10FBB8003068F8F729F9184B34601C702C7002B0C3
:10FBC80070BD00BFC4050020090D0020C00500203D
:10FBD800140D0020041F0020C5050020180D00206A
:10FBE8006C0D00205C0D0020D0050020720D002057
:10FBF800CC05002064570108740D00203816002039
:10FC0800780D0020DC050020800D0020D80500209C
:10FC1800D4050020840D0020880D0020D82B00205A
:10FC28008C0D002008B5044B1B7803F00503052B49
:10FC380001D1FFF759FAFEE7AC2F0020D0400B1C8A
:10FC48001141203A03D49C4613411843634652425B
:10FC580093401843704700BF81F0004102E000BFA5
:10FC680083F0004330B54FEA41044FEA430594EA74
:10FC7800050F08BF90EA020F1FBF54EA000C55EAAF
:10FC8800020C7FEA645C7FEA655C00F0E2804FEA80
:10FC98005454D4EB5555B8BF6D420CDD2C4480EA62
:10FCA800020281EA030382EA000083EA010180EA92
:10FCB800020281EA0303362D88BF30BD11F0004FE0
:10FCC8004FEA01314FF4801C4CEA113102D0404216
:10FCD80061EB410113F0004F4FEA03334CEA133351
:10FCE80002D0524263EB430394EA050F00F0A78069
:10FCF800A4F10104D5F1200E0DDB02FA0EFC22FA64
:10FD080005F2801841F1000103FA0EF2801843FA57
:10FD180005F359410EE0A5F120050EF1200E012A48
:10FD280003FA0EFC28BF4CF0020C43FA05F3C01886
:10FD380051EBE37101F0004507D54FF0000EDCF1FF
:10FD4800000C7EEB00006EEB0101B1F5801F1BD3A8
:10FD5800B1F5001F0CD349085FEA30004FEA3C0CAC
:10FD680004F101044FEA445212F5800F80F09A80A2
:10FD7800BCF1004F08BF5FEA500C50F1000041EBA6
:10FD8800045141EA050130BD5FEA4C0C404141EBAA
:10FD9800010111F4801FA4F10104E9D191F0000FD1
:10FDA80004BF01460020B1FA81F308BF2033A3F154
:10FDB8000B03B3F120020CDA0C3208DD02F1140C4B
:10FDC800C2F10C0201FA0CF021FA02F10CE002F186
:10FDD8001402D8BFC2F1200C01FA02F120FA0CFC7F
:10FDE800DCBF41EA0C019040E41AA2BF01EB0451C8
:10FDF800294330BD6FEA04041F3C1CDA0C340EDCC6
:10FE080004F11404C4F1200220FA04F001FA02F308
:10FE180040EA030021FA04F345EA030130BDC4F1C6
:10FE28000C04C4F1200220FA02F001FA04F340EABB
:10FE38000300294630BD21FA04F0294630BD94F06C
:10FE4800000F83F4801306BF81F480110134013D53
:10FE58004EE77FEA645C18BF7FEA655C29D094EAC4
:10FE6800050F08BF90EA020F05D054EA000C04BF42
:10FE78001946104630BD91EA030F1EBF002100202D
:10FE880030BD5FEA545C05D14000494128BF41F0CC
:10FE9800004130BD14F580043CBF01F5801130BD30
:10FEA80001F0004545F0FE4141F470014FF00000BB
:10FEB80030BD7FEA645C1ABF194610467FEA655C6C
:10FEC8001CBF0B46024650EA013406BF52EA03350E
:10FED80091EA030F41F4002130BD00BF90F0000FFC
:10FEE80004BF0021704730B54FF4806404F1320438
:10FEF8004FF000054FF0000150E700BF90F0000FF1
:10FF080004BF0021704730B54FF4806404F1320417
:10FF180010F0004548BF40424FF000013EE700BFE7
:10FF280042004FEAE2014FEA31014FEA02701FBF77
:10FF380012F07F4393F07F4F81F06051704792F049
:10FF4800000F14BF93F07F4F704730B54FF46074C3
:10FF580001F0004521F0004120E700BF50EA01020E
:10FF680008BF704730B54FF000050AE050EA0102BB
:10FF780008BF704730B511F0004502D5404261EB2B
:10FF880041014FF4806404F132045FEA915C3FF46C
:10FF9800DCAE4FF003025FEADC0C18BF03325FEA05
:10FFA800DC0C18BF033202EBDC02C2F1200300FABA
:10FFB80003FC20FA02F001FA03FE40EA0E0021FADF
:10FFC80002F11444C1E600BF4FEA4102B2F1E04336
:10FFD80024BFB3F5001CDCF1FE5C0DD901F0004C28
:10FFE8004FEAC0024CEA5070B2F1004F40EB830078
:08FFF80008BF20F00100704772
:020000040801F1
:1000000011F0804F21D113F13872BCBF01F00040D4
:10001000704741F480114FEA5252C2F11802C2F106
:10002000200C10FA0CF320FA02F018BF40F0010087
:100030004FEAC1234FEAD32303FA0CFC40EA0C0039
:1000400023FA02F34FEA4303CCE77FEA625307D176
:1000500050EA01331EBF4FF0FE4040F440007047AD
:1000600001F0004040F0FE4040F40000704700BF47
:100070007BB972B90029BEBF00204FF0004106E0F5
:1000800008BF00281CBF6FF000414FF0FF3000F0A8
:1000900073B882B0EC462DE9005000F03DF8DDF871
:1000A00004E002B00CBC704707EE900AF5EEC07A8F
:1000B000F1EE10FA01D400F009B808B580F0004064
:1000C00000F004F8404261EB410108BDD0B5FFF7F4
:1000D0002BFF00220E4B06460F4600F04FF800F0B3
:1000E0005FFA0446FFF7FEFE00220A4B00F046F8D6
:1000F00002460B4630463946FFF7B6FD00F050FA8F
:100100002346002242EA000210461946D0BD00BF35
:100110000000F03D0000F0412DE9F041069C15463D
:1001200006460F46984600F05BFA05FB01F300FB1C
:100130000838A5FB0023B21A434467EB0303C4E964
:100140000023BDE8F08100BF2DE9F041069C9046F8
:1001500006460F461D4600F091FB00FB05F5A0FB8F
:10016000082308FB0155B21A2B4467EB0303C4E9CB
:100170000023BDE8F08100BF704700BF70B54FF0AD
:10018000FF0C4CF4E06C1CEA11541DBF1CEA135523
:1001900094EA0C0F95EA0C0F00F0DEF82C4481EA8B
:1001A000030621EA4C5123EA4C5350EA013518BFAB
:1001B00052EA033541F4801143F4801338D0A0FB98
:1001C00002CE4FF00005E1FB02E506F00042E0FB45
:1001D00003E54FF00006E1FB03569CF0000F18BF4B
:1001E0004EF0010EA4F1FF04B6F5007F64F54074F3
:1001F00004D25FEA4E0E6D4146EB060642EAC62186
:1002000041EA55514FEAC52040EA5E504FEACE2EF2
:10021000B4F1FD0C88BFBCF5E06F1ED8BEF1004FF5
:1002200008BF5FEA500E50F1000041EB045170BD71
:1002300006F0004646EA010140EA020081EA0301B5
:10024000B4EB5C04C2BFD4EB0C0541EA045170BDB1
:1002500041F480114FF0000E013C00F3AB8014F12B
:10026000360FDEBF002001F0004170BDC4F1000474
:10027000203C35DA0C341BDC04F11404C4F12005F5
:1002800000FA05F320FA04F001FA05F240EA020050
:1002900001F0004221F0004110EBD37021FA04F686
:1002A00042EB06015EEA430E08BF20EAD37070BD40
:1002B000C4F10C04C4F1200500FA04F320FA05F09F
:1002C00001FA04F240EA020001F0004110EBD370A1
:1002D00041F100015EEA430E08BF20EAD37070BD11
:1002E000C4F1200500FA05F24EEA020E20FA04F3EA
:1002F00001FA05F243EA020321FA04F001F0004199
:1003000021FA04F220EA020000EBD3705EEA430E09
:1003100008BF20EAD37070BD94F0000F0FD101F038
:100320000046400041EB010111F4801F08BF013C71
:10033000F7D041EA060195F0000F18BF704703F0AF
:100340000046520043EB030313F4801F08BF013D36
:10035000F7D043EA0603704794EA0C0F0CEA1355F2
:1003600018BF95EA0C0F0CD050EA410618BF52EAAC
:100370004306D1D181EA030101F000414FF00000B2
:1003800070BD50EA410606BF1046194652EA4306C0
:1003900019D094EA0C0F02D150EA013613D195EA34
:1003A0000C0F05D152EA03361CBF104619460AD17C
:1003B00081EA030101F0004141F0FE4141F4700186
:1003C0004FF0000070BD41F0FE4141F4780170BD76
:1003D00070B54FF0FF0C4CF4E06C1CEA11541DBFDB
:1003E0001CEA135594EA0C0F95EA0C0F00F0A7F8DD
:1003F000A4EB050481EA030E52EA03354FEA01310A
:1004000000F088804FEA03334FF0805545EA13131C
:1004100043EA12634FEA022245EA111545EA1065E4
:100420004FEA00260EF000419D4208BF964244F17B
:10043000FD0404F5407402D25B084FEA3202B61A9A
:1004400065EB03055B084FEA32024FF480104FF46E
:10045000002CB6EB020E75EB030E22BFB61A7546E2
:1004600040EA0C005B084FEA3202B6EB020E75EB75
:10047000030E22BFB61A754640EA5C005B084FEADD
:100480003202B6EB020E75EB030E22BFB61A7546AA
:1004900040EA9C005B084FEA3202B6EB020E75EBB5
:1004A000030E22BFB61A754640EADC0055EA060E76
:1004B00018D04FEA051545EA16754FEA06164FEAB9
:1004C000C30343EA52734FEAC2025FEA1C1CC0D165
:1004D00011F4801F0BD141EA00014FF000004FF0F2
:1004E000004CB6E711F4801F04BF01430020B4F1B3
:1004F000FD0C88BFBCF5E06F3FF6AFAEB5EB030C6B
:1005000004BFB6EB020C5FEA500C50F1000041EB67
:10051000045170BD0EF0004E4EEA113114EB5C0434
:10052000C2BFD4EB0C0541EA045170BD41F4801107
:100530004FF0000E013C90E645EA060E8DE60CEA0F
:10054000135594EA0C0F08BF95EA0C0F3FF43BAF2C
:1005500094EA0C0F0AD150EA01347FF434AF95EAE3
:100560000C0F7FF425AF104619462CE795EA0C0FC7
:1005700006D152EA03353FF4FDAE1046194622E794
:1005800050EA410618BF52EA43067FF4C5AE50EA6E
:1005900041047FF40DAF52EA43057FF4EBAE12E75E
:1005A0004A0011D212F5001211D20DD56FF47873F2
:1005B000B3EB62520ED44FEAC12343F0004343EA47
:1005C000505323FA02F070474FF00000704750EA92
:1005D000013002D14FF0FF3070474FF000007047FC
:1005E00000292DE9F043C0F2A6800026002BC0F2BE
:1005F0009C80884694469E46154604460F46002B2E
:100600003DD18A4259D9B2FA82F33BB1C3F12002FB
:100610009F4020FA02F29D4017439C40290C220C77
:10062000B7FBF1FEA8B201FB1E7742EA074700FBC9
:100630000EF3BB420AD97F190EF1FF3280F005811B
:10064000BB4240F20281AEF1020E2F44FF1AA4B267
:10065000B7FBF1F301FB137744EA074700FB03F014
:10066000B84208D97F1903F1FF3280F0F080B84218
:1006700040F2ED80023B43EA0E43002203E08B424E
:100680000FD900221346341C18BF012460424FF0DA
:10069000000565EB45015840514000196941BDE82E
:1006A000F083B3FA83F2002A40F086808B4202D3B3
:1006B000844500F2DB800123E5E712B90123B3FB97
:1006C000F2F5B5FA85F000283BD1781B4FEA154EBC
:1006D0001FFA85FC0122B0FBFEF8210C0EFB180767
:1006E00041EA07470CFB08F3BB4207D97F1908F121
:1006F000FF3102D2BB4200F2BD808846FF1AA4B28D
:10070000B7FBFEF30EFB137744EA07470CFB03FC31
:10071000BC4507D97F1903F1FF3102D2BC4500F275
:10072000A7800B4643EA0843ADE752426FEA06064C
:1007300063EB43035DE7404261EB41014FF0FF365D
:1007400054E7C0F1200224FA02F107FA00F38540D1
:100750004FEA154ED7401943B7FBFEF20B0C0EFBC8
:1007600012771FFA85FC43EA07430CFB02F79F420E
:1007700004FA00F407D95B1902F1FF3074D29F42EA
:1007800072D9023A2B44DF1B89B2B7FBFEF80EFB8D
:10079000187341EA03430CFB08F79F4208D95B1921
:1007A00008F1FF315CD29F425AD9A8F102082B44CC
:1007B000D81B48EA02428EE7C2F120032CFA03F16B
:1007C0000EFA02FE20FA03F741EA0E0E08FA02F0D2
:1007D00028FA03F14FEA1E453843B1FBF5F8030C44
:1007E00005FB18111FFA8EF743EA014107FB08F3D6
:1007F0008B420CFA02FC09D911EB0E0108F1FF390A
:1008000030D28B422ED9A8F102087144C91A80B2A5
:10081000B1FBF5F305FB131140EA014107FB03F7B8
:100820008F4208D911EB0E0103F1FF3016D28F422F
:1008300014D9023B714443EA0843C91BA3FB0C894A
:10084000494509D305D000221DE79646FEE613462A
:1008500011E794404445F6D2013BF4E70346EAE74A
:100860008846A5E7C846D1E702468CE713460AE763
:10087000023B57E7A8F102082F443FE72DE9F0417A
:10088000002B44D18A42154604464FD9B2FA82F76A
:100890000E464FB1C7F12003B94020FA03F602FA21
:1008A00007F50E4300FA07F44FEA154E230CB6FB8A
:1008B000FEF0AFB20EFB106143EA014307FB00F10B
:1008C000994209D95B1900F1FF3280F0EC8099421E
:1008D00040F2E98002382B445A1AA4B2B2FBFEF36C
:1008E0000EFB132244EA024207FB03F7974208D9A2
:1008F000521903F1FF3180F0D880974240F2D58041
:10090000023B43EA004000263146BDE8F0818B42BD
:1009100047D8B3FA83F6002E48D18B4202D38242E5
:1009200000F2CD8001203146BDE8F08112B90125E9
:10093000B5FBF2F5B5FA85F8B8F1000F77D14A1B8F
:100940004FEA154EAFB20126B2FBFEF0230C0EFBB0
:10095000102143EA014107FB00F38B4207D94919F3
:1009600000F1FF3202D28B4200F2BA801046C91A5F
:10097000A4B2B1FBFEF30EFB131144EA014407FBE2
:1009800003F7A74208D9641903F1FF3280F08F8082
:10099000A74240F28C80023B43EA00403146BDE86A
:1009A000F081002630463146BDE8F081C6F12004D2
:1009B00022FA04F5B3402B4320FA04FC01FA06F7AF
:1009C00021FA04F54FEA134E4CEA0707B5FBFEF88F
:1009D000390C0EFB18551FFA83FC41EA05450CFB48
:1009E00008F1A94202FA06F204D9ED1808F1FF3421
:1009F00067D3A0466D1ABFB2B5FBFEF40EFB1455CB
:100A000047EA05410CFB04FC8C4504D9C91804F1E4
:100A1000FF355CD32C4644EA0844CCEB0101A4FB2F
:100A20000223994248D344D0204600266CE7C8F1FF
:100A3000200401FA08F305FA08F520FA04F7E1406A
:100A40004FEA154E1F43B1FBFEF63A0C0EFB161192
:100A50001FFA85FC42EA01430CFB06F29A4200FAB7
:100A600008F407D95B1906F1FF3137D29A4235D91C
:100A7000023E2B449B1ABFB2B3FBFEF00EFB1033B9
:100A800047EA03430CFB00F1994207D95B1900F1D7
:100A9000FF3221D299421FD902382B445A1A40EA18
:100AA0000646674650E7104616E70B4629E7134609
:100AB00072E7B0409042B7D2601E002624E730466D
:100AC00022E7A94295D9A8F102081D4492E78C4576
:100AD000A0D9023C19449EE71046DFE70E46C9E75D
:100AE0000238294443E700BF4FF0FF3C06E000BF57
:100AF0004FF0010C02E000BF4FF0010C4DF804CDA7
:100B00004FEA410C7FEA6C5C4FEA430C18BF7FEA66
:100B10006C5C1BD001B050EA410C0CBF52EA430C94
:100B200091EA030F02BF90EA020F0020704710F114
:100B3000000F91EA030F58BF994208BF90422CBFA3
:100B4000D8176FEAE37040F0010070474FEA410C9C
:100B50007FEA6C5C02D150EA013C07D14FEA430CBA
:100B60007FEA6C5CD6D152EA033CD3D05DF8040B2B
:100B7000704700BF8446104662468C46194663465D
:100B800000E000BF01B5FFF7B7FF002848BF10F134
:100B9000000F01BD4DF808EDFFF7F4FF0CBF012079
:100BA00000205DF808FB00BF4DF808EDFFF7EAFFF5
:100BB00034BF012000205DF808FB00BF4DF808EDB0
:100BC000FFF7E0FF94BF012000205DF808FB00BFA5
:100BD0004DF808EDFFF7CEFF94BF012000205DF82F
:100BE00008FB00BF4DF808EDFFF7C4FF34BF01203C
:100BF00000205DF808FB00BF114812490268006040
:100C00008A4218D0002103E00F4B5B584350043157
:100C10000E480F4B42189A42F6D30E4A02E00023C8
:100C200042F8043B0C4B9A42F9D3FCF7CDFE00F09E
:100C300019F87047FEE70948D0F800D0406800472F
:100C4000FC9F0020EFBEADDEE08201080000002026
:100C5000D8000020D8000020DC2F002000D8FF1F83
:100C6000FEE700002DE9804893B0EFF78DFAB34B13
:100C7000B34C1968237843B1B24B1B68CB1A002BD5
:100C8000A1BFB14A002323701370DFF810B3DBF863
:100C9000000042F2010303400BB9AA4A137107078F
:100CA00040F19381A94B1B681B7A062B00F27C81D3
:100CB000DFE813F0070007003400D40010013C0106
:100CC0003C01A34B1A78002A00F06E8100221A70B2
:100CD000A04B93F800E0A04B1B6893F800C09F4B1B
:100CE00093F8008002229E4EB35C43FA0EF303F0A9
:100CF0000F03634502F101090CD20B2B9FBFB55CBA
:100D000016F8096005EA080506EB05259CBF954E17
:100D100046F823500232102AE5D10CE1924B1A78A2
:100D2000002A00F0418100221A70904B904A93F8FB
:100D300002C093F803E05D780CF0070645EA06254B
:100D40000EF03F06760146EADC0615601D79566016
:100D50005E7993F806C0AD0045EA9E1506F0010ED7
:100D600045EA8E25956093F807E00CF00F05ED013C
:100D700045EA56050EF07F06D56036011D7A46EA33
:100D80001C1693F809C016616D000CF0030645EAC5
:100D9000DE1545EA462593F80AE05561DD7A0EF046
:100DA0001F06B601ED0046EA9C0645EA5E1593F87B
:100DB0000DC093F80EE0D5611D7B96610CF007061F
:100DC00045EA06250EF03F06760146EADC06156286
:100DD000DD7B56621E7C93F811C0AD0045EA9E157E
:100DE00006F0010E45EA8E25956293F812E00CF0AC
:100DF0000F05ED0145EA56050EF07F06360146EA7D
:100E00001C16D562DD7C166393F814C06D0045EAAC
:100E1000DE150CF0030693F815E045EA4625556308
:100E20000EF01F069D7DDB7DB60146EA9C06ED00B7
:100E300045EA5E159663DE07D5634CBF40F2147534
:100E4000AD2515649D074CBF40F21475AD2513F018
:100E5000080F556414BF03230123A6E0454A137805
:100E6000002B00F0A18000231370434ADFF830E12B
:100E70001678424D0EEB460CB5F800809CF80390B6
:100E80009CF8045045EA0925A84540F08D809EF85D
:100E90000150012D04D0812D40F08780032300E014
:100EA0002B46102E84BF10251570354D92F800E0AA
:100EB0000022D6B2764505F1020576D215F802CCAD
:100EC00015F8016C46EA0C26DFF8D8C02CF8126041
:100ED0000132EEE72B4B1A78002A65D000221A70F7
:100EE000294B1A78A82A1E465ED1DA7C002A5BD1EB
:100EF00006EB42059FED257A95F803E02B7903EB8D
:100F00000E2307EE903AF8EEE77A214BC7EE877A88
:100F10009FED207A77EEC77AFCEEE77A17EE905ACB
:100F200043F822500132082AE2D104E01A4B1A7821
:100F3000D2B300221A70012337E000BFB82F00207F
:100F4000400E0020E8050020410E0020A42B0020C8
:100F5000552A0020BA1E0020B41E0020BB1E00200F
:100F6000452A00203C290020C62A0020AD2A002066
:100F7000AC2900207D2A0020802A00207E2A002023
:100F8000842A0020762A0020612A0020CDCCCC4083
:100F90006C2900200080BB433A290020A82B0020A8
:100FA000812A00208C2900200023DF070DD58F4ADD
:100FB000012515718E4DC3F340032B7083F001039F
:100FC000237001F5C333A0331360460411D5894A59
:100FD00013780BB100251570844A13714BB10123AE
:100FE0002370834B00241C7001F5433303F5A07379
:100FF0001360C5070FD57D4B5C799A79A2420AD060
:101000007D4A9C71012515707C4A0025157001F5FB
:10101000C332A0321A60840409D50023784A32F81A
:101020001320002A41F0138701330C2BF6D16F4CAB
:10103000237923B9734B1B68CB1A002B55DBA368AC
:10104000CB1A13F1500F03D4684B1B7B002B4CD0F1
:10105000F1F710F8012363732373A37B634EE3B1AD
:10106000694B1B68580718D5684B1B68190703D4D0
:101070000820F8F769FF10E0654B1D8805F00805AA
:10108000ADB255B90820F8F76FFF624BB5611B6828
:101090003361614BF561DB88B382A37B534E002B38
:1010A00000F08982584B1B68DA0640F18482574B66
:1010B0001B689B0204D44FF40070F8F745FF7AE2F6
:1010C000534B1D8805F40075ADB2002D40F07382BE
:1010D0004FF40070F8F748FF4E4BB5611B68336161
:1010E0004D4BF561DB88B38265E2206A3F4D431CBE
:1010F0000128236200F04282022800F08F8000283D
:1011000040F05382404B1B685F0740F14E826B6A90
:10111000C91A0029C0F2498295F828306862012B6B
:101120000FD002D3022B1ED059E06B6B9847AB6BEC
:101130009847012385F82830EA8D6B6A13446B6267
:101140004DE0EB6B98472B6B98476B6AAA8D134465
:101150006B6205F144002B6C05F1480198470223AE
:1011600085F828303BE0696D2A6D097885F82800FC
:10117000561C8E4204BF012185F85810E16D6B6C3E
:10118000D5F84CE008BF0646481C032802BF1748A4
:10119000012580F86050154D05EB810108BF002046
:1011A0004B6694F86010E06569B105F164000BC806
:1011B0008842DEBF0D46014628468342A8BF03464B
:1011C0008B42B8BF0B460949266501EB82021367C3
:1011D00001EB8602126FC2EB0E0E7344E364FDF75F
:1011E00077FD636A18446062DFE100BFE805002014
:1011F000080000208E0F0020410E00200900002072
:10120000182A0020180E0020A40F0020AC0F002088
:10121000A80F00200C100020AC2B0020C64B1B6830
:101220005E0702D595F8582012B9D80640F1BD8165
:10123000D4F83031C14DC3EB010846F2A7139845ED
:1012400040F2B381BE4EC5F830113388DFEDBD9A50
:101250009FEDBD9ADFEDBD8AB7EE008A4BB36B6D93
:10126000D5F834211978EB6CDFEDB90A0820013983
:10127000B3FBF1F192FBF0F3D21A8B18C5F83431BD
:1012800093FBF0F300EE103AB8EEC00A80EE290AA4
:1012900002F07CF93388013B338038EE400AC5ED1B
:1012A0004F8A20EE090AC5ED508ABDEEC00A85EDD1
:1012B0004E0A656DE26C2B78DFEDA50A013BB2FBAF
:1012C000F3F300EE103AB8EE400A80EE290A02F07D
:1012D0005DF938EE400A20EE090A02F0AFF8D4F8C2
:1012E000383195ED017AD4ED517A9A4DC01A06EE57
:1012F000900AB8EEE60A78EE476AF8EEE77A20EE52
:10130000260AA7EE870A02F099F8B5F90030B5F978
:101310000210C4F8440183EAE372A2EBE37281EAAB
:10132000E173A3EBE1739A42B8BF1A468A4B12B23B
:101330003B211B6893FBF1F3B3F5967FC8BF4FF0D9
:10134000FF33FA2ADFBF07EE903AB8EEE77A07EEEE
:10135000902ADFED826A8249D5BFF8EEE77A4FF036
:10136000FF3376EEE77A0B60DFBF67EE277AC7EED2
:10137000A67AFDEEE77AC1ED007A0A68511EC62909
:1013800005D8801AC4F84801C4F8442126E0D4F8EE
:1013900048716A4BB1F5967FA0EB070002D3C3F802
:1013A00044011BE0C2F5967706EE907ADFED6D7A88
:1013B000F8EEE66AC6EEA76A07EE902AB8EEE77A7C
:1013C00007EE900A38EE666AF8EEE77A67EE867AFC
:1013D000E7EE267AFDEEE77AC3ED517A6248D4F85B
:1013E0004C31D0ED007AB8EE677ADFED607A67EEC7
:1013F000277A5BB1514A06EE103A92ED569AF8EE12
:10140000C96AB8EEC69A86EE899A01E09FED4F9AB6
:1014100094ED4F6AD4F85C91D4F84421D9ED035A85
:1014200069EE288AF6EE006A68EE878A26EE277A49
:1014300068EEA66A0023A6EEA77AC4F85031C4F875
:101440005431D4ED507AC4F8583137EE277A07EE8C
:10145000902A78EE656AF8EEE77A76EE288A67EEEB
:10146000A67AC4F84C31E7EE257A03603388C4EDE0
:101470004F8AC4ED507A002B40F09780D4F8603149
:10148000DFF8F4A0C4F86021D31AC62988BFFDEEA6
:10149000E77A07EE103A88BFCAED007AB8EEC77A4D
:1014A000DFED337A98BFCAF8002027EE277A07EEDF
:1014B000908AF8EE677A40F2DC53C7EE277A0A2169
:1014C0001E4EFDEEE77A17EE900A9842A8BF184626
:1014D000A3F6B8339842B8BF1846F8F74BFCD9EDDD
:1014E000027A07EE100A38EE678AB8EEC70A20EED5
:1014F000080AA8EEA70A84ED4F0A01F09FFF052114
:101500008046F8F737FC1B4B94ED598A18602B88FE
:1015100003F21F339BB240F23E62934207D80D4B59
:101520005B8803F21F339BB2934241F2D9840023BC
:10153000E36184ED599A38E0A40F0020E80500200B
:10154000CC2F002080E6C547D048874A0000000025
:10155000B1DC423E04100020000000200000614485
:10156000141000200000C842B02F0020BD3786357F
:1015700000247449101000200C100020B44B1B688C
:10158000DA0612D5B34B1A68D5F86C313C339A425F
:101590000BD3D5F87061C5F86C21AF4D3388AB61C2
:1015A0000B20FDF7B1FB33882B85236A032BC2BFC9
:1015B000AA4B00221A62FDF78BFBA94B1860A94BBE
:1015C0000BADDB68284698479DF82C3033B9A44B07
:1015D000A2681B689B1A642B00F1BD87DFF8B892E4
:1015E0009F4BD9F800201B689F4E1344A360002333
:1015F00023739E4B30681988643001B10221FBF7D8
:101600007DFAFDF765FB964BD9ED007A1860D4F8AA
:101610007431974F9FED977ADFF88082C4F8740198
:10162000F8EE677AC31A3B8067EE877A924BC8ED73
:10163000007A2A4603F1080C186859689646AEE805
:101640000300083363457246F6D118689B88CEF8CC
:101650000000AEF80430BDF838908849002200231D
:101660008E4618463EF802CF35F803A02EF802CC7D
:1016700002330C2B1CFB0A00F4D1DFF824E23EF805
:1016800012308B8113FB09004FF4807390FBF3F051
:101690002EF812000132032A01F10E01DFD1F1F719
:1016A00065FD3B88DFF8B491D8ED000AB4F8A2518B
:1016B00000EE103A09F5D270B8EE400A0121F8F7B1
:1016C0001BF9BCEEC00A637B8DED040ABDF8100067
:1016D000B5FBF0F0451CADB2A4F8AC5133B3B9F88A
:1016E000AE31049300235D49654ABDF810A032F87D
:1016F000138001F5DC7C01F5D8793CF813E039F86A
:1017000013202CF81380CEEB080E12FB0AF20FFA0E
:1017100085FA92FBFAF2724429F813200133042B64
:10172000E1D100234B73A1F8AE0104E0B9F8AE316A
:10173000013BA9F8AE31B4F8AE01484A03B2002B20
:101740004FF0000313DDB2F9AC514E4931F81320CC
:10175000083112FB00F231F8131092FBF5F28A1AED
:10176000474921F813200133042BEED101E0A2F800
:10177000AE310123A373444BDFF8F0901B68DFF810
:10178000DCA0DFF8E48013F4801FB9F8003000F02B
:10179000BA8003F400639DB2002D40F0A0803B4B63
:1017A0001B785B0740F19B804FF40060F8F7DCFB8F
:1017B000D8F80020CAF8C0211378B2F85C10D4F829
:1017C000C0014FF47A72A3F1020E51433A8891FBA3
:1017D000F2F12F4ADEF10003C1F1000143EB0E03E9
:1017E00089B292F800C08AF8C4311F46A4F8C61125
:1017F00000F1200E2B4690F8575090F854200DB170
:10180000AA4204D8BCF1030F04D8022B02D1002550
:1018100080F857501F4D002F44D007EE902A9EEDC0
:10182000007AF2EE046AF8EEE77A27EE267AB4EE52
:10183000E77AF1EE10FA44BFC7EEA67ACEED007A51
:10184000DEED007AFDEEE77A17EE902A30E000BF79
:10185000A40F0020D82B002000040048E805002039
:10186000B82F002008270020E80F0020A80F002034
:10187000980F0020BD378635184A01086007002000
:101880009426002098070020AC0F0020D22F0020C3
:101890004C2C0020B007002024100020A826002097
:1018A000D20F002090F801A0924538BF42704278D4
:1018B000920125F81320BD4A02F5E7754FF0000AA2
:1018C00025F813A002F5EA75013025F8131001334D
:1018D000032B0EF1040E8ED1012382F8DA31B9F810
:1018E0000030180519D4B24B1B7803F0040303F041
:1018F000FF0593B994F8DA317BB1F8F7DFFDAB4B14
:1019000083F8DA5109E0190507D5A94B1B785A0766
:1019100003D54FF40060F8F717FBA64BA64D1B68E4
:10192000A64F13F0140F70D0B9F8003003F402730F
:10193000002B6AD0A24B1B7803F0100303F0FF00CA
:1019400043B16B8897F9EC21B4F91C1001FB023309
:101950006B805AE0D4F8DC11944B91F803E0994A7B
:101960008978BEF1000F23D0B3F914E0B2F9062054
:10197000CEEB020A8AEAEA7CACEBEA7C8C450CDD11
:10198000986172454FF0010083F8E001C8BF4942F9
:10199000EB8889B21944E98037E093F8E02122B15D
:1019A000894A83F8E00112681A61E369734421E00F
:1019B000B3F91400B2F90620121A82EAE27CACEB09
:1019C000E27C8C450ADD022192FBF1F27F490A603C
:1019D000012283F8E82183F8E02109E093F8E0216F
:1019E00032B1794A83F8E8E112681A6183F8E0E1DC
:1019F000E3690344D4F8E4110A884988934203DB7D
:101A00008B42A8BF0B461A46EA80714B1B78ABB1DC
:101A10006C4BB3F90620B7F898319A420EDC674B4D
:101A20005B79012B01D0192B02D197F8E6212AB955
:101A30000E2B03D0082B1CBF0023AB80D8F800303E
:101A400093F82481B8F1000F47D0B9F800309B0714
:101A500043D09FED608ADFED607A88EE088AB4EEAD
:101A6000E78AF1EE10FA34D9B7EE000A30EE480AF0
:101A700001F02EFF9FED597ADFED597AE8EE077AF3
:101A80009FED587AA8EE277ADFED577AE8EE077ACD
:101A900020EE270AD4ED7B7A20EE270A01F0CEFC57
:101AA000B0F5617FA8BF4FF4617007EE900AB8EE01
:101AB000E70ADFED4E7A80EE270AF8F7DDF907EE48
:101AC000908AF8EEE77A27EE800A01F0B7FC80B240
:101AD00000E00020EB881844E880454B3068B7F8F8
:101AE0006C210093434B1E68434B196800F164035B
:101AF000B047424B42481B78032B18D9D4F8F02149
:101B00005788B7F5FA7F12D2B5F90460B0F904E04E
:101B100086EAE67CACEBE67C7942CCEB01029645AA
:101B200004DB07EB0C027245A8BF72468280ED8889
:101B3000D4F8F0E1334946880788B0F904C00020A2
:101B4000984201F1100161D29EF9012051ED045A31
:101B5000DFF8B48052420CFB02F207EE902A3AB250
:101B600006EE902A2AB206EE102A32B2B8EEE77AD2
:101B700007EE902AF8EEE77AB8EEC66A67EEA57A25
:101B800051ED065AE6EE257AF8EEE66A11ED056AA1
:101B9000E6EE867A51ED036AE7EE267AFDEEE77A05
:101BA00017EE902A28F810200130C9E7E805002038
:101BB000D22F0020A40F002094260020D016002051
:101BC00000280020AC2B00200C100020B42F002097
:101BD0000A000020000000008FC2753C306E99BCE6
:101BE0002716983D843459BEA40DC93FEFB6B044C2
:101BF0005818002060000020281000204C2C0020E5
